 pdfbench

 Timestamp is 4a8b394d (Wed Aug 19 07:29:17 2009)

 Preferred load address is 00400000

 Start         Length     Name                   Class
 0001:00000000 00096b3bH .text                   CODE
 0002:00000000 00000148H .idata$5                DATA
 0002:00000148 00000004H .CRT$XCA                DATA
 0002:0000014c 00000004H .CRT$XCZ                DATA
 0002:00000150 00000004H .CRT$XIA                DATA
 0002:00000154 00000014H .CRT$XIC                DATA
 0002:00000168 00000004H .CRT$XIY                DATA
 0002:0000016c 00000004H .CRT$XIZ                DATA
 0002:00000170 00000004H .CRT$XPA                DATA
 0002:00000174 00000004H .CRT$XPX                DATA
 0002:00000178 00000004H .CRT$XPXA               DATA
 0002:0000017c 00000004H .CRT$XPZ                DATA
 0002:00000180 00000004H .CRT$XTA                DATA
 0002:00000184 00000004H .CRT$XTZ                DATA
 0002:00000190 00155f98H .rdata                  DATA
 0002:00156128 0000004eH .rdata$debug            DATA
 0002:00156180 0000000cH .rdata$sxdata           DATA
 0002:0015618c 00000004H .rtc$IAA                DATA
 0002:00156190 00000004H .rtc$IZZ                DATA
 0002:00156194 00000004H .rtc$TAA                DATA
 0002:00156198 00000004H .rtc$TZZ                DATA
 0002:001561a0 000005d4H .xdata$x                DATA
 0002:00156774 00000014H .idata$2                DATA
 0002:00156788 00000014H .idata$3                DATA
 0002:0015679c 00000148H .idata$4                DATA
 0002:001568e4 000005caH .idata$6                DATA
 0002:00156eae 00000000H .edata                  DATA
 0003:00000000 000378e0H .data                   DATA
 0003:000378e0 0000362cH .bss                    DATA

  Address         Publics by Value              Rva+Base       Lib:Object

 0000:00000000       __except_list              00000000     <absolute>
 0000:00000003       ___safe_se_handler_count   00000003     <absolute>
 0000:00000000       ___ImageBase               00400000     <linker-defined>
 0001:00000000       _adler32                   00401000 f   adler32.obj
 0001:0000021a       _crc32                     0040121a f   crc32.obj
 0001:0000047a       _inflateReset              0040147a f   inflate.obj
 0001:000004d1       _inflateInit2_             004014d1 f   inflate.obj
 0001:0000064d       _inflate                   0040164d f   inflate.obj
 0001:00001845       _inflateEnd                00402845 f   inflate.obj
 0001:0000187c       _zcalloc                   0040287c f   zutil.obj
 0001:0000188d       _zcfree                    0040288d f   zutil.obj
 0001:00001898       _inflate_fast              00402898 f   inffast.obj
 0001:00001c74       _inflate_table             00402c74 f   inftrees.obj
 0001:00003897       __tr_stored_block          00404897 f   trees.obj
 0001:00003981       __tr_flush_block           00404981 f   trees.obj
 0001:00004004       _FT_Stream_Open            00405004 f   ftsystem.obj
 0001:00004266       _FT_Get_Glyph              00405266 f   ftglyph.obj
 0001:00004306       _FT_Done_Glyph             00405306 f   ftglyph.obj
 0001:00004328       _FT_Bitmap_Copy            00405328 f   ftbitmap.obj
 0001:000043d8       _FT_Bitmap_Done            004053d8 f   ftbitmap.obj
 0001:0000440b       _FT_Init_FreeType          0040540b f   ftinit.obj
 0001:00004499       _FT_Done_FreeType          00405499 f   ftinit.obj
 0001:00009430       _FT_RoundFix               0040a430 f   ftbase.obj
 0001:0000944f       _FT_MulDiv                 0040a44f f   ftbase.obj
 0001:000094a5       _FT_MulDiv_No_Round        0040a4a5 f   ftbase.obj
 0001:000094ef       _FT_MulFix                 0040a4ef f   ftbase.obj
 0001:00009524       _FT_DivFix                 0040a524 f   ftbase.obj
 0001:0000957a       _FT_Matrix_Invert          0040a57a f   ftbase.obj
 0001:000095f6       _FT_Matrix_Multiply_Scaled 0040a5f6 f   ftbase.obj
 0001:000096c7       _FT_Vector_Transform_Scaled 0040a6c7 f   ftbase.obj
 0001:00009725       _FT_SqrtFixed              0040a725 f   ftbase.obj
 0001:00009754       _ft_corner_orientation     0040a754 f   ftbase.obj
 0001:000097c7       _ft_corner_is_flat         0040a7c7 f   ftbase.obj
 0001:00009816       _FT_GlyphLoader_New        0040a816 f   ftbase.obj
 0001:0000983b       _FT_GlyphLoader_Rewind     0040a83b f   ftbase.obj
 0001:00009857       _FT_GlyphLoader_Reset      0040a857 f   ftbase.obj
 0001:000098b6       _FT_GlyphLoader_Done       0040a8b6 f   ftbase.obj
 0001:00009916       _FT_GlyphLoader_CheckPoints 0040a916 f   ftbase.obj
 0001:00009a2d       _FT_GlyphLoader_CheckSubGlyphs 0040aa2d f   ftbase.obj
 0001:00009a81       _FT_GlyphLoader_Prepare    0040aa81 f   ftbase.obj
 0001:00009aa0       _FT_GlyphLoader_Add        0040aaa0 f   ftbase.obj
 0001:00009ae6       _FT_GlyphLoader_CopyPoints 0040aae6 f   ftbase.obj
 0001:00009b86       _FT_Get_Sfnt_Name          0040ab86 f   ftbase.obj
 0001:00009c72       _ft_service_list_lookup    0040ac72 f   ftbase.obj
 0001:00009cc0       _FT_Stream_New             0040acc0 f   ftbase.obj
 0001:00009d70       _FT_Stream_Free            0040ad70 f   ftbase.obj
 0001:00009dfc       _ft_glyphslot_free_bitmap  0040adfc f   ftbase.obj
 0001:00009e34       _ft_glyphslot_alloc_bitmap 0040ae34 f   ftbase.obj
 0001:00009f2f       _FT_New_GlyphSlot          0040af2f f   ftbase.obj
 0001:00009fad       _FT_Done_GlyphSlot         0040afad f   ftbase.obj
 0001:00009ff7       _FT_Set_Transform          0040aff7 f   ftbase.obj
 0001:0000a106       _FT_Load_Glyph             0040b106 f   ftbase.obj
 0001:0000a61c       _FT_Open_Face              0040b61c f   ftbase.obj
 0001:0000a85b       _FT_Done_Face              0040b85b f   ftbase.obj
 0001:0000a8b2       _FT_New_Size               0040b8b2 f   ftbase.obj
 0001:0000a962       _FT_Done_Size              0040b962 f   ftbase.obj
 0001:0000a9f4       _FT_Match_Size             0040b9f4 f   ftbase.obj
 0001:0000aabb       _ft_synthesize_vertical_metrics 0040babb f   ftbase.obj
 0001:0000ab42       _FT_Select_Metrics         0040bb42 f   ftbase.obj
 0001:0000abc1       _FT_Request_Metrics        0040bbc1 f   ftbase.obj
 0001:0000ad7c       _FT_Select_Size            0040bd7c f   ftbase.obj
 0001:0000adb5       _FT_Request_Size           0040bdb5 f   ftbase.obj
 0001:0000ae28       _FT_Set_Char_Size          0040be28 f   ftbase.obj
 0001:0000ae85       _FT_Set_Pixel_Sizes        0040be85 f   ftbase.obj
 0001:0000aedf       _FT_Select_Charmap         0040bedf f   ftbase.obj
 0001:0000af33       _FT_Set_Charmap            0040bf33 f   ftbase.obj
 0001:0000af96       _FT_CMap_New               0040bf96 f   ftbase.obj
 0001:0000b05f       _FT_Get_Char_Index         0040c05f f   ftbase.obj
 0001:0000b07a       _FT_Get_Next_Char          0040c07a f   ftbase.obj
 0001:0000b0b1       _FT_Get_Name_Index         0040c0b1 f   ftbase.obj
 0001:0000b116       _FT_Get_Glyph_Name         0040c116 f   ftbase.obj
 0001:0000b191       _FT_Load_Sfnt_Table        0040c191 f   ftbase.obj
 0001:0000b1d2       _FT_Get_CMap_Format        0040c1d2 f   ftbase.obj
 0001:0000b212       _FT_Activate_Size          0040c212 f   ftbase.obj
 0001:0000b22c       _FT_Lookup_Renderer        0040c22c f   ftbase.obj
 0001:0000b372       _FT_Set_Renderer           0040c372 f   ftbase.obj
 0001:0000b3e2       _FT_Render_Glyph_Internal  0040c3e2 f   ftbase.obj
 0001:0000b4f9       _FT_Add_Module             0040c4f9 f   ftbase.obj
 0001:0000b679       _FT_Get_Module             0040c679 f   ftbase.obj
 0001:0000b6d9       _FT_Get_Module_Interface   0040c6d9 f   ftbase.obj
 0001:0000b6f0       _ft_module_get_service     0040c6f0 f   ftbase.obj
 0001:0000b742       _FT_Remove_Module          0040c742 f   ftbase.obj
 0001:0000b793       _FT_New_Library            0040c793 f   ftbase.obj
 0001:0000b7fc       _FT_Done_Library           0040c7fc f   ftbase.obj
 0001:0000b893       _ft_stub_set_char_sizes    0040c893 f   ftbase.obj
 0001:0000b8f0       _ft_stub_set_pixel_sizes   0040c8f0 f   ftbase.obj
 0001:0000b938       _FT_Outline_Decompose      0040c938 f   ftbase.obj
 0001:0000bba3       _FT_Outline_New_Internal   0040cba3 f   ftbase.obj
 0001:0000bc56       _FT_Outline_New            0040cc56 f   ftbase.obj
 0001:0000bc75       _FT_Outline_Check          0040cc75 f   ftbase.obj
 0001:0000bcc3       _FT_Outline_Copy           0040ccc3 f   ftbase.obj
 0001:0000bd31       _FT_Outline_Done_Internal  0040cd31 f   ftbase.obj
 0001:0000bd86       _FT_Outline_Get_CBox       0040cd86 f   ftbase.obj
 0001:0000be05       _FT_Outline_Translate      0040ce05 f   ftbase.obj
 0001:0000be35       _FT_Vector_Transform       0040ce35 f   ftbase.obj
 0001:0000be82       _FT_Outline_Transform      0040ce82 f   ftbase.obj
 0001:0000beab       _FT_Outline_Get_Orientation 0040ceab f   ftbase.obj
 0001:0000c0ee       _FT_Stream_Seek            0040d0ee f   ftbase.obj
 0001:0000c116       _FT_Stream_Read            0040d116 f   ftbase.obj
 0001:0000c12f       _FT_Stream_ReadAt          0040d12f f   ftbase.obj
 0001:0000c191       _FT_Stream_ExtractFrame    0040d191 f   ftbase.obj
 0001:0000c1ae       _FT_Stream_ReleaseFrame    0040d1ae f   ftbase.obj
 0001:0000c1c6       _FT_Stream_EnterFrame      0040d1c6 f   ftbase.obj
 0001:0000c257       _FT_Stream_ExitFrame       0040d257 f   ftbase.obj
 0001:0000c274       _FT_Stream_GetChar         0040d274 f   ftbase.obj
 0001:0000c285       _FT_Stream_GetShort        0040d285 f   ftbase.obj
 0001:0000c2a3       _FT_Stream_GetShortLE      0040d2a3 f   ftbase.obj
 0001:0000c2c0       _FT_Stream_GetLong         0040d2c0 f   ftbase.obj
 0001:0000c2f4       _FT_Stream_GetLongLE       0040d2f4 f   ftbase.obj
 0001:0000c329       _FT_Stream_ReadChar        0040d329 f   ftbase.obj
 0001:0000c370       _FT_Stream_ReadShort       0040d370 f   ftbase.obj
 0001:0000c3c5       _FT_Stream_ReadShortLE     0040d3c5 f   ftbase.obj
 0001:0000c41a       _FT_Stream_ReadOffset      0040d41a f   ftbase.obj
 0001:0000c479       _FT_Stream_ReadLong        0040d479 f   ftbase.obj
 0001:0000c4e1       _FT_Stream_ReadLongLE      0040d4e1 f   ftbase.obj
 0001:0000c54a       _FT_Stream_ReadFields      0040d54a f   ftbase.obj
 0001:0000c879       _ft_mem_alloc              0040d879 f   ftbase.obj
 0001:0000c8b3       _ft_mem_qalloc             0040d8b3 f   ftbase.obj
 0001:0000c8dd       _ft_mem_realloc            0040d8dd f   ftbase.obj
 0001:0000c92f       _ft_mem_qrealloc           0040d92f f   ftbase.obj
 0001:0000c9c3       _ft_mem_free               0040d9c3 f   ftbase.obj
 0001:0000c9d5       _ft_mem_strdup             0040d9d5 f   ftbase.obj
 0001:0000ca2c       _ft_mem_strcpyn            0040da2c f   ftbase.obj
 0001:0000ca4e       _FT_List_Find              0040da4e f   ftbase.obj
 0001:0000ca63       _FT_List_Add               0040da63 f   ftbase.obj
 0001:0000ca7b       _FT_List_Remove            0040da7b f   ftbase.obj
 0001:0000ca96       _FT_List_Finalize          0040da96 f   ftbase.obj
 0001:0000f755       _FTC_Manager_LookupSize    00410755 f   ftcache.obj
 0001:0000f857       _FTC_Manager_LookupFace    00410857 f   ftcache.obj
 0001:0000fa3b       _ftc_node_destroy          00410a3b f   ftcache.obj
 0001:00027877       _ps_hints_apply            00428877 f   pshinter.obj
 0001:00036742       _TT_RunIns                 00437742 f   truetype.obj
 0001:0003e605       _jpeg_abort                0043f605 f   jcomapi.obj
 0001:0003e631       _jpeg_destroy              0043f631 f   jcomapi.obj
 0001:0003e646       _jpeg_alloc_quant_table    0043f646 f   jcomapi.obj
 0001:0003e65e       _jpeg_alloc_huff_table     0043f65e f   jcomapi.obj
 0001:0003e676       _jpeg_CreateDecompress     0043f676 f   jdapimin.obj
 0001:0003e8e7       _jpeg_read_header          0043f8e7 f   jdapimin.obj
 0001:0003e93f       _jpeg_consume_input        0043f93f f   jdapimin.obj
 0001:0003e9d7       _jpeg_finish_decompress    0043f9d7 f   jdapimin.obj
 0001:0003ea7a       _jpeg_start_decompress     0043fa7a f   jdapistd.obj
 0001:0003ec04       _jpeg_read_scanlines       0043fc04 f   jdapistd.obj
 0001:0003f827       _jinit_d_coef_controller   00440827 f   jdcoefct.obj
 0001:0003fcf6       _jinit_color_deconverter   00440cf6 f   jdcolor.obj
 0001:0003ffd8       _jinit_inverse_dct         00440fd8 f   jddctmgr.obj
 0001:00040182       _jpeg_make_d_derived_tbl   00441182 f   jdhuff.obj
 0001:00040440       _jpeg_fill_bit_buffer      00441440 f   jdhuff.obj
 0001:0004053a       _jpeg_huff_decode          0044153a f   jdhuff.obj
 0001:000409f2       _jinit_huff_decoder        004419f2 f   jdhuff.obj
 0001:00041452       _jinit_d_main_controller   00442452 f   jdmainct.obj
 0001:000429c9       _jpeg_resync_to_restart    004439c9 f   jdmarker.obj
 0001:00042b36       _jpeg_calc_output_dimensions 00443b36 f   jdmaster.obj
 0001:00043579       _jinit_merged_upsampler    00444579 f   jdmerge.obj
 0001:000440b7       _jinit_phuff_decoder       004450b7 f   jdphuff.obj
 0001:00044339       _jinit_d_post_controller   00445339 f   jdpostct.obj
 0001:000447eb       _jinit_upsampler           004457eb f   jdsample.obj
 0001:00044af1       _jpeg_std_error            00445af1 f   jerror.obj
 0001:00044b39       _jpeg_idct_float           00445b39 f   jidctflt.obj
 0001:00044f76       _jpeg_idct_ifast           00445f76 f   jidctfst.obj
 0001:0004533b       _jpeg_idct_islow           0044633b f   jidctint.obj
 0001:0004581a       _jpeg_idct_4x4             0044681a f   jidctred.obj
 0001:00045af5       _jpeg_idct_2x2             00446af5 f   jidctred.obj
 0001:00045ca4       _jpeg_idct_1x1             00446ca4 f   jidctred.obj
 0001:00046665       _jinit_1pass_quantizer     00447665 f   jquant1.obj
 0001:0004761e       _jinit_2pass_quantizer     0044861e f   jquant2.obj
 0001:00047728       _jcopy_sample_rows         00448728 f   jutils.obj
 0001:00048085       _jinit_memory_mgr          00449085 f   jmemmgr.obj
 0001:0004820a       _jbig2_error               0044920a f   jbig2.obj
 0001:00048283       _jbig2_ctx_new             00449283 f   jbig2.obj
 0001:00048334       _jbig2_get_int32           00449334 f   jbig2.obj
 0001:0004834e       _jbig2_data_in             0044934e f   jbig2.obj
 0001:0004867d       _jbig2_ctx_free            0044967d f   jbig2.obj
 0001:0004875e       _jbig2_word_stream_buf_new 0044975e f   jbig2.obj
 0001:00048839       _jbig2_arith_new           00449839 f   jbig2_arith.obj
 0001:0004889b       _jbig2_arith_decode        0044989b f   jbig2_arith.obj
 0001:0004890d       _jbig2_arith_iaid_ctx_new  0044990d f   jbig2_arith_iaid.obj
 0001:0004893d       _jbig2_arith_iaid_decode   0044993d f   jbig2_arith_iaid.obj
 0001:0004897f       _jbig2_arith_iaid_ctx_free 0044997f f   jbig2_arith_iaid.obj
 0001:00048993       _jbig2_arith_int_ctx_new   00449993 f   jbig2_arith_int.obj
 0001:000489b3       _jbig2_arith_int_decode    004499b3 f   jbig2_arith_int.obj
 0001:00048aba       _jbig2_huffman_new         00449aba f   jbig2_huffman.obj
 0001:00048aea       _jbig2_huffman_skip        00449aea f   jbig2_huffman.obj
 0001:00048b4f       _jbig2_huffman_advance     00449b4f f   jbig2_huffman.obj
 0001:00048bad       _jbig2_huffman_get_bits    00449bad f   jbig2_huffman.obj
 0001:00048c1d       _jbig2_huffman_get         00449c1d f   jbig2_huffman.obj
 0001:00048d23       _jbig2_build_huffman_table 00449d23 f   jbig2_huffman.obj
 0001:00048fed       _jbig2_release_huffman_table 00449fed f   jbig2_huffman.obj
 0001:000499cb       _jbig2_decode_generic_region 0044a9cb f   jbig2_generic.obj
 0001:00049ac2       _jbig2_immediate_generic_region 0044aac2 f   jbig2_generic.obj
 0001:0004a042       _jbig2_decode_refinement_region 0044b042 f   jbig2_refinement.obj
 0001:0004a0b4       _jbig2_region_find_referred 0044b0b4 f   jbig2_refinement.obj
 0001:0004a11c       _jbig2_refinement_region   0044b11c f   jbig2_refinement.obj
 0001:0004a3e0       _jbig2_image_new           0044b3e0 f   jbig2_image.obj
 0001:0004a468       _jbig2_image_release       0044b468 f   jbig2_image.obj
 0001:0004a481       _jbig2_image_resize        0044b481 f   jbig2_image.obj
 0001:0004a4db       _jbig2_image_compose_unopt 0044b4db f   jbig2_image.obj
 0001:0004a76e       _jbig2_image_compose       0044b76e f   jbig2_image.obj
 0001:0004a9bc       _jbig2_image_get_pixel     0044b9bc f   jbig2_image.obj
 0001:0004a9f1       _jbig2_image_set_pixel     0044b9f1 f   jbig2_image.obj
 0001:0004aa3c       _jbig2_parse_segment_header 0044ba3c f   jbig2_segment.obj
 0001:0004abf3       _jbig2_free_segment        0044bbf3 f   jbig2_segment.obj
 0001:0004ac6c       _jbig2_find_segment        0044bc6c f   jbig2_segment.obj
 0001:0004acb8       _jbig2_get_region_segment_info 0044bcb8 f   jbig2_segment.obj
 0001:0004acf0       _jbig2_parse_extension_segment 0044bcf0 f   jbig2_segment.obj
 0001:0004ad77       _jbig2_parse_segment       0044bd77 f   jbig2_segment.obj
 0001:0004af21       _jbig2_sd_new              0044bf21 f   jbig2_symbol_dict.obj
 0001:0004af72       _jbig2_sd_release          0044bf72 f   jbig2_symbol_dict.obj
 0001:0004afbd       _jbig2_sd_count_referred   0044bfbd f   jbig2_symbol_dict.obj
 0001:0004aff9       _jbig2_sd_list_referred    0044bff9 f   jbig2_symbol_dict.obj
 0001:0004b082       _jbig2_sd_cat              0044c082 f   jbig2_symbol_dict.obj
 0001:0004bd5a       _jbig2_symbol_dictionary   0044cd5a f   jbig2_symbol_dict.obj
 0001:0004c0ca       _jbig2_decode_text_region  0044d0ca f   jbig2_text.obj
 0001:0004c887       _jbig2_parse_text_region   0044d887 f   jbig2_text.obj
 0001:0004d567       _jbig2_decode_generic_mmr  0044e567 f   jbig2_mmr.obj
 0001:0004d689       _jbig2_parse_page_info     0044e689 f   jbig2_page.obj
 0001:0004d891       _jbig2_parse_end_of_stripe 0044e891 f   jbig2_page.obj
 0001:0004d8eb       _jbig2_complete_page       0044e8eb f   jbig2_page.obj
 0001:0004d949       _jbig2_parse_end_of_page   0044e949 f   jbig2_page.obj
 0001:0004d992       _jbig2_page_add_result     0044e992 f   jbig2_page.obj
 0001:0004da11       _jbig2_page_out            0044ea11 f   jbig2_page.obj
 0001:0004da64       _jbig2_release_page        0044ea64 f   jbig2_page.obj
 0001:0004dace       _jbig2_metadata_free       0044eace f   jbig2_metadata.obj
 0001:0004db6f       _jbig2_metadata_add        0044eb6f f   jbig2_metadata.obj
 0001:0004dbfe       _jbig2_parse_comment_ascii 0044ebfe f   jbig2_metadata.obj
 0001:0004e094       _fz_scalepixmaptile        0044f094 f   imagescale.obj
 0001:0004e380       _fz_scalepixmap            0044f380 f   imagescale.obj
 0001:0004e93c       _fz_fillpath               0044f93c f   pathfill.obj
 0001:0004eb14       _fz_newpixmap              0044fb14 f   pixmap.obj
 0001:0004eb97       _fz_newpixmapwithrect      0044fb97 f   pixmap.obj
 0001:0004ebba       _fz_droppixmap             0044fbba f   pixmap.obj
 0001:0004ebcb       _fz_clearpixmap            0044fbcb f   pixmap.obj
 0001:0004ec17       _fz_newglyphcache          0044fc17 f   glyphcache.obj
 0001:0004ed0b       _fz_dropglyphcache         0044fd0b f   glyphcache.obj
 0001:0004ee29       _fz_renderglyph            0044fe29 f   glyphcache.obj
 0001:0004f64e       _fz_newgel                 0045064e f   pathscan.obj
 0001:0004f6e1       _fz_boundgel               004506e1 f   pathscan.obj
 0001:0004f7b2       _fz_insertgel              004507b2 f   pathscan.obj
 0001:0004f9c9       _fz_sortgel                004509c9 f   pathscan.obj
 0001:0004faa7       _fz_newael                 00450aa7 f   pathscan.obj
 0001:0004fdb0       _fz_scanconvert            00450db0 f   pathscan.obj
 0001:000514c1       _fz_rendershade            004524c1 f   meshdraw.obj
 0001:00052893       _fz_strokepath             00453893 f   pathstroke.obj
 0001:00052e01       _fz_dashpath               00453e01 f   pathstroke.obj
 0001:00052fe4       _fz_newrenderer            00453fe4 f   render.obj
 0001:000530f3       _fz_droprenderer           004540f3 f   render.obj
 0001:00054843       _fz_rendertree             00455843 f   render.obj
 0001:000548f0       _fz_rendertreeover         004558f0 f   render.obj
 0001:00054962       _fz_malloc                 00455962 f   base_memory.obj
 0001:00054994       _fz_realloc                00455994 f   base_memory.obj
 0001:000549cb       _fz_warn                   004559cb f   base_error.obj
 0001:00054a10       _fz_throwimp               00455a10 f   base_error.obj
 0001:00054a64       _fz_rethrowimp             00455a64 f   base_error.obj
 0001:00054ab8       _fz_catchimp               00455ab8 f   base_error.obj
 0001:00054b45       _fz_newhash                00455b45 f   base_hash.obj
 0001:00054bd9       _fz_resizehash             00455bd9 f   base_hash.obj
 0001:00054ce9       _fz_hashfind               00455ce9 f   base_hash.obj
 0001:00054d42       _fz_hashinsert             00455d42 f   base_hash.obj
 0001:00054e17       _fz_hashremove             00455e17 f   base_hash.obj
 0001:00054f26       _fz_concat                 00455f26 f   base_matrix.obj
 0001:00054f96       _fz_translate              00455f96 f   base_matrix.obj
 0001:00054fb4       _fz_invertmatrix           00455fb4 f   base_matrix.obj
 0001:0005503f       _fz_transformpoint         0045603f f   base_matrix.obj
 0001:00055074       _fz_transformaabb          00456074 f   base_matrix.obj
 0001:00055308       _fz_roundrect              00456308 f   base_rect.obj
 0001:0005535e       _fz_intersectrects         0045635e f   base_rect.obj
 0001:0005542e       _fz_mergerects             0045642e f   base_rect.obj
 0001:00055500       _fz_intersectirects        00456500 f   base_rect.obj
 0001:0005557c       _fz_strsep                 0045657c f   base_string.obj
 0001:000555a3       _fz_strlcpy                004565a3 f   base_string.obj
 0001:000555d0       _fz_strlcat                004565d0 f   base_string.obj
 0001:0005562d       _fz_dropnode               0045662d f   node_misc1.obj
 0001:000556b2       _fz_boundnode              004566b2 f   node_misc1.obj
 0001:0005585e       _fz_issolidnode            0045685e f   node_misc1.obj
 0001:00055870       _fz_newovernode            00456870 f   node_misc2.obj
 0001:000558b5       _fz_boundblendnode         004568b5 f   node_misc2.obj
 0001:000558b5       _fz_boundovernode          004568b5 f   node_misc2.obj
 0001:00055933       _fz_newmasknode            00456933 f   node_misc2.obj
 0001:00055978       _fz_boundmasknode          00456978 f   node_misc2.obj
 0001:000559f0       _fz_newblendnode           004569f0 f   node_misc2.obj
 0001:00055a4a       _fz_newtransformnode       00456a4a f   node_misc2.obj
 0001:00055a9e       _fz_boundtransformnode     00456a9e f   node_misc2.obj
 0001:00055afd       _fz_newsolidnode           00456afd f   node_misc2.obj
 0001:00055b7b       _fz_newimagenode           00456b7b f   node_misc2.obj
 0001:00055bc8       _fz_boundimagenode         00456bc8 f   node_misc2.obj
 0001:00055c15       _fz_newshadenode           00456c15 f   node_misc2.obj
 0001:00055c62       _fz_boundshadenode         00456c62 f   node_misc2.obj
 0001:00056176       _fz_optimizetree           00457176 f   node_optimize.obj
 0001:000561a5       _fz_newpathnode            004571a5 f   node_path.obj
 0001:00056211       _fz_clonepathnode          00457211 f   node_path.obj
 0001:00056325       _fz_moveto                 00457325 f   node_path.obj
 0001:00056382       _fz_lineto                 00457382 f   node_path.obj
 0001:00056403       _fz_curveto                00457403 f   node_path.obj
 0001:000564c5       _fz_curvetov               004574c5 f   node_path.obj
 0001:00056514       _fz_closepath              00457514 f   node_path.obj
 0001:000565cc       _fz_boundpathnode          004575cc f   node_path.obj
 0001:000567d4       _fz_newdash                004577d4 f   node_path.obj
 0001:00056831       _fz_newtextnode            00457831 f   node_text.obj
 0001:000568b2       _fz_clonetextnode          004578b2 f   node_text.obj
 0001:00056985       _fz_boundtextnode          00457985 f   node_text.obj
 0001:00056b02       _fz_addtext                00457b02 f   node_text.obj
 0001:00056bc0       _fz_newtree                00457bc0 f   node_tree.obj
 0001:00056bff       _fz_droptree               00457bff f   node_tree.obj
 0001:00056c1f       _fz_boundtree              00457c1f f   node_tree.obj
 0001:00056c5d       _fz_insertnodelast         00457c5d f   node_tree.obj
 0001:00056c75       _fz_removenode             00457c75 f   node_tree.obj
 0001:00056caf       _fz_dropcolorspace         00457caf f   res_colorspace.obj
 0001:00056cd1       _fz_stdconvcolor           00457cd1 f   res_colorspace.obj
 0001:00056d52       _fz_stdconvpixmap          00457d52 f   res_colorspace.obj
 0001:00056e8f       _fz_dropfont               00457e8f f   res_font.obj
 0001:00056f29       _ft_errorstring            00457f29 f   res_font.obj
 0001:00056ffd       _fz_newfontfromfile        00457ffd f   res_font.obj
 0001:000570c2       _fz_newfontfrombuffer      004580c2 f   res_font.obj
 0001:00057192       _fz_renderftglyph          00458192 f   res_font.obj
 0001:00057413       _fz_newtype3font           00458413 f   res_font.obj
 0001:000574fb       _fz_rendert3glyph          004584fb f   res_font.obj
 0001:00057691       _fz_dropimage              00458691 f   res_image.obj
 0001:000576ba       _fz_dropshade              004586ba f   res_shade.obj
 0001:0005779c       _rijndael_setup            0045879c f   crypt_aes.obj
 0001:00057b66       _rijndael_ecb_decrypt      00458b66 f   crypt_aes.obj
 0001:0005804f       _aes_cbc_decrypt           0045904f f   crypt_aes.obj
 0001:0005810e       _fz_aesdecrypt             0045910e f   crypt_aes.obj
 0001:00058131       _fz_arc4init               00459131 f   crypt_arc4.obj
 0001:00058195       _fz_arc4encrypt            00459195 f   crypt_arc4.obj
 0001:000588ca       _fz_md5init                004598ca f   crypt_md5.obj
 0001:000588ee       _fz_md5update              004598ee f   crypt_md5.obj
 0001:00058984       _fz_md5final               00459984 f   crypt_md5.obj
 0001:000589f9       _fz_newa85d                004599f9 f   filt_a85d.obj
 0001:00058a64       _fz_processa85d            00459a64 f   filt_a85d.obj
 0001:00058c86       _fz_newaesfilter           00459c86 f   filt_aes.obj
 0001:00058d0b       _fz_processaesfilter       00459d0b f   filt_aes.obj
 0001:00058e23       _fz_newahxd                00459e23 f   filt_ahxd.obj
 0001:00058e8e       _fz_processahxd            00459e8e f   filt_ahxd.obj
 0001:00058f62       _fz_newarc4filter          00459f62 f   filt_arc4.obj
 0001:00058fcd       _fz_processarc4filter      00459fcd f   filt_arc4.obj
 0001:0005912b       _fz_newfaxd                0045a12b f   filt_faxd.obj
 0001:0005932a       _fz_dropfaxd               0045a32a f   filt_faxd.obj
 0001:0005977f       _fz_processfaxd            0045a77f f   filt_faxd.obj
 0001:000599f8       _fz_newflated              0045a9f8 f   filt_flate.obj
 0001:00059ae4       _fz_dropflated             0045aae4 f   filt_flate.obj
 0001:00059b10       _fz_processflated          0045ab10 f   filt_flate.obj
 0001:00059c3f       _fz_newlzwd                0045ac3f f   filt_lzwd.obj
 0001:00059d60       _fz_processlzwd            0045ad60 f   filt_lzwd.obj
 0001:00059f2f       _fz_newnullfilter          0045af2f f   filt_null.obj
 0001:00059f8f       _fz_processnullfilter      0045af8f f   filt_null.obj
 0001:0005a027       _fz_newpipeline            0045b027 f   filt_pipeline.obj
 0001:0005a0dc       _fz_droppipeline           0045b0dc f   filt_pipeline.obj
 0001:0005a0fd       _fz_processpipeline        0045b0fd f   filt_pipeline.obj
 0001:0005a21e       _fz_newpredict             0045b21e f   filt_predict.obj
 0001:0005a3d1       _fz_droppredict            0045b3d1 f   filt_predict.obj
 0001:0005a788       _fz_processpredict         0045b788 f   filt_predict.obj
 0001:0005a89d       _fz_newrld                 0045b89d f   filt_rld.obj
 0001:0005a8fb       _fz_droprld                0045b8fb f   filt_rld.obj
 0001:0005a8fb       _fz_dropa85d               0045b8fb f   filt_a85d.obj
 0001:0005a8fb       _fz_droparc4filter         0045b8fb f   filt_arc4.obj
 0001:0005a8fb       _fz_droplzwd               0045b8fb f   filt_lzwd.obj
 0001:0005a8fb       _fz_dropahxd               0045b8fb f   filt_ahxd.obj
 0001:0005a8fb       _fz_dropnullfilter         0045b8fb f   filt_null.obj
 0001:0005a8fb       _fz_dropaesfilter          0045b8fb f   filt_aes.obj
 0001:0005a8fc       _fz_processrld             0045b8fc f   filt_rld.obj
 0001:0005a9c9       _fz_newarray               0045b9c9 f   obj_array.obj
 0001:0005aa55       _fz_arraylen               0045ba55 f   obj_array.obj
 0001:0005aa74       _fz_arrayget               0045ba74 f   obj_array.obj
 0001:0005aaf6       _fz_arraypush              0045baf6 f   obj_array.obj
 0001:0005ab74       _fz_freearray              0045bb74 f   obj_array.obj
 0001:0005abed       _fz_newdict                0045bbed f   obj_dict.obj
 0001:0005acf0       _fz_dictlen                0045bcf0 f   obj_dict.obj
 0001:0005ad29       _fz_dictgetkey             0045bd29 f   obj_dict.obj
 0001:0005ad56       _fz_dictgetval             0045bd56 f   obj_dict.obj
 0001:0005ae12       _fz_dictgets               0045be12 f   obj_dict.obj
 0001:0005ae45       _fz_dictget                0045be45 f   obj_dict.obj
 0001:0005ae6d       _fz_dictgetsa              0045be6d f   obj_dict.obj
 0001:0005ae90       _fz_dictput                0045be90 f   obj_dict.obj
 0001:0005afe6       _fz_dictputs               0045bfe6 f   obj_dict.obj
 0001:0005b054       _fz_freedict               0045c054 f   obj_dict.obj
 0001:0005bb8a       _fz_packobj                0045cb8a f   obj_parse.obj
 0001:0005bbd1       _fz_newnull                0045cbd1 f   obj_simple.obj
 0001:0005bc0c       _fz_newbool                0045cc0c f   obj_simple.obj
 0001:0005bc4c       _fz_newint                 0045cc4c f   obj_simple.obj
 0001:0005bc91       _fz_newreal                0045cc91 f   obj_simple.obj
 0001:0005bcd6       _fz_newstring              0045ccd6 f   obj_simple.obj
 0001:0005bd35       _fz_newname                0045cd35 f   obj_simple.obj
 0001:0005bd98       _fz_newindirect            0045cd98 f   obj_simple.obj
 0001:0005bdef       _fz_dropobj                0045cdef f   obj_simple.obj
 0001:0005be39       _fz_isindirect             0045ce39 f   obj_simple.obj
 0001:0005be4c       _fz_isnull                 0045ce4c f   obj_simple.obj
 0001:0005be68       _fz_isbool                 0045ce68 f   obj_simple.obj
 0001:0005be85       _fz_isint                  0045ce85 f   obj_simple.obj
 0001:0005bea2       _fz_isreal                 0045cea2 f   obj_simple.obj
 0001:0005bebf       _fz_isstring               0045cebf f   obj_simple.obj
 0001:0005bedc       _fz_isname                 0045cedc f   obj_simple.obj
 0001:0005bef9       _fz_isarray                0045cef9 f   obj_simple.obj
 0001:0005bf16       _fz_isdict                 0045cf16 f   obj_simple.obj
 0001:0005bf3c       _fz_tobool                 0045cf3c f   obj_simple.obj
 0001:0005bf5d       _fz_toint                  0045cf5d f   obj_simple.obj
 0001:0005bf92       _fz_toreal                 0045cf92 f   obj_simple.obj
 0001:0005bfc3       _fz_toname                 0045cfc3 f   obj_simple.obj
 0001:0005bfe5       _fz_tostrbuf               0045cfe5 f   obj_simple.obj
 0001:0005c007       _fz_tostrlen               0045d007 f   obj_simple.obj
 0001:0005c029       _fz_tonum                  0045d029 f   obj_simple.obj
 0001:0005c03b       _fz_togen                  0045d03b f   obj_simple.obj
 0001:0005c04d       _fz_resolveindirect        0045d04d f   obj_simple.obj
 0001:0005c0ce       _fz_objcmp                 0045d0ce f   obj_simple.obj
 0001:0005c29e       _fz_objkindstr             0045d29e f   obj_simple.obj
 0001:0005c31a       _fz_newbuffer              0045d31a f   stm_buffer.obj
 0001:0005c390       _fz_dropbuffer             0045d390 f   stm_buffer.obj
 0001:0005c3ab       _fz_growbuffer             0045d3ab f   stm_buffer.obj
 0001:0005c428       _fz_rewindbuffer           0045d428 f   stm_buffer.obj
 0001:0005c46e       _fz_process                0045d46e f   stm_filter.obj
 0001:0005c4ec       _fz_dropfilter             0045d4ec f   stm_filter.obj
 0001:0005c503       _fz_readline               0045d503 f   stm_misc.obj
 0001:0005c615       _fz_readall                0045d615 f   stm_misc.obj
 0001:0005c6d4       _fz_dropstream             0045d6d4 f   stm_open.obj
 0001:0005c73c       _fz_openrfile              0045d73c f   stm_open.obj
 0001:0005c805       _fz_openrfilter            0045d805 f   stm_open.obj
 0001:0005c88a       _fz_openrbuffer            0045d88a f   stm_open.obj
 0001:0005c8ca       _fz_readimp                0045d8ca f   stm_read.obj
 0001:0005caa9       _fz_tell                   0045daa9 f   stm_read.obj
 0001:0005cb1e       _fz_seek                   0045db1e f   stm_read.obj
 0001:0005ccd5       _fz_read                   0045dcd5 f   stm_read.obj
 0001:0005cd4a       _fz_readerror              0045dd4a f   stm_read.obj
 0001:0005cd76       _fz_readbytex              0045dd76 f   stm_read.obj
 0001:0005cdcf       _fz_peekbytex              0045ddcf f   stm_read.obj
 0001:0005cf01       _fz_newdctd                0045df01 f   filt_dctd.obj
 0001:0005d064       _fz_dropdctd               0045e064 f   filt_dctd.obj
 0001:0005d0a7       _fz_processdctd            0045e0a7 f   filt_dctd.obj
 0001:0005d29f       _fz_newjbig2d              0045e29f f   filt_jbig2d.obj
 0001:0005d319       _fz_dropjbig2d             0045e319 f   filt_jbig2d.obj
 0001:0005d334       _fz_processjbig2d          0045e334 f   filt_jbig2d.obj
 0001:0005d467       _fz_newjpxd                0045e467 f   filt_jpxd_opj.obj
 0001:0005d5be       _fz_dropjpxd               0045e5be f   filt_jpxd_opj.obj
 0001:0005d60c       _fz_processjpxd            0045e60c f   filt_jpxd_opj.obj
 0001:0005d88e       _pdf_newlink               0045e88e f   pdf_annot.obj
 0001:0005d8dd       _pdf_droplink              0045e8dd f   pdf_annot.obj
 0001:0005d973       _pdf_loadlink              0045e973 f   pdf_annot.obj
 0001:0005dc14       _pdf_loadannots            0045ec14 f   pdf_annot.obj
 0001:0005dd1e       _pdf_initgstate            0045ed1e f   pdf_build.obj
 0001:0005de43       _pdf_setcolorspace         0045ee43 f   pdf_build.obj
 0001:0005df39       _pdf_setcolor              0045ef39 f   pdf_build.obj
 0001:0005e0f6       _pdf_setpattern            0045f0f6 f   pdf_build.obj
 0001:0005e1a0       _pdf_setshade              0045f1a0 f   pdf_build.obj
 0001:0005e20b       _pdf_buildstrokepath       0045f20b f   pdf_build.obj
 0001:0005e7ca       _pdf_addshade              0045f7ca f   pdf_build.obj
 0001:0005e9e9       _pdf_addfillshape          0045f9e9 f   pdf_build.obj
 0001:0005eaeb       _pdf_addstrokeshape        0045faeb f   pdf_build.obj
 0001:0005ebed       _pdf_addclipmask           0045fbed f   pdf_build.obj
 0001:0005ec8a       _pdf_addtransform          0045fc8a f   pdf_build.obj
 0001:0005ece2       _pdf_showimage             0045fce2 f   pdf_build.obj
 0001:0005ee26       _pdf_showpath              0045fe26 f   pdf_build.obj
 0001:0005f01e       _pdf_flushtext             0046001e f   pdf_build.obj
 0001:0005f54b       _pdf_showtext              0046054b f   pdf_build.obj
 0001:0005f699       _pdf_newcmap               00460699 f   pdf_cmap.obj
 0001:0005f714       _pdf_dropcmap              00460714 f   pdf_cmap.obj
 0001:0005f753       _pdf_setusecmap            00460753 f   pdf_cmap.obj
 0001:0005f79f       _pdf_addcodespace          0046079f f   pdf_cmap.obj
 0001:0005f93c       _pdf_maprangetorange       0046093c f   pdf_cmap.obj
 0001:0005f984       _pdf_maponetomany          00460984 f   pdf_cmap.obj
 0001:0005fa7a       _pdf_sortcmap              00460a7a f   pdf_cmap.obj
 0001:0005fcf0       _pdf_lookupcmap            00460cf0 f   pdf_cmap.obj
 0001:0005fd72       _pdf_decodecmap            00460d72 f   pdf_cmap.obj
 0001:000608c7       _pdf_loadcolorspace        004618c7 f   pdf_colorspace1.obj
 0001:000610de       _pdf_convpixmap            004620de f   pdf_colorspace2.obj
 0001:00061201       _pdf_convcolor             00462201 f   pdf_colorspace2.obj
 0001:00061897       _pdf_newdecrypt            00462897 f   pdf_crypt.obj
 0001:00061b9f       _pdf_freecrypt             00462b9f f   pdf_crypt.obj
 0001:00061e4f       _pdf_setpassword           00462e4f f   pdf_crypt.obj
 0001:00061e94       _pdf_setuserpassword       00462e94 f   pdf_crypt.obj
 0001:00061f03       _pdf_setownerpassword      00462f03 f   pdf_crypt.obj
 0001:00062054       _pdf_cryptobj              00463054 f   pdf_crypt.obj
 0001:0006221e       _pdf_cryptstream           0046321e f   pdf_crypt.obj
 0001:00062438       _pdf_logxref               00463438 f   pdf_debug.obj
 0001:00062453       _pdf_logrsrc               00463453 f   pdf_debug.obj
 0001:0006246e       _pdf_logfont               0046346e f   pdf_debug.obj
 0001:00062489       _pdf_logimage              00463489 f   pdf_debug.obj
 0001:000624a4       _pdf_logshade              004634a4 f   pdf_debug.obj
 0001:000624bf       _pdf_logpage               004634bf f   pdf_debug.obj
 0001:00062695       _pdf_dropfont              00463695 f   pdf_font.obj
 0001:0006270d       _pdf_newfontdesc           0046370d f   pdf_font.obj
 0001:00063e4f       _pdf_loadfontdescriptor    00464e4f f   pdf_font.obj
 0001:00064074       _pdf_loadfont              00465074 f   pdf_font.obj
 0001:0006429d       _pdf_lookupagl             0046529d f   pdf_fontagl.obj
 0001:00064499       _pdf_loadencoding          00465499 f   pdf_fontenc.obj
 0001:0006458e       _pdf_addhmtx               0046558e f   pdf_fontmtx.obj
 0001:00064608       _pdf_addvmtx               00465608 f   pdf_fontmtx.obj
 0001:000646b2       _pdf_endhmtx               004656b2 f   pdf_fontmtx.obj
 0001:00064707       _pdf_endvmtx               00465707 f   pdf_fontmtx.obj
 0001:0006475c       _pdf_gethmtx               0046575c f   pdf_fontmtx.obj
 0001:000647a7       _pdf_getvmtx               004657a7 f   pdf_fontmtx.obj
 0001:00068193       _pdf_dropfunction          00469193 f   pdf_function.obj
 0001:00068212       _pdf_loadfunction          00469212 f   pdf_function.obj
 0001:00068609       _pdf_evalfunction          00469609 f   pdf_function.obj
 0001:00068829       _pdf_dropimage             00469829 f   pdf_image.obj
 0001:00068849       _pdf_loadinlineimage       00469849 f   pdf_image.obj
 0001:00068dc6       _pdf_loadimage             00469dc6 f   pdf_image.obj
 0001:000694b0       _pdf_loadtile              0046a4b0 f   pdf_image.obj
 0001:000696fc       _pdf_newcsi                0046a6fc f   pdf_interpret.obj
 0001:000699b4       _pdf_dropcsi               0046a9b4 f   pdf_interpret.obj
 0001:0006c911       _pdf_runcsi                0046d911 f   pdf_interpret.obj
 0001:0006d3fc       _pdf_lex                   0046e3fc f   pdf_lex.obj
 0001:0006d7ed       _pdf_lookupdest            0046e7ed f   pdf_nametree.obj
 0001:0006e8e7       _pdf_loadobjstm            0046f8e7 f   pdf_open.obj
 0001:0006edc0       _pdf_loadxref              0046fdc0 f   pdf_open.obj
 0001:0006f211       _pdf_loadpage              00470211 f   pdf_page.obj
 0001:0006f7f8       _pdf_getpagecount          004707f8 f   pdf_pagetree.obj
 0001:0006fc91       _pdf_getpageobject         00470c91 f   pdf_pagetree.obj
 0001:0006fd4f       _pdf_torect                00470d4f f   pdf_parse.obj
 0001:0006fe1d       _pdf_tomatrix              00470e1d f   pdf_parse.obj
 0001:0006fe96       _pdf_parsearray            00470e96 f   pdf_parse.obj
 0001:00070185       _pdf_parsedict             00471185 f   pdf_parse.obj
 0001:0007056d       _pdf_parsestmobj           0047156d f   pdf_parse.obj
 0001:0007069e       _pdf_parseindobj           0047169e f   pdf_parse.obj
 0001:00070a01       _pdf_droppattern           00471a01 f   pdf_pattern.obj
 0001:00070a1f       _pdf_loadpattern           00471a1f f   pdf_pattern.obj
 0001:000717ce       _pdf_repairxref            004727ce f   pdf_repair.obj
 0001:00071de6       _pdf_loadresources         00472de6 f   pdf_resources.obj
 0001:0007242d       _pdf_loadshadefunction     0047342d f   pdf_shade.obj
 0001:0007280c       _pdf_loadshade             0047380c f   pdf_shade.obj
 0001:00072a29       _pdf_loadtype1shade        00473a29 f   pdf_shade1.obj
 0001:0007314c       _pdf_loadtype2shade        0047414c f   pdf_shade1.obj
 0001:000738fb       _pdf_loadtype3shade        004748fb f   pdf_shade1.obj
 0001:00073cf2       _pdf_loadtype4shade        00474cf2 f   pdf_shade4.obj
 0001:000742bf       _pdf_loadtype5shade        004752bf f   pdf_shade4.obj
 0001:00075231       _pdf_loadtype6shade        00476231 f   pdf_shade4.obj
 0001:000756e3       _pdf_loadtype7shade        004766e3 f   pdf_shade4.obj
 0001:00075d02       _pdf_newstore              00476d02 f   pdf_store.obj
 0001:00075d6d       _pdf_emptystore            00476d6d f   pdf_store.obj
 0001:00075e0c       _pdf_storeitem             00476e0c f   pdf_store.obj
 0001:00075efa       _pdf_finditem              00476efa f   pdf_store.obj
 0001:00075f6d       _pdf_removeitem            00476f6d f   pdf_store.obj
 0001:00076894       _pdf_buildinlinefilter     00477894 f   pdf_stream.obj
 0001:00076a57       _pdf_openstream            00477a57 f   pdf_stream.obj
 0001:00076ba6       _pdf_loadstream            00477ba6 f   pdf_stream.obj
 0001:00076d0d       _pdf_loadtype3font         00477d0d f   pdf_type3.obj
 0001:00077438       _pdf_loadtounicode         00478438 f   pdf_unicode.obj
 0001:0007777b       _pdf_loadxobject           0047877b f   pdf_xobject.obj
 0001:00077a98       _pdf_dropxobject           00478a98 f   pdf_xobject.obj
 0001:00077ac4       _pdf_newxref               00478ac4 f   pdf_xref.obj
 0001:00077b39       _pdf_closexref             00478b39 f   pdf_xref.obj
 0001:00077bc4       _pdf_flushxref             00478bc4 f   pdf_xref.obj
 0001:00077c05       _pdf_decryptxref           00478c05 f   pdf_xref.obj
 0001:00077c75       _pdf_cacheobject           00478c75 f   pdf_xref.obj
 0001:00077e5d       _pdf_loadobject            00478e5d f   pdf_xref.obj
 0001:00078c47       _pdf_loadbuiltinfont2      00479c47 f   pdf_fontfilems.obj
 0001:000791b4       _pdf_loadbuiltinfont       0047a1b4 f   pdf_fontfilems.obj
 0001:000791da       _pdf_loadsystemfont        0047a1da f   pdf_fontfilems.obj
 0001:0007922b       _pdf_loadembeddedfont      0047a22b f   pdf_fontfilems.obj
 0001:000792e7       _pdf_loadembeddedcmap      0047a2e7 f   pdf_cmap_load.obj
 0001:0007951d       _pdf_newidentitycmap       0047a51d f   pdf_cmap_load.obj
 0001:00079615       _pdf_loadsystemcmap        0047a615 f   pdf_cmap_load.obj
 0001:0007a404       _pdf_parsecmap             0047b404 f   pdf_cmap_parse.obj
 0001:0007a706       _bio_read                  0047b706 f   bio.obj
 0001:0007a737       _bio_inalign               0047b737 f   bio.obj
 0001:0007a757       _opj_cio_open              0047b757 f   cio.obj
 0001:0007a813       _opj_cio_close             0047b813 f   cio.obj
 0001:0007a82e       _cio_read                  0047b82e f   cio.obj
 0001:0007a9e1       _dwt_getgain               0047b9e1 f   dwt.obj
 0001:0007afe9       _dwt_decode_real           0047bfe9 f   dwt.obj
 0001:0007b27e       _opj_event_msg             0047c27e f   event.obj
 0001:0007b301       _opj_image_destroy         0047c301 f   image.obj
 0001:0007c36c       _j2k_create_decompress     0047d36c f   j2k.obj
 0001:0007c3ae       _j2k_destroy_decompress    0047d3ae f   j2k.obj
 0001:0007c4a9       _j2k_setup_decoder         0047d4a9 f   j2k.obj
 0001:0007c4d4       _j2k_decode                0047d4d4 f   j2k.obj
 0001:0007c5dc       _j2k_decode_jpt_stream     0047d5dc f   j2k.obj
 0001:0007c76f       _opj_clock                 0047d76f f   j2k_lib.obj
 0001:0007c9f2       _jp2_read_jp2h             0047d9f2 f   jp2.obj
 0001:0007cc31       _jp2_destroy_decompress    0047dc31 f   jp2.obj
 0001:0007cc63       _jp2_decode                0047dc63 f   jp2.obj
 0001:0007cced       _jpt_read_VBAS_info        0047dced f   jpt.obj
 0001:0007cd11       _jpt_read_msg_header       0047dd11 f   jpt.obj
 0001:0007ce77       _mqc_decode                0047de77 f   mqc.obj
 0001:0007cee1       _opj_create_decompress     0047dee1 f   openjpeg.obj
 0001:0007db62       _pi_create_decode          0047eb62 f   pi.obj
 0001:0007dfa9       _pi_destroy                0047efa9 f   pi.obj
 0001:0007e033       _pi_next                   0047f033 f   pi.obj
 0001:0007e07b       _raw_decode                0047f07b f   raw.obj
 0001:0007e920       _t1_create                 0047f920 f   t1.obj
 0001:0007e961       _t1_destroy                0047f961 f   t1.obj
 0001:0007e99b       _t1_decode_cblks           0047f99b f   t1.obj
 0001:0007f2b1       _t2_decode_packets         004802b1 f   t2.obj
 0001:0007f50a       _t2_create                 0048050a f   t2.obj
 0001:0007f52c       _tcd_create                0048052c f   tcd.obj
 0001:0007f562       _tcd_malloc_decode         00480562 f   tcd.obj
 0001:0007f7bd       _tcd_malloc_decode_tile    004807bd f   tcd.obj
 0001:0007fd9c       _tcd_decode_tile           00480d9c f   tcd.obj
 0001:00080453       _tcd_free_decode_tile      00481453 f   tcd.obj
 0001:0008055a       _tgt_create                0048155a f   tgt.obj
 0001:00080698       _tgt_destroy               00481698 f   tgt.obj
 0001:000806a9       _tgt_reset                 004816a9 f   tgt.obj
 0001:000806dd       _tgt_decode                004816dd f   tgt.obj
 0001:00080765       _timeinms                  00481765 f   pdfbench.obj
 0001:00080796       _openxref                  00481796 f   pdfbench.obj
 0001:00080861       _benchloadpage             00481861 f   pdfbench.obj
 0001:00080905       _benchrenderpage           00481905 f   pdfbench.obj
 0001:00080a99       _freepage                  00481a99 f   pdfbench.obj
 0001:00080ae2       _benchfile                 00481ae2 f   pdfbench.obj
 0001:00080c70       _usage                     00481c70 f   pdfbench.obj
 0001:00080c8d       _isarg                     00481c8d f   pdfbench.obj
 0001:00080ccf       _main                      00481ccf f   pdfbench.obj
 0001:00080d48       @__security_check_cookie@4 00481d48 f   LIBCMT:secchk.obj
 0001:00080d57       _free                      00481d57 f   LIBCMT:free.obj
 0001:00080de5       _V6_HeapAlloc              00481de5 f   LIBCMT:malloc.obj
 0001:00080e34       _malloc                    00481e34 f   LIBCMT:malloc.obj
 0001:00080ef7       _sprintf                   00481ef7 f   LIBCMT:sprintf.obj
 0001:00080f72       __get_sys_err_msg          00481f72 f i LIBCMT:strerror.obj
 0001:00080f95       _strerror                  00481f95 f   LIBCMT:strerror.obj
 0001:00080ffc       __flush                    00481ffc f   LIBCMT:fflush.obj
 0001:0008105e       __fflush_nolock            0048205e f   LIBCMT:fflush.obj
 0001:0008117a       _fflush                    0048217a f   LIBCMT:fflush.obj
 0001:000811cd       __flushall                 004821cd f   LIBCMT:fflush.obj
 0001:000811d6       __get_errno_from_oserr     004821d6 f   LIBCMT:dosmap.obj
 0001:00081211       __errno                    00482211 f   LIBCMT:dosmap.obj
 0001:00081224       ___doserrno                00482224 f   LIBCMT:dosmap.obj
 0001:00081237       __dosmaperr                00482237 f   LIBCMT:dosmap.obj
 0001:00081255       __fsopen                   00482255 f   LIBCMT:fopen.obj
 0001:00081319       _fopen                     00482319 f   LIBCMT:fopen.obj
 0001:0008132c       __fread_nolock_s           0048232c f   LIBCMT:fread.obj
 0001:00081532       _fread_s                   00482532 f   LIBCMT:fread.obj
 0001:000815c8       _fread                     004825c8 f   LIBCMT:fread.obj
 0001:000815e3       _fprintf                   004825e3 f   LIBCMT:fprintf.obj
 0001:00081732       __vsnprintf_l              00482732 f   LIBCMT:vsnprint.obj
 0001:000817e3       __vsnprintf                004827e3 f   LIBCMT:vsnprint.obj
 0001:000817fe       __ftell_nolock             004827fe f   LIBCMT:ftell.obj
 0001:00081996       _ftell                     00482996 f   LIBCMT:ftell.obj
 0001:00081a04       __fseek_nolock             00482a04 f   LIBCMT:fseek.obj
 0001:00081a8b       _fseek                     00482a8b f   LIBCMT:fseek.obj
 0001:00081b10       __fclose_nolock            00482b10 f   LIBCMT:fclose.obj
 0001:00081b82       _fclose                    00482b82 f   LIBCMT:fclose.obj
 0001:00081bfe       _realloc                   00482bfe f   LIBCMT:realloc.obj
 0001:00081e19       __recalloc                 00482e19 f   LIBCMT:realloc.obj
 0001:00081ea0       _memmove                   00482ea0 f   LIBCMT:memmove.obj
 0001:000822d0       _qsort                     004832d0 f   LIBCMT:qsort.obj
 0001:00082578       _longjmp                   00483578 f   LIBCMT:longjmp.obj
 0001:00082629       _strncmp                   00483629 f   LIBCMT:strncmp.obj
 0001:000826e7       _atol                      004836e7 f   LIBCMT:atox.obj
 0001:000826f8       _atoi                      004836f8 f   LIBCMT:atox.obj
 0001:00082700       _memchr                    00483700 f   LIBCMT:memchr.obj
 0001:000827b0       _strstr                    004837b0 f   LIBCMT:strstr.obj
 0001:00082836       ___iob_func                00483836 f   LIBCMT:_file.obj
 0001:0008283c       ___initstdio               0048383c f   LIBCMT:_file.obj
 0001:000828ed       ___endstdio                004838ed f   LIBCMT:_file.obj
 0001:0008290d       __lock_file                0048390d f   LIBCMT:_file.obj
 0001:00082949       __lock_file2               00483949 f   LIBCMT:_file.obj
 0001:00082977       __unlock_file              00483977 f   LIBCMT:_file.obj
 0001:000829ad       __unlock_file2             004839ad f   LIBCMT:_file.obj
 0001:000829d7       __amsg_exit                004839d7 f   LIBCMT:crt0dat.obj
 0001:000829fb       ___crtCorExitProcess       004839fb f   LIBCMT:crt0dat.obj
 0001:00082a21       ___crtExitProcess          00483a21 f   LIBCMT:crt0dat.obj
 0001:00082a36       __lockexit                 00483a36 f   LIBCMT:crt0dat.obj
 0001:00082a3f       __unlockexit               00483a3f f   LIBCMT:crt0dat.obj
 0001:00082a60       __initterm_e               00483a60 f   LIBCMT:crt0dat.obj
 0001:00082a80       __get_osplatform           00483a80 f   LIBCMT:crt0dat.obj
 0001:00082ab7       __get_winmajor             00483ab7 f   LIBCMT:crt0dat.obj
 0001:00082af3       __cinit                    00483af3 f   LIBCMT:crt0dat.obj
 0001:00082c67       _exit                      00483c67 f   LIBCMT:crt0dat.obj
 0001:00082c78       __exit                     00483c78 f   LIBCMT:crt0dat.obj
 0001:00082c89       __cexit                    00483c89 f   LIBCMT:crt0dat.obj
 0001:00082c98       __c_exit                   00483c98 f   LIBCMT:crt0dat.obj
 0001:00082ca7       __init_pointers            00483ca7 f   LIBCMT:crt0dat.obj
 0001:00082d5b       _sscanf                    00483d5b f   LIBCMT:sscanf.obj
 0001:00082d7a       __getenv_helper_nolock     00483d7a f   LIBCMT:getenv.obj
 0001:00082dfb       _getenv                    00483dfb f   LIBCMT:getenv.obj
 0001:00082e80       _strncpy                   00483e80 f   LIBCMT:strncpy.obj
 0001:00082fa4       _printf                    00483fa4 f   LIBCMT:printf.obj
 0001:00083053       __get_printf_count_output  00484053 f   LIBCMT:printf.obj
 0001:00083069       __isnan                    00484069 f   LIBCMT:ieeemisc.obj
 0001:00083097       __fpclass                  00484097 f   LIBCMT:ieeemisc.obj
 0001:00083130       _ceil                      00484130 f   LIBCMT:ceil_pentium4.obj
 0001:00083170       __ceil_pentium4            00484170 f   LIBCMT:ceil_pentium4.obj
 0001:0008324d       _vfprintf_helper           0048424d f   LIBCMT:vfprintf.obj
 0001:0008339b       _vfprintf                  0048439b f   LIBCMT:vfprintf.obj
 0001:000833c0       _strpbrk                   004843c0 f   LIBCMT:strpbrk.obj
 0001:00083410       _strchr                    00484410 f   LIBCMT:strchr.obj
 0001:00083416       ___from_strstr_to_strchr   00484416     LIBCMT:strchr.obj
 0001:000834d0       _strrchr                   004844d0 f   LIBCMT:strrchr.obj
 0001:000834fd       ??0_LocaleUpdate@@QAE@PAUlocaleinfo_struct@@@Z 004844fd f i LIBCMT:atof.obj
 0001:0008357f       __atof_l                   0048457f f   LIBCMT:atof.obj
 0001:00083628       _atof                      00484628 f   LIBCMT:atof.obj
 0001:00083636       _vprintf_helper            00484636 f   LIBCMT:vprintf.obj
 0001:000836c6       _vprintf                   004846c6 f   LIBCMT:vprintf.obj
 0001:00083909       _strtol                    00484909 f   LIBCMT:strtol.obj
 0001:00083932       __tolower_l                00484932 f   LIBCMT:tolower.obj
 0001:00083a49       _tolower                   00484a49 f   LIBCMT:tolower.obj
 0001:00083a70       __aligned_offset_malloc    00484a70 f   LIBCMT:align.obj
 0001:00083b09       __aligned_free             00484b09 f   LIBCMT:align.obj
 0001:00083b1e       __aligned_malloc           00484b1e f   LIBCMT:align.obj
 0001:00083b31       __vsprintf_l               00484b31 f   LIBCMT:vsprintf.obj
 0001:00083bad       _vsprintf                  00484bad f   LIBCMT:vsprintf.obj
 0001:00083bc4       __calloc_impl              00484bc4 f   LIBCMT:calloc.obj
 0001:00083ce2       _calloc                    00484ce2 f   LIBCMT:calloc.obj
 0001:00083f3c       _mainCRTStartup            00484f3c f   LIBCMT:crt0.obj
 0001:00083f46       ___report_gsfailure        00484f46 f   LIBCMT:gs_report.obj
 0001:0008404a       ___heap_select             0048504a f   LIBCMT:heapinit.obj
 0001:000840a5       __heap_init                004850a5 f   LIBCMT:heapinit.obj
 0001:000840ff       __mtinitlocks              004850ff f   LIBCMT:mlock.obj
 0001:00084148       __mtdeletelocks            00485148 f   LIBCMT:mlock.obj
 0001:0008419d       __unlock                   0048519d f   LIBCMT:mlock.obj
 0001:000841b2       __mtinitlocknum            004851b2 f   LIBCMT:mlock.obj
 0001:00084275       __lock                     00485275 f   LIBCMT:mlock.obj
 0001:000842a6       ___sbh_heap_init           004852a6 f   LIBCMT:sbheap.obj
 0001:000842ee       ___sbh_find_block          004852ee f   LIBCMT:sbheap.obj
 0001:00084319       ___sbh_free_block          00485319 f   LIBCMT:sbheap.obj
 0001:0008462d       ___sbh_alloc_new_region    0048562d f   LIBCMT:sbheap.obj
 0001:000846dd       ___sbh_alloc_new_group     004856dd f   LIBCMT:sbheap.obj
 0001:000847e3       ___sbh_resize_block        004857e3 f   LIBCMT:sbheap.obj
 0001:00084ac2       ___sbh_alloc_block         00485ac2 f   LIBCMT:sbheap.obj
 0001:00084da8       __SEH_prolog4              00485da8 f   LIBCMT:sehprolg4.obj
 0001:00084ded       __SEH_epilog4              00485ded f   LIBCMT:sehprolg4.obj
 0001:00084e10       __except_handler4          00485e10 f   LIBCMT:chandler4.obj
 0001:00084fa6       __NMSG_WRITE               00485fa6 f   LIBCMT:crt0msg.obj
 0001:00085146       __FF_MSGBANNER             00486146 f   LIBCMT:crt0msg.obj
 0001:0008517f       __initp_heap_handler       0048617f f   LIBCMT:handler.obj
 0001:00085189       __callnewh                 00486189 f   LIBCMT:handler.obj
 0001:000851ab       __flsbuf                   004861ab f   LIBCMT:_flsbuf.obj
 0001:0008530b       __ioinit                   0048630b f   LIBCMT:ioinit.obj
 0001:0008554b       __fileno                   0048654b f   LIBCMT:fileno.obj
 0001:00085578       __initp_misc_invarg        00486578 f   LIBCMT:invarg.obj
 0001:00085582       __invoke_watson            00486582 f   LIBCMT:invarg.obj
 0001:0008567e       __invalid_parameter        0048667e f   LIBCMT:invarg.obj
 0001:00085743       __output_l                 00486743 f   LIBCMT:output.obj
 0001:000860d7       ___sys_nerr                004870d7 f   LIBCMT:syserr.obj
 0001:000860dd       ___sys_errlist             004870dd f   LIBCMT:syserr.obj
 0001:000860e3       _strcpy_s                  004870e3 f   LIBCMT:strcpy_s.obj
 0001:00086148       __malloc_crt               00487148 f   LIBCMT:crtheap.obj
 0001:00086188       __calloc_crt               00487188 f   LIBCMT:crtheap.obj
 0001:000861d0       __realloc_crt              004871d0 f   LIBCMT:crtheap.obj
 0001:0008621b       __recalloc_crt             0048721b f   LIBCMT:crtheap.obj
 0001:000862d7       __encode_pointer           004872d7 f   LIBCMT:tidtable.obj
 0001:00086345       __encoded_null             00487345 f   LIBCMT:tidtable.obj
 0001:0008634e       __decode_pointer           0048734e f   LIBCMT:tidtable.obj
 0001:000863bc       ___crtTlsAlloc@4           004873bc f   LIBCMT:tidtable.obj
 0001:000863c5       ___set_flsgetvalue         004873c5 f   LIBCMT:tidtable.obj
 0001:000863f7       __mtterm                   004873f7 f   LIBCMT:tidtable.obj
 0001:00086434       __initptd                  00487434 f   LIBCMT:tidtable.obj
 0001:000864f3       __getptd_noexit            004874f3 f   LIBCMT:tidtable.obj
 0001:0008656a       __getptd                   0048756a f   LIBCMT:tidtable.obj
 0001:00086582       __freefls@4                00487582 f   LIBCMT:tidtable.obj
 0001:000866a3       __mtinit                   004876a3 f   LIBCMT:tidtable.obj
 0001:00086827       _strncpy_s                 00487827 f   LIBCMT:strncpy_s.obj
 0001:000868da       __write_nolock             004878da f   LIBCMT:write.obj
 0001:00086ea0       __write                    00487ea0 f   LIBCMT:write.obj
 0001:00086f7c       __commit                   00487f7c f   LIBCMT:commit.obj
 0001:0008705d       __openfile                 0048805d f   LIBCMT:_open.obj
 0001:000872fd       __getstream                004882fd f   LIBCMT:stream.obj
 0001:00087430       __local_unwind4            00488430 f   LIBCMT:exsup4.obj
 0001:00087506       __seh_longjmp_unwind4@4    00488506 f   LIBCMT:exsup4.obj
 0001:00087522       @_EH4_CallFilterFunc@8     00488522 f   LIBCMT:exsup4.obj
 0001:00087539       @_EH4_TransferToHandler@8  00488539 f   LIBCMT:exsup4.obj
 0001:00087552       @_EH4_GlobalUnwind@4       00488552 f   LIBCMT:exsup4.obj
 0001:0008756c       @_EH4_LocalUnwind@16       0048856c f   LIBCMT:exsup4.obj
 0001:00087583       __filbuf                   00488583 f   LIBCMT:_filbuf.obj
 0001:000876a3       __read_nolock              004886a3 f   LIBCMT:read.obj
 0001:00087c64       __read                     00488c64 f   LIBCMT:read.obj
 0001:00087c64       _read                      00488c64 f   LIBCMT:read.obj
 0001:00087d61       _memcpy_s                  00488d61 f   LIBCMT:memcpy_s.obj
 0001:00087de0       _memset                    00488de0 f   LIBCMT:memset.obj
 0001:00087e5a       __stbuf                    00488e5a f   LIBCMT:_sftbuf.obj
 0001:00087ef0       __ftbuf                    00488ef0 f   LIBCMT:_sftbuf.obj
 0001:00087f20       _memcpy                    00488f20 f   LIBCMT:memcpy.obj
 0001:00088285       __lseek_nolock             00489285 f   LIBCMT:lseek.obj
 0001:000882f7       __lseek                    004892f7 f   LIBCMT:lseek.obj
 0001:000882f7       _lseek                     004892f7 f   LIBCMT:lseek.obj
 0001:000883d3       __close_nolock             004893d3 f   LIBCMT:close.obj
 0001:00088467       _close                     00489467 f   LIBCMT:close.obj
 0001:00088467       __close                    00489467 f   LIBCMT:close.obj
 0001:00088534       __freebuf                  00489534 f   LIBCMT:_freebuf.obj
 0001:00088560       __msize                    00489560 f   LIBCMT:msize.obj
 0001:0008868a       __VEC_memcpy               0048968a f   LIBCMT:p4_memcpy.obj
 0001:0008876d       __sse2_mathfcns_init       0048976d f   LIBCMT:mathfcns.obj
 0001:00088784       __global_unwind2           00489784 f   LIBCMT:exsup.obj
 0001:000887e9       __local_unwind2            004897e9 f   LIBCMT:exsup.obj
 0001:0008886d       __abnormal_termination     0048986d f   LIBCMT:exsup.obj
 0001:00088890       __NLG_Notify1              00489890 f   LIBCMT:exsup.obj
 0001:00088899       __NLG_Notify               00489899 f   LIBCMT:exsup.obj
 0001:000888b0       __NLG_Dispatch             004898b0     LIBCMT:exsup.obj
 0001:000888b0       __NLG_Dispatch2            004898b0     LIBCMT:exsup.obj
 0001:000888b8       __NLG_Call                 004898b8 f   LIBCMT:exsup.obj
 0001:000888ba       __NLG_Return2              004898ba     LIBCMT:exsup.obj
 0001:000888bb       __rt_probe_read4@4         004898bb f   LIBCMT:sehsupp.obj
 0001:00088906       __fcloseall                00489906 f   LIBCMT:closeall.obj
 0001:00088a5e       ___onexitinit              00489a5e f   LIBCMT:onexit.obj
 0001:00088a8d       __onexit                   00489a8d f   LIBCMT:onexit.obj
 0001:00088ac9       _atexit                    00489ac9 f   LIBCMT:onexit.obj
 0001:00088adb       __RTC_Initialize           00489adb f   LIBCMT:initsect.obj
 0001:00088aff       __RTC_Terminate            00489aff f   LIBCMT:initsect.obj
 0001:00088b23       __initp_misc_cfltcvt_tab   00489b23 f   LIBCMT:cmiscdat.obj
 0001:00088b50       __ValidateImageBase        00489b50 f   LIBCMT:pesect.obj
 0001:00088b80       __FindPESection            00489b80 f   LIBCMT:pesect.obj
 0001:00088bd0       __IsNonwritableInCurrentImage 00489bd0 f   LIBCMT:pesect.obj
 0001:00088c8b       ?terminate@@YAXXZ          00489c8b f   LIBCMT:hooks.obj
 0001:00088cc4       __initp_eh_hooks           00489cc4 f   LIBCMT:hooks.obj
 0001:00088cd5       __initp_misc_winxfltr      00489cd5 f   LIBCMT:winxfltr.obj
 0001:00088cd5       __fpclear                  00489cd5 f   LIBCMT:fpinit.obj
 0001:00088cd6       __XcptFilter               00489cd6 f   LIBCMT:winxfltr.obj
 0001:00088e34       __initp_misc_winsig        00489e34 f   LIBCMT:winsig.obj
 0001:00088e81       ___get_sigabrt             00489e81 f   LIBCMT:winsig.obj
 0001:00088e8e       _raise                     00489e8e f   LIBCMT:winsig.obj
 0001:0008903e       __initp_misc_rand_s        0048a03e f   LIBCMT:rand_s.obj
 0001:00089048       __initp_misc_purevirt      0048a048 f   LIBCMT:inithelp.obj
 0001:00089052       __initp_misc_initcrit      0048a052 f   LIBCMT:initcrit.obj
 0001:0008906c       ___crtInitCritSecAndSpinCount 0048a06c f   LIBCMT:initcrit.obj
 0001:00089140       _strlen                    0048a140 f   LIBCMT:strlen.obj
 0001:0008925a       __input_l                  0048a25a f   LIBCMT:input.obj
 0001:00089ea7       __mbsnbicoll_l             0048aea7 f   LIBCMT:mbsnbico.obj
 0001:00089f93       __mbsnbicoll               0048af93 f   LIBCMT:mbsnbico.obj
 0001:00089faa       ___wtomb_environ           0048afaa f   LIBCMT:wtombenv.obj
 0001:0008a03f       _strnlen                   0048b03f f   LIBCMT:strlen_s.obj
 0001:0008a059       __cfltcvt_init             0048b059 f   LIBCMT:fpinit.obj
 0001:0008a0b9       __fpmath                   0048b0b9 f   LIBCMT:fpinit.obj
 0001:0008a0d7       __set_exp                  0048b0d7 f   LIBCMT:util.obj
 0001:0008a101       __get_exp                  0048b101 f   LIBCMT:util.obj
 0001:0008a116       __sptype                   0048b116 f   LIBCMT:util.obj
 0001:0008a171       __decomp                   0048b171 f   LIBCMT:util.obj
 0001:0008a220       __raise_exc_ex             0048b220 f   LIBCMT:fpexcept.obj
 0001:0008a4fa       __raise_exc                0048b4fa f   LIBCMT:fpexcept.obj
 0001:0008a51b       __handle_exc               0048b51b f   LIBCMT:fpexcept.obj
 0001:0008a6fc       __set_errno_from_matherr   0048b6fc f   LIBCMT:fpexcept.obj
 0001:0008a724       __errcode                  0048b724 f   LIBCMT:fpexcept.obj
 0001:0008a751       __umatherr                 0048b751 f   LIBCMT:fpexcept.obj
 0001:0008a7ef       __handle_qnan1             0048b7ef f   LIBCMT:fpexcept.obj
 0001:0008a842       __handle_qnan2             0048b842 f   LIBCMT:fpexcept.obj
 0001:0008a8a1       __except1                  0048b8a1 f   LIBCMT:fpexcept.obj
 0001:0008a95b       __except2                  0048b95b f   LIBCMT:fpexcept.obj
 0001:0008aa27       __statfp                   0048ba27 f   LIBCMT:fpctrl.obj
 0001:0008aa32       __clrfp                    0048ba32 f   LIBCMT:fpctrl.obj
 0001:0008aa3e       __ctrlfp                   0048ba3e f   LIBCMT:fpctrl.obj
 0001:0008aa65       __set_statfp               0048ba65 f   LIBCMT:fpctrl.obj
 0001:0008aabb       ___set_fpsr_sse2           0048babb f   LIBCMT:fpctrl.obj
 0001:0008ab2d       ___libm_error_support      0048bb2d f   LIBCMT:libm_error.obj
 0001:0008addd       __ceil_default             0048bddd f   LIBCMT:ceil.obj
 0001:0008aeb0       _strcmp                    0048beb0 f   LIBCMT:strcmp.obj
 0001:0008b146       ___updatetmbcinfo          0048c146 f   LIBCMT:mbctype.obj
 0001:0008b264       __setmbcp_nolock           0048c264 f   LIBCMT:mbctype.obj
 0001:0008b43d       __setmbcp                  0048c43d f   LIBCMT:mbctype.obj
 0001:0008b5d7       ___initmbctable            0048c5d7 f   LIBCMT:mbctype.obj
 0001:0008b5f5       ___freetlocinfo            0048c5f5 f   LIBCMT:setlocal.obj
 0001:0008b735       ___addlocaleref            0048c735 f   LIBCMT:setlocal.obj
 0001:0008b7bb       ___removelocaleref         0048c7bb f   LIBCMT:setlocal.obj
 0001:0008b885       ___updatetlocinfo          0048c885 f   LIBCMT:setlocal.obj
 0001:0008b8fb       __fltin2                   0048c8fb f   LIBCMT:cfin.obj
 0001:0008b9a0       __isctype_l                0048c9a0 f   LIBCMT:isctype.obj
 0001:0008ba56       ___strgtold12_l            0048ca56 f   LIBCMT:strgtold.obj
 0001:0008c116       __lseeki64_nolock          0048d116 f   LIBCMT:lseeki64.obj
 0001:0008c199       __lseeki64                 0048d199 f   LIBCMT:lseeki64.obj
 0001:0008c2b2       __set_osfhnd               0048d2b2 f   LIBCMT:osfinfo.obj
 0001:0008c32f       __free_osfhnd              0048d32f f   LIBCMT:osfinfo.obj
 0001:0008c3b0       __get_osfhandle            0048d3b0 f   LIBCMT:osfinfo.obj
 0001:0008c421       ___lock_fhandle            0048d421 f   LIBCMT:osfinfo.obj
 0001:0008c4c1       __unlock_fhandle           0048d4c1 f   LIBCMT:osfinfo.obj
 0001:0008c4e3       __alloc_osfhnd             0048d4e3 f   LIBCMT:osfinfo.obj
 0001:0008c682       __chsize_nolock            0048d682 f   LIBCMT:chsize.obj
 0001:0008c836       __setmode_nolock           0048d836 f   LIBCMT:setmode.obj
 0001:0008c8f2       __get_fmode                0048d8f2 f   LIBCMT:setmode.obj
 0001:0008c926       __freea                    0048d926 f i LIBCMT:a_map.obj
 0001:0008cce3       ___crtLCMapStringA         0048dce3 f   LIBCMT:a_map.obj
 0001:0008cd26       __isleadbyte_l             0048dd26 f i LIBCMT:_wctype.obj
 0001:0008cd5c       _isleadbyte                0048dd5c f i LIBCMT:_wctype.obj
 0001:0008cd6a       ?__CxxUnhandledExceptionFilter@@YGJPAU_EXCEPTION_POINTERS@@@Z 0048dd6a f   LIBCMT:unhandld.obj
 0001:0008cda7       ___CxxSetUnhandledExceptionFilter 0048dda7 f   LIBCMT:unhandld.obj
 0001:0008cdb5       __setenvp                  0048ddb5 f   LIBCMT:stdenvp.obj
 0001:0008d028       __setargv                  0048e028 f   LIBCMT:stdargv.obj
 0001:0008d0e1       ___crtGetEnvironmentStringsA 0048e0e1 f   LIBCMT:a_env.obj
 0001:0008d216       ___security_init_cookie    0048e216 f   LIBCMT:gs_support.obj
 0001:0008d2aa       __crt_debugger_hook        0048e2aa f   LIBCMT:dbghook.obj
 0001:0008d2b2       ___crtMessageBoxA          0048e2b2 f   LIBCMT:crtmbox.obj
 0001:0008d46f       _strcat_s                  0048e46f f   LIBCMT:strcat_s.obj
 0001:0008d4e0       __set_error_mode           0048e4e0 f   LIBCMT:errmode.obj
 0001:0008d526       __getbuf                   0048e526 f   LIBCMT:_getbuf.obj
 0001:0008d56a       __isatty                   0048e56a f   LIBCMT:isatty.obj
 0001:0008d5c8       __wctomb_s_l               0048e5c8 f   LIBCMT:wctomb.obj
 0001:0008d727       _wctomb_s                  0048e727 f   LIBCMT:wctomb.obj
 0001:0008d750       __aulldvrm                 0048e750 f   LIBCMT:ulldvrm.obj
 0001:0008d7e5       __putwch_nolock            0048e7e5 f   LIBCMT:putwch.obj
 0001:0008d8a7       __mbtowc_l                 0048e8a7 f   LIBCMT:mbtowc.obj
 0001:0008d9ba       _mbtowc                    0048e9ba f   LIBCMT:mbtowc.obj
 0001:0008e12a       _open                      0048f12a f   LIBCMT:open.obj
 0001:0008e12a       __open                     0048f12a f   LIBCMT:open.obj
 0001:0008e1e0       __sopen_helper             0048f1e0 f   LIBCMT:open.obj
 0001:0008e2ac       __sopen_s                  0048f2ac f   LIBCMT:open.obj
 0001:0008e2ca       __mbsicmp_l                0048f2ca f   LIBCMT:mbsicmp.obj
 0001:0008e4e4       __mbsicmp                  0048f4e4 f   LIBCMT:mbsicmp.obj
 0001:0008e4f7       __mbsnbcmp_l               0048f4f7 f   LIBCMT:mbsnbcmp.obj
 0001:0008e660       __mbsnbcmp                 0048f660 f   LIBCMT:mbsnbcmp.obj
 0001:0008e6ce       __VEC_memzero              0048f6ce f   LIBCMT:p4_memset.obj
 0001:0008e7ad       __get_sse2_info            0048f7ad f   LIBCMT:cpu_disp.obj
 0001:0008e80d       ___sse2_available_init     0048f80d f   LIBCMT:cpu_disp.obj
 0001:0008e820       __allmul                   0048f820 f   LIBCMT:llmul.obj
 0001:0008e854       __fptrap                   0048f854 f   LIBCMT:crt0fp.obj
 0001:0008e85d       _abort                     0048f85d f   LIBCMT:abort.obj
 0001:0008e950       __isdigit_l                0048f950 f i LIBCMT:_ctype.obj
 0001:0008e99f       _isdigit                   0048f99f f i LIBCMT:_ctype.obj
 0001:0008e9c8       __isxdigit_l               0048f9c8 f i LIBCMT:_ctype.obj
 0001:0008ea1c       _isxdigit                  0048fa1c f i LIBCMT:_ctype.obj
 0001:0008ea47       __isspace_l                0048fa47 f i LIBCMT:_ctype.obj
 0001:0008ea96       _isspace                   0048fa96 f i LIBCMT:_ctype.obj
 0001:0008eabf       __ungetc_nolock            0048fabf f   LIBCMT:ungetc.obj
 0001:0008ef66       ___crtCompareStringA       0048ff66 f   LIBCMT:a_cmp.obj
 0001:0008efa6       __strnicoll_l              0048ffa6 f   LIBCMT:strnicol.obj
 0001:0008f148       ___crtsetenv               00490148 f   LIBCMT:setenv.obj
 0001:0008f394       __forcdecpt_l              00490394 f   LIBCMT:cvt.obj
 0001:0008f405       __cropzeros_l              00490405 f   LIBCMT:cvt.obj
 0001:0008f485       __positive                 00490485 f   LIBCMT:cvt.obj
 0001:0008f49b       __fassign_l                0049049b f   LIBCMT:cvt.obj
 0001:0008f4db       __fassign                  004904db f   LIBCMT:cvt.obj
 0001:0008f50f       __forcdecpt                0049050f f   LIBCMT:cvt.obj
 0001:0008f51d       __cropzeros                0049051d f   LIBCMT:cvt.obj
 0001:0008f698       __cftoe_l                  00490698 f   LIBCMT:cvt.obj
 0001:0008f766       __cftoe                    00490766 f   LIBCMT:cvt.obj
 0001:0008f784       __cftoa_l                  00490784 f   LIBCMT:cvt.obj
 0001:0008fbea       __cftof_l                  00490bea f   LIBCMT:cvt.obj
 0001:0008fca3       __cftog_l                  00490ca3 f   LIBCMT:cvt.obj
 0001:0008fd9b       __cfltcvt_l                00490d9b f   LIBCMT:cvt.obj
 0001:0008fe21       __cfltcvt                  00490e21 f   LIBCMT:cvt.obj
 0001:0008fe42       __setdefaultprecision      00490e42 f   LIBCMT:fp8.obj
 0001:0008fe6b       __ms_p5_test_fdiv          00490e6b f   LIBCMT:testfdiv.obj
 0001:0008fea7       __ms_p5_mp_test_fdiv       00490ea7 f   LIBCMT:testfdiv.obj
 0001:0008fed0       __matherr                  00490ed0 f   LIBCMT:matherr.obj
 0001:0008fed3       __frnd                     00490ed3 f   LIBCMT:frnd.obj
 0001:0009009c       ___crtGetStringTypeA       0049109c f   LIBCMT:a_str.obj
 0001:000900dc       ___free_lc_time            004910dc f   LIBCMT:inittime.obj
 0001:0009026c       ___free_lconv_num          0049126c f   LIBCMT:initnum.obj
 0001:000902ac       ___free_lconv_mon          004912ac f   LIBCMT:initmon.obj
 0001:00090340       _strcspn                   00491340 f   LIBCMT:strcspn.obj
 0001:00090386       __ld12tod                  00491386 f   LIBCMT:intrncvt.obj
 0001:000908c8       __ld12tof                  004918c8 f   LIBCMT:intrncvt.obj
 0001:00090e0a       ___mtold12                 00491e0a f   LIBCMT:mantold.obj
 0001:00090fd6       ___ansicp                  00491fd6 f   LIBCMT:convrtcp.obj
 0001:0009101d       ___convertcp               0049201d f   LIBCMT:convrtcp.obj
 0001:000911d0       __alloca_probe_16          004921d0 f   LIBCMT:alloca16.obj
 0001:000911e6       __alloca_probe_8           004921e6     LIBCMT:alloca16.obj
 0001:0009124d       __ismbblead                0049224d f   LIBCMT:ismbbyte.obj
 0001:00091260       ___initconout              00492260 f   LIBCMT:initcon.obj
 0001:0009127f       ___termcon                 0049227f f   LIBCMT:initcon.obj
 0001:000912ac       ___ascii_stricmp           004922ac f   LIBCMT:stricmp.obj
 0001:000912e1       __stricmp_l                004922e1 f   LIBCMT:stricmp.obj
 0001:000913b4       __stricmp                  004923b4 f   LIBCMT:stricmp.obj
 0001:000913b4       _stricmp                   004923b4 f   LIBCMT:stricmp.obj
 0001:00091404       __strnicmp_l               00492404 f   LIBCMT:strnicmp.obj
 0001:000914f4       __strdup                   004924f4 f   LIBCMT:strdup.obj
 0001:00091544       __mbschr_l                 00492544 f   LIBCMT:mbschr.obj
 0001:000915fe       __mbschr                   004925fe f   LIBCMT:mbschr.obj
 0001:00091611       __atodbl_l                 00492611 f   LIBCMT:atodbl.obj
 0001:000916b7       __atoflt_l                 004926b7 f   LIBCMT:atodbl.obj
 0001:0009175d       __fptostr                  0049275d f   LIBCMT:_fptostr.obj
 0001:0009181a       ___dtold                   0049281a f   LIBCMT:cfout.obj
 0001:000918d5       __fltout2                  004928d5 f   LIBCMT:cfout.obj
 0001:00091970       __alldvrm                  00492970 f   LIBCMT:lldvrm.obj
 0001:00091a50       __aullshr                  00492a50 f   LIBCMT:ullshr.obj
 0001:00091a6f       __controlfp_s              00492a6f f   LIBCMT:contrlfp.obj
 0001:00091ae0       __chkstk                   00492ae0 f   LIBCMT:chkstk.obj
 0001:00091ae0       __alloca_probe             00492ae0     LIBCMT:chkstk.obj
 0001:00091b10       ___ascii_strnicmp          00492b10 f   LIBCMT:_strnicm.obj
 0001:00091b71       _$I10_OUTPUT               00492b71 f   LIBCMT:x10fout.obj
 0001:00092565       __control87                00493565 f i LIBCMT:ieee87.obj
 0001:00092868       _RtlUnwind@16              00493868 f   kernel32:KERNEL32.dll
 0001:00092aba       __hypot                    00493aba f   LIBCMT:hypot.obj
 0001:00092aba       _hypot                     00493aba f   LIBCMT:hypot.obj
 0001:00092ae0       __CIsqrt                   00493ae0 f   LIBCMT:sqrt.obj
 0001:00092af4       _sqrt                      00493af4     LIBCMT:sqrt.obj
 0001:00092ba0       __trandisp1                00493ba0 f   LIBCMT:87disp.obj
 0001:00092c07       __trandisp2                00493c07 f   LIBCMT:87disp.obj
 0001:00092c93       __rttospopde               00493c93     LIBCMT:87disp.obj
 0001:00092c98       __rttospop                 00493c98     LIBCMT:87disp.obj
 0001:00092c9a       __rtnospop                 00493c9a     LIBCMT:87disp.obj
 0001:00092c9c       __rttosnpop                00493c9c     LIBCMT:87disp.obj
 0001:00092c9d       __rtnospopde               00493c9d     LIBCMT:87disp.obj
 0001:00092ca4       __rtzeropop                00493ca4     LIBCMT:87disp.obj
 0001:00092ca6       __rtzeronpop               00493ca6     LIBCMT:87disp.obj
 0001:00092cab       __rtonepop                 00493cab     LIBCMT:87disp.obj
 0001:00092cad       __rtonenpop                00493cad     LIBCMT:87disp.obj
 0001:00092cb2       __tosnan1                  00493cb2     LIBCMT:87disp.obj
 0001:00092cdd       __nosnan2                  00493cdd     LIBCMT:87disp.obj
 0001:00092cdf       __tosnan2                  00493cdf     LIBCMT:87disp.obj
 0001:00092d07       __nan2                     00493d07     LIBCMT:87disp.obj
 0001:00092d46       __rtindfpop                00493d46     LIBCMT:87disp.obj
 0001:00092d48       __rtindfnpop               00493d48     LIBCMT:87disp.obj
 0001:00092d59       __rttosnpopde              00493d59     LIBCMT:87disp.obj
 0001:00092d63       __rtchsifneg               00493d63     LIBCMT:87disp.obj
 0001:00092d70       __startTwoArgErrorHandling 00493d70 f   LIBCMT:genexcep.obj
 0001:00092d87       __startOneArgErrorHandling 00493d87 f   LIBCMT:genexcep.obj
 0001:00092dd0       __twoToTOS                 00493dd0 f   LIBCMT:common.obj
 0001:00092de5       __load_CW                  00493de5 f   LIBCMT:common.obj
 0001:00092dfc       __convertTOStoQNaN         00493dfc f   LIBCMT:common.obj
 0001:00092e15       __fload_withFB             00493e15 f   LIBCMT:common.obj
 0001:00092e58       __checkTOS_withFB          00493e58 f   LIBCMT:common.obj
 0001:00092e6e       __fast_exit                00493e6e f   LIBCMT:common.obj
 0001:00092e7b       __math_exit                00493e7b f   LIBCMT:common.obj
 0001:00092ea5       __check_overflow_exit      00493ea5 f   LIBCMT:common.obj
 0001:00092eb9       __check_range_exit         00493eb9 f   LIBCMT:common.obj
 0001:00092f5c       __87except                 00493f5c f   LIBCMT:87except.obj
 0001:00093060       __ftol2_sse                00494060 f   LIBCMT:ftol2.obj
 0001:00093069       __ftol2_pentium4           00494069 f   LIBCMT:ftol2.obj
 0001:0009307c       __ftol2_sse_excpt          0049407c f   LIBCMT:ftol2.obj
 0001:00093096       __ftol2                    00494096 f   LIBCMT:ftol2.obj
 0001:00093110       _pow                       00494110 f   LIBCMT:pow.obj
 0001:00093150       __CIpow                    00494150 f   LIBCMT:pow.obj
 0001:0009318b       __CIpow_default            0049418b f   LIBCMT:pow.obj
 0001:000931a4       __pow_default              004941a4     LIBCMT:pow.obj
 0001:000933a0       _floor                     004943a0 f   LIBCMT:floor_pentium4.obj
 0001:000933e0       __floor_pentium4           004943e0 f   LIBCMT:floor_pentium4.obj
 0001:000934d0       __alldiv                   004944d0 f   LIBCMT:lldiv.obj
 0001:00093580       __allshr                   00494580 f   LIBCMT:llshr.obj
 0001:000935b0       _sin                       004945b0 f   LIBCMT:sin.obj
 0001:000935f0       __CIsin                    004945f0 f   LIBCMT:sin.obj
 0001:0009362b       __CIsin_default            0049462b f   LIBCMT:sin.obj
 0001:0009363f       __sin_default              0049463f     LIBCMT:sin.obj
 0001:000936e0       _cos                       004946e0 f   LIBCMT:cos.obj
 0001:00093720       __CIcos                    00494720 f   LIBCMT:cos.obj
 0001:0009375b       __CIcos_default            0049475b f   LIBCMT:cos.obj
 0001:0009376f       __cos_default              0049476f     LIBCMT:cos.obj
 0001:00093810       _atan2                     00494810 f   LIBCMT:87ctriga.obj
 0001:0009381a       __CIatan2                  0049481a f   LIBCMT:87ctriga.obj
 0001:00093830       _asin                      00494830 f   LIBCMT:asin.obj
 0001:00093870       __CIasin                   00494870 f   LIBCMT:asin.obj
 0001:000938ab       __CIasin_default           004948ab f   LIBCMT:asin.obj
 0001:000938bf       __asin_default             004948bf     LIBCMT:asin.obj
 0001:00093978       __setjmp3                  00494978 f   LIBCMT:setjmp3.obj
 0001:00093a00       _log10                     00494a00 f   LIBCMT:log10.obj
 0001:00093a40       __CIlog10                  00494a40 f   LIBCMT:log10.obj
 0001:00093a7b       __CIlog10_default          00494a7b f   LIBCMT:log10.obj
 0001:00093a8f       __log10_default            00494a8f     LIBCMT:log10.obj
 0001:00093b50       _log                       00494b50 f   LIBCMT:log.obj
 0001:00093b90       __CIlog                    00494b90 f   LIBCMT:log.obj
 0001:00093bcb       __CIlog_default            00494bcb f   LIBCMT:log.obj
 0001:00093bdf       __log_default              00494bdf     LIBCMT:log.obj
 0001:00093ca0       __CIpow_pentium4           00494ca0 f   LIBCMT:pow_pentium4.obj
 0001:00093cb9       __pow_pentium4             00494cb9     LIBCMT:pow_pentium4.obj
 0001:00094811       __fFEXP                    00495811     LIBCMT:87tran.obj
 0001:00094878       __rtinfpopse               00495878     LIBCMT:87tran.obj
 0001:0009487a       __rtinfnpopse              0049587a     LIBCMT:87tran.obj
 0001:0009488a       __fFLN                     0049588a     LIBCMT:87tran.obj
 0001:0009493f       __rtinfpop                 0049593f     LIBCMT:87tran.obj
 0001:00094941       __rtinfnpop                00495941     LIBCMT:87tran.obj
 0001:0009495e       __ffexpm1                  0049595e     LIBCMT:87tran.obj
 0001:00094a07       __d_inttype                00495a07 f   LIBCMT:powhlp.obj
 0001:00094a6b       __powhlp                   00495a6b f   LIBCMT:powhlp.obj
 0001:00094ba9       __floor_default            00495ba9 f   LIBCMT:floor.obj
 0001:00094c80       __CIsin_pentium4           00495c80 f   LIBCMT:sin_pentium4.obj
 0001:00094c98       __sin_pentium4             00495c98     LIBCMT:sin_pentium4.obj
 0001:00094e50       __CIcos_pentium4           00495e50 f   LIBCMT:cos_pentium4.obj
 0001:00094e68       __cos_pentium4             00495e68     LIBCMT:cos_pentium4.obj
 0001:0009501c       __fFATN2                   0049601c     LIBCMT:87triga.obj
 0001:0009506c       __rtpiby2                  0049606c     LIBCMT:87triga.obj
 0001:000950b0       __cintrindisp2             004960b0 f   LIBCMT:87cdisp.obj
 0001:000950ee       __cintrindisp1             004960ee f   LIBCMT:87cdisp.obj
 0001:0009512b       __ctrandisp2               0049612b f   LIBCMT:87cdisp.obj
 0001:000952c1       __ctrandisp1               004962c1 f   LIBCMT:87cdisp.obj
 0001:000952f4       __fload                    004962f4 f   LIBCMT:87cdisp.obj
 0001:00095330       __CIasin_pentium4          00496330 f   LIBCMT:asin_pentium4.obj
 0001:00095348       __asin_pentium4            00496348     LIBCMT:asin_pentium4.obj
 0001:000958b0       __CIlog10_pentium4         004968b0 f   LIBCMT:log10_pentium4.obj
 0001:000958c8       __log10_pentium4           004968c8     LIBCMT:log10_pentium4.obj
 0001:00095b40       __CIlog_pentium4           00496b40 f   LIBCMT:log_pentium4.obj
 0001:00095b58       __log_pentium4             00496b58     LIBCMT:log_pentium4.obj
 0001:00095db0       _fdiv_main_routine         00496db0 f   LIBCMT:adj_fdiv.obj
 0001:00095ec7       __adj_fdiv_r               00496ec7 f   LIBCMT:adj_fdiv.obj
 0001:00096366       __fdivp_sti_st             00497366 f   LIBCMT:adj_fdiv.obj
 0001:00096379       __fdivrp_sti_st            00497379 f   LIBCMT:adj_fdiv.obj
 0001:0009638c       __adj_fdiv_m32             0049738c f   LIBCMT:adj_fdiv.obj
 0001:000963d8       __adj_fdiv_m64             004973d8 f   LIBCMT:adj_fdiv.obj
 0001:00096424       __adj_fdiv_m16i            00497424 f   LIBCMT:adj_fdiv.obj
 0001:00096458       __adj_fdiv_m32i            00497458 f   LIBCMT:adj_fdiv.obj
 0001:0009648c       __adj_fdivr_m32            0049748c f   LIBCMT:adj_fdiv.obj
 0001:000964d8       __adj_fdivr_m64            004974d8 f   LIBCMT:adj_fdiv.obj
 0001:00096524       __adj_fdivr_m16i           00497524 f   LIBCMT:adj_fdiv.obj
 0001:00096558       __adj_fdivr_m32i           00497558 f   LIBCMT:adj_fdiv.obj
 0001:0009658c       __safe_fdiv                0049758c f   LIBCMT:adj_fdiv.obj
 0001:000965a1       __safe_fdivr               004975a1 f   LIBCMT:adj_fdiv.obj
 0001:000965b6       __fprem_common             004975b6 f   LIBCMT:adj_fdiv.obj
 0001:000967bc       __adj_fprem                004977bc f   LIBCMT:adj_fdiv.obj
 0001:0009686e       __fprem1_common            0049786e f   LIBCMT:adj_fdiv.obj
 0001:00096a74       __adj_fprem1               00497a74 f   LIBCMT:adj_fdiv.obj
 0001:00096b29       __safe_fprem               00497b29 f   LIBCMT:adj_fdiv.obj
 0001:00096b2f       __safe_fprem1              00497b2f f   LIBCMT:adj_fdiv.obj
 0001:00096b35       __adj_fpatan               00497b35 f   LIBCMT:adj_fdiv.obj
 0001:00096b38       __adj_fptan                00497b38 f   LIBCMT:adj_fdiv.obj
 0002:00000000       __imp__GetSystemTimeAsFileTime@4 00498000     kernel32:KERNEL32.dll
 0002:00000004       __imp__GetWindowsDirectoryA@8 00498004     kernel32:KERNEL32.dll
 0002:00000008       __imp__WideCharToMultiByte@32 00498008     kernel32:KERNEL32.dll
 0002:0000000c       __imp__FindFirstFileA@8    0049800c     kernel32:KERNEL32.dll
 0002:00000010       __imp__GetLastError@0      00498010     kernel32:KERNEL32.dll
 0002:00000014       __imp__FindClose@4         00498014     kernel32:KERNEL32.dll
 0002:00000018       __imp__FindNextFileA@8     00498018     kernel32:KERNEL32.dll
 0002:0000001c       __imp__QueryPerformanceCounter@4 0049801c     kernel32:KERNEL32.dll
 0002:00000020       __imp__QueryPerformanceFrequency@4 00498020     kernel32:KERNEL32.dll
 0002:00000024       __imp__HeapFree@12         00498024     kernel32:KERNEL32.dll
 0002:00000028       __imp__HeapAlloc@12        00498028     kernel32:KERNEL32.dll
 0002:0000002c       __imp__HeapReAlloc@16      0049802c     kernel32:KERNEL32.dll
 0002:00000030       __imp__RtlUnwind@16        00498030     kernel32:KERNEL32.dll
 0002:00000034       __imp__EnterCriticalSection@4 00498034     kernel32:KERNEL32.dll
 0002:00000038       __imp__LeaveCriticalSection@4 00498038     kernel32:KERNEL32.dll
 0002:0000003c       __imp__GetProcAddress@8    0049803c     kernel32:KERNEL32.dll
 0002:00000040       __imp__GetModuleHandleA@4  00498040     kernel32:KERNEL32.dll
 0002:00000044       __imp__ExitProcess@4       00498044     kernel32:KERNEL32.dll
 0002:00000048       __imp__CloseHandle@4       00498048     kernel32:KERNEL32.dll
 0002:0000004c       __imp__GetFileType@4       0049804c     kernel32:KERNEL32.dll
 0002:00000050       __imp__GetCommandLineA@0   00498050     kernel32:KERNEL32.dll
 0002:00000054       __imp__GetVersionExA@4     00498054     kernel32:KERNEL32.dll
 0002:00000058       __imp__GetProcessHeap@0    00498058     kernel32:KERNEL32.dll
 0002:0000005c       __imp__TerminateProcess@8  0049805c     kernel32:KERNEL32.dll
 0002:00000060       __imp__GetCurrentProcess@0 00498060     kernel32:KERNEL32.dll
 0002:00000064       __imp__UnhandledExceptionFilter@4 00498064     kernel32:KERNEL32.dll
 0002:00000068       __imp__SetUnhandledExceptionFilter@4 00498068     kernel32:KERNEL32.dll
 0002:0000006c       __imp__IsDebuggerPresent@0 0049806c     kernel32:KERNEL32.dll
 0002:00000070       __imp__HeapDestroy@4       00498070     kernel32:KERNEL32.dll
 0002:00000074       __imp__HeapCreate@12       00498074     kernel32:KERNEL32.dll
 0002:00000078       __imp__VirtualFree@12      00498078     kernel32:KERNEL32.dll
 0002:0000007c       __imp__DeleteCriticalSection@4 0049807c     kernel32:KERNEL32.dll
 0002:00000080       __imp__VirtualAlloc@16     00498080     kernel32:KERNEL32.dll
 0002:00000084       __imp__WriteFile@20        00498084     kernel32:KERNEL32.dll
 0002:00000088       __imp__GetStdHandle@4      00498088     kernel32:KERNEL32.dll
 0002:0000008c       __imp__GetModuleFileNameA@12 0049808c     kernel32:KERNEL32.dll
 0002:00000090       __imp__SetHandleCount@4    00498090     kernel32:KERNEL32.dll
 0002:00000094       __imp__GetStartupInfoA@4   00498094     kernel32:KERNEL32.dll
 0002:00000098       __imp__Sleep@4             00498098     kernel32:KERNEL32.dll
 0002:0000009c       __imp__TlsGetValue@4       0049809c     kernel32:KERNEL32.dll
 0002:000000a0       __imp__TlsAlloc@0          004980a0     kernel32:KERNEL32.dll
 0002:000000a4       __imp__TlsSetValue@8       004980a4     kernel32:KERNEL32.dll
 0002:000000a8       __imp__TlsFree@4           004980a8     kernel32:KERNEL32.dll
 0002:000000ac       __imp__InterlockedIncrement@4 004980ac     kernel32:KERNEL32.dll
 0002:000000b0       __imp__SetLastError@4      004980b0     kernel32:KERNEL32.dll
 0002:000000b4       __imp__GetCurrentThreadId@0 004980b4     kernel32:KERNEL32.dll
 0002:000000b8       __imp__InterlockedDecrement@4 004980b8     kernel32:KERNEL32.dll
 0002:000000bc       __imp__GetConsoleCP@0      004980bc     kernel32:KERNEL32.dll
 0002:000000c0       __imp__GetConsoleMode@8    004980c0     kernel32:KERNEL32.dll
 0002:000000c4       __imp__FlushFileBuffers@4  004980c4     kernel32:KERNEL32.dll
 0002:000000c8       __imp__MultiByteToWideChar@24 004980c8     kernel32:KERNEL32.dll
 0002:000000cc       __imp__ReadFile@20         004980cc     kernel32:KERNEL32.dll
 0002:000000d0       __imp__SetFilePointer@16   004980d0     kernel32:KERNEL32.dll
 0002:000000d4       __imp__HeapSize@12         004980d4     kernel32:KERNEL32.dll
 0002:000000d8       __imp__LoadLibraryA@4      004980d8     kernel32:KERNEL32.dll
 0002:000000dc       __imp__InitializeCriticalSection@4 004980dc     kernel32:KERNEL32.dll
 0002:000000e0       __imp__RaiseException@16   004980e0     kernel32:KERNEL32.dll
 0002:000000e4       __imp__GetCPInfo@8         004980e4     kernel32:KERNEL32.dll
 0002:000000e8       __imp__GetACP@0            004980e8     kernel32:KERNEL32.dll
 0002:000000ec       __imp__GetOEMCP@0          004980ec     kernel32:KERNEL32.dll
 0002:000000f0       __imp__IsValidCodePage@4   004980f0     kernel32:KERNEL32.dll
 0002:000000f4       __imp__SetStdHandle@8      004980f4     kernel32:KERNEL32.dll
 0002:000000f8       __imp__SetEndOfFile@4      004980f8     kernel32:KERNEL32.dll
 0002:000000fc       __imp__LCMapStringA@24     004980fc     kernel32:KERNEL32.dll
 0002:00000100       __imp__LCMapStringW@24     00498100     kernel32:KERNEL32.dll
 0002:00000104       __imp__FreeEnvironmentStringsA@4 00498104     kernel32:KERNEL32.dll
 0002:00000108       __imp__GetEnvironmentStrings@0 00498108     kernel32:KERNEL32.dll
 0002:0000010c       __imp__FreeEnvironmentStringsW@4 0049810c     kernel32:KERNEL32.dll
 0002:00000110       __imp__GetEnvironmentStringsW@0 00498110     kernel32:KERNEL32.dll
 0002:00000114       __imp__GetTickCount@0      00498114     kernel32:KERNEL32.dll
 0002:00000118       __imp__GetCurrentProcessId@0 00498118     kernel32:KERNEL32.dll
 0002:0000011c       __imp__WriteConsoleA@20    0049811c     kernel32:KERNEL32.dll
 0002:00000120       __imp__GetConsoleOutputCP@0 00498120     kernel32:KERNEL32.dll
 0002:00000124       __imp__WriteConsoleW@20    00498124     kernel32:KERNEL32.dll
 0002:00000128       __imp__CreateFileA@28      00498128     kernel32:KERNEL32.dll
 0002:0000012c       __imp__GetLocaleInfoA@16   0049812c     kernel32:KERNEL32.dll
 0002:00000130       __imp__CompareStringA@24   00498130     kernel32:KERNEL32.dll
 0002:00000134       __imp__CompareStringW@24   00498134     kernel32:KERNEL32.dll
 0002:00000138       __imp__SetEnvironmentVariableA@8 00498138     kernel32:KERNEL32.dll
 0002:0000013c       __imp__GetStringTypeA@20   0049813c     kernel32:KERNEL32.dll
 0002:00000140       __imp__GetStringTypeW@16   00498140     kernel32:KERNEL32.dll
 0002:00000144       \177KERNEL32_NULL_THUNK_DATA 00498144     kernel32:KERNEL32.dll
 0002:00000148       ___xc_a                    00498148     LIBCMT:crt0init.obj
 0002:0000014c       ___xc_z                    0049814c     LIBCMT:crt0init.obj
 0002:00000150       ___xi_a                    00498150     LIBCMT:crt0init.obj
 0002:0000016c       ___xi_z                    0049816c     LIBCMT:crt0init.obj
 0002:00000170       ___xp_a                    00498170     LIBCMT:crt0init.obj
 0002:0000017c       ___xp_z                    0049817c     LIBCMT:crt0init.obj
 0002:00000180       ___xt_a                    00498180     LIBCMT:crt0init.obj
 0002:00000184       ___xt_z                    00498184     LIBCMT:crt0init.obj
 0002:000001b0       ??_C@_0EA@FCLIIPNN@Visual?5C?$CL?$CL?5CRT?3?5Not?5enough?5memor@ 004981b0     LIBCMT:strerror.obj
 0002:000001f0       ??_C@_0P@MIGLKIOC@CorExitProcess?$AA@ 004981f0     LIBCMT:crt0dat.obj
 0002:00000200       ??_C@_0M@MBOPBNBK@mscoree?4dll?$AA@ 00498200     LIBCMT:crt0dat.obj
 0002:00000258       ___dnames                  00498258     LIBCMT:timeset.obj
 0002:00000270       ___mnames                  00498270     LIBCMT:timeset.obj
 0002:000002a0       ??_C@_0P@GGKDKEEG@runtime?5error?5?$AA@ 004982a0     LIBCMT:crt0msg.obj
 0002:000002b0       ??_C@_02PCIJFNDE@?$AN?6?$AA@ 004982b0     LIBCMT:crt0msg.obj
 0002:000002b4       ??_C@_0O@MJNIPGOH@TLOSS?5error?$AN?6?$AA@ 004982b4     LIBCMT:crt0msg.obj
 0002:000002c4       ??_C@_0N@BONNPDHF@SING?5error?$AN?6?$AA@ 004982c4     LIBCMT:crt0msg.obj
 0002:000002d4       ??_C@_0P@MBDAJNE@DOMAIN?5error?$AN?6?$AA@ 004982d4     LIBCMT:crt0msg.obj
 0002:000002e8       ??_C@_0JL@DFDOOABL@R6034?$AN?6An?5application?5has?5made?5a@ 004982e8     LIBCMT:crt0msg.obj
 0002:00000388       ??_C@_0PH@EPAFIJ@R6033?$AN?6?9?5Attempt?5to?5use?5MSIL?5cod@ 00498388     LIBCMT:crt0msg.obj
 0002:00000480       ??_C@_0DD@BKEEABMM@R6032?$AN?6?9?5not?5enough?5space?5for?5lo@ 00498480     LIBCMT:crt0msg.obj
 0002:000004b8       ??_C@_0GD@OFKILIED@R6031?$AN?6?9?5Attempt?5to?5initialize?5t@ 004984b8     LIBCMT:crt0msg.obj
 0002:0000051c       ??_C@_0BP@LPMHJOKI@R6030?$AN?6?9?5CRT?5not?5initialized?$AN?6?$AA@ 0049851c     LIBCMT:crt0msg.obj
 0002:0000053c       ??_C@_0CF@KJDAIALP@R6028?$AN?6?9?5unable?5to?5initialize?5he@ 0049853c     LIBCMT:crt0msg.obj
 0002:00000564       ??_C@_0DF@GAKBPDFP@R6027?$AN?6?9?5not?5enough?5space?5for?5lo@ 00498564     LIBCMT:crt0msg.obj
 0002:0000059c       ??_C@_0DF@IBLNNAIG@R6026?$AN?6?9?5not?5enough?5space?5for?5st@ 0049859c     LIBCMT:crt0msg.obj
 0002:000005d4       ??_C@_0CG@IOHKGFNJ@R6025?$AN?6?9?5pure?5virtual?5function?5c@ 004985d4     LIBCMT:crt0msg.obj
 0002:000005fc       ??_C@_0DF@JIJJFJDC@R6024?$AN?6?9?5not?5enough?5space?5for?5_o@ 004985fc     LIBCMT:crt0msg.obj
 0002:00000634       ??_C@_0CJ@EGEJHFME@R6019?$AN?6?9?5unable?5to?5open?5console?5@ 00498634     LIBCMT:crt0msg.obj
 0002:00000660       ??_C@_0CB@GNHNIELH@R6018?$AN?6?9?5unexpected?5heap?5error?$AN?6@ 00498660     LIBCMT:crt0msg.obj
 0002:00000684       ??_C@_0CN@FOLDKNG@R6017?$AN?6?9?5unexpected?5multithread?5@ 00498684     LIBCMT:crt0msg.obj
 0002:000006b4       ??_C@_0CM@FAHFJNHO@R6016?$AN?6?9?5not?5enough?5space?5for?5th@ 004986b4     LIBCMT:crt0msg.obj
 0002:000006e0       ??_C@_0JG@LBKMGKLD@?$AN?6This?5application?5has?5requested@ 004986e0     LIBCMT:crt0msg.obj
 0002:00000778       ??_C@_0CM@FLCNIPKK@R6009?$AN?6?9?5not?5enough?5space?5for?5en@ 00498778     LIBCMT:crt0msg.obj
 0002:000007a4       ??_C@_0CK@KMMJOAPP@R6008?$AN?6?9?5not?5enough?5space?5for?5ar@ 004987a4     LIBCMT:crt0msg.obj
 0002:000007d0       ??_C@_0CN@LEKKICBM@R6002?$AN?6?9?5floating?5point?5support?5@ 004987d0     LIBCMT:crt0msg.obj
 0002:00000800       ??_C@_0CF@GOGNBNAK@Microsoft?5Visual?5C?$CL?$CL?5Runtime?5Lib@ 00498800     LIBCMT:crt0msg.obj
 0002:00000828       ??_C@_02PHMGELLB@?6?6?$AA@ 00498828     LIBCMT:crt0msg.obj
 0002:0000082c       ??_C@_03KHICJKCI@?4?4?4?$AA@ 0049882c     LIBCMT:crt0msg.obj
 0002:00000830       ??_C@_0BH@DNAGHKFM@?$DMprogram?5name?5unknown?$DO?$AA@ 00498830     LIBCMT:crt0msg.obj
 0002:00000848       ??_C@_0BK@OFGJDLJJ@Runtime?5Error?$CB?6?6Program?3?5?$AA@ 00498848     LIBCMT:crt0msg.obj
 0002:00000864       ??_C@_1O@CEDCILHN@?$AA?$CI?$AAn?$AAu?$AAl?$AAl?$AA?$CJ?$AA?$AA@ 00498864     LIBCMT:output.obj
 0002:00000874       ??_C@_06OJHGLDPL@?$CInull?$CJ?$AA@ 00498874     LIBCMT:output.obj
 0002:00000880       ___lookuptable             00498880     LIBCMT:output.obj
 0002:000008dc       ??_C@_0BG@KLEAJEFJ@Illegal?5byte?5sequence?$AA@ 004988dc     LIBCMT:syserr.obj
 0002:000008f4       ??_C@_0BE@ICMCHPHH@Directory?5not?5empty?$AA@ 004988f4     LIBCMT:syserr.obj
 0002:00000908       ??_C@_0BJ@IHEHINLI@Function?5not?5implemented?$AA@ 00498908     LIBCMT:syserr.obj
 0002:00000924       ??_C@_0BD@CLHBCGPB@No?5locks?5available?$AA@ 00498924     LIBCMT:syserr.obj
 0002:00000938       ??_C@_0BC@BEDIHIDK@Filename?5too?5long?$AA@ 00498938     LIBCMT:syserr.obj
 0002:0000094c       ??_C@_0BK@JAEBMJJM@Resource?5deadlock?5avoided?$AA@ 0049894c     LIBCMT:syserr.obj
 0002:00000968       ??_C@_0BB@FCBJFCAJ@Result?5too?5large?$AA@ 00498968     LIBCMT:syserr.obj
 0002:0000097c       ??_C@_0N@MMJPGLJK@Domain?5error?$AA@ 0049897c     LIBCMT:syserr.obj
 0002:0000098c       ??_C@_0M@LHEPIIOM@Broken?5pipe?$AA@ 0049898c     LIBCMT:syserr.obj
 0002:00000998       ??_C@_0P@PKCJJLLM@Too?5many?5links?$AA@ 00498998     LIBCMT:syserr.obj
 0002:000009a8       ??_C@_0BG@DDBFNKBH@Read?9only?5file?5system?$AA@ 004989a8     LIBCMT:syserr.obj
 0002:000009c0       ??_C@_0N@FEHLOILP@Invalid?5seek?$AA@ 004989c0     LIBCMT:syserr.obj
 0002:000009d0       ??_C@_0BI@FEALHKLD@No?5space?5left?5on?5device?$AA@ 004989d0     LIBCMT:syserr.obj
 0002:000009e8       ??_C@_0P@LFMMIPAE@File?5too?5large?$AA@ 004989e8     LIBCMT:syserr.obj
 0002:000009f8       ??_C@_0CE@ONOKNLPF@Inappropriate?5I?1O?5control?5operat@ 004989f8     LIBCMT:syserr.obj
 0002:00000a1c       ??_C@_0BE@INBJMKGG@Too?5many?5open?5files?$AA@ 00498a1c     LIBCMT:syserr.obj
 0002:00000a30       ??_C@_0BO@IIFBODJE@Too?5many?5open?5files?5in?5system?$AA@ 00498a30     LIBCMT:syserr.obj
 0002:00000a50       ??_C@_0BB@HMGGCEBG@Invalid?5argument?$AA@ 00498a50     LIBCMT:syserr.obj
 0002:00000a64       ??_C@_0P@NDHGCGKE@Is?5a?5directory?$AA@ 00498a64     LIBCMT:syserr.obj
 0002:00000a74       ??_C@_0BA@CJBACOOL@Not?5a?5directory?$AA@ 00498a74     LIBCMT:syserr.obj
 0002:00000a84       ??_C@_0P@NLEIANHE@No?5such?5device?$AA@ 00498a84     LIBCMT:syserr.obj
 0002:00000a94       ??_C@_0O@OAMDNOCP@Improper?5link?$AA@ 00498a94     LIBCMT:syserr.obj
 0002:00000aa4       ??_C@_0M@NAAJNNGH@File?5exists?$AA@ 00498aa4     LIBCMT:syserr.obj
 0002:00000ab0       ??_C@_0BA@BIBLIOEK@Resource?5device?$AA@ 00498ab0     LIBCMT:syserr.obj
 0002:00000ac0       ??_C@_0O@NIPGCINC@Unknown?5error?$AA@ 00498ac0     LIBCMT:syserr.obj
 0002:00000ad0       ??_C@_0M@LOEHLCJD@Bad?5address?$AA@ 00498ad0     LIBCMT:syserr.obj
 0002:00000adc       ??_C@_0BC@HFNFNKAI@Permission?5denied?$AA@ 00498adc     LIBCMT:syserr.obj
 0002:00000af0       ??_C@_0BB@IMDKMPFB@Not?5enough?5space?$AA@ 00498af0     LIBCMT:syserr.obj
 0002:00000b04       ??_C@_0CB@EPFKGNAK@Resource?5temporarily?5unavailable@ 00498b04     LIBCMT:syserr.obj
 0002:00000b28       ??_C@_0BD@LOHELEP@No?5child?5processes?$AA@ 00498b28     LIBCMT:syserr.obj
 0002:00000b3c       ??_C@_0BE@NFGDDCEF@Bad?5file?5descriptor?$AA@ 00498b3c     LIBCMT:syserr.obj
 0002:00000b50       ??_C@_0BC@HKPNECK@Exec?5format?5error?$AA@ 00498b50     LIBCMT:syserr.obj
 0002:00000b64       ??_C@_0BC@MFFGCDFL@Arg?5list?5too?5long?$AA@ 00498b64     LIBCMT:syserr.obj
 0002:00000b78       ??_C@_0BK@DPKMCKJ@No?5such?5device?5or?5address?$AA@ 00498b78     LIBCMT:syserr.obj
 0002:00000b94       ??_C@_0BD@KKNFOBBD@Input?1output?5error?$AA@ 00498b94     LIBCMT:syserr.obj
 0002:00000ba8       ??_C@_0BK@FJBOAFDK@Interrupted?5function?5call?$AA@ 00498ba8     LIBCMT:syserr.obj
 0002:00000bc4       ??_C@_0BA@FKIAIBGA@No?5such?5process?$AA@ 00498bc4     LIBCMT:syserr.obj
 0002:00000bd4       ??_C@_0BK@FMDHKPNF@No?5such?5file?5or?5directory?$AA@ 00498bd4     LIBCMT:syserr.obj
 0002:00000bf0       ??_C@_0BI@BJFCGOHL@Operation?5not?5permitted?$AA@ 00498bf0     LIBCMT:syserr.obj
 0002:00000c08       ??_C@_08INEPGKHH@No?5error?$AA@ 00498c08     LIBCMT:syserr.obj
 0002:00000c14       ??_C@_07EPKMNAGK@?4mixcrt?$AA@ 00498c14     LIBCMT:tidtable.obj
 0002:00000c1c       ??_C@_0O@NLDKAIKN@EncodePointer?$AA@ 00498c1c     LIBCMT:tidtable.obj
 0002:00000c2c       ??_C@_0N@NHGLKGEC@KERNEL32?4DLL?$AA@ 00498c2c     LIBCMT:tidtable.obj
 0002:00000c3c       ??_C@_0O@KBPMFGHI@DecodePointer?$AA@ 00498c3c     LIBCMT:tidtable.obj
 0002:00000c4c       ??_C@_07PEJMOBNF@FlsFree?$AA@ 00498c4c     LIBCMT:tidtable.obj
 0002:00000c54       ??_C@_0M@JCPCPOEF@FlsSetValue?$AA@ 00498c54     LIBCMT:tidtable.obj
 0002:00000c60       ??_C@_0M@GDNOONDI@FlsGetValue?$AA@ 00498c60     LIBCMT:tidtable.obj
 0002:00000c6c       ??_C@_08KNHFBNJ@FlsAlloc?$AA@ 00498c6c     LIBCMT:tidtable.obj
 0002:00000c9c       ??_C@_0CG@PKBDLMEO@InitializeCriticalSectionAndSpin@ 00498c9c     LIBCMT:initcrit.obj
 0002:00000cc4       ??_C@_0N@MDJJJHMB@kernel32?4dll?$AA@ 00498cc4     LIBCMT:initcrit.obj
 0002:00000cd4       __FPinit                   00498cd4     LIBCMT:fpinit.obj
 0002:00000cd8       __FPmtinit                 00498cd8     LIBCMT:fpinit.obj
 0002:00000cdc       __FPmtterm                 00498cdc     LIBCMT:fpinit.obj
 0002:00000ce0       ??_C@_0L@KDOEJCKC@_nextafter?$AA@ 00498ce0     LIBCMT:fpexcept.obj
 0002:00000cec       ??_C@_05JGDBENOH@_logb?$AA@ 00498cec     LIBCMT:fpexcept.obj
 0002:00000cf4       ??_C@_03ONILCKOB@_yn?$AA@  00498cf4     LIBCMT:fpexcept.obj
 0002:00000cf8       ??_C@_03NAKIGLHK@_y1?$AA@  00498cf8     LIBCMT:fpexcept.obj
 0002:00000cfc       ??_C@_03MJLDFKDL@_y0?$AA@  00498cfc     LIBCMT:fpexcept.obj
 0002:00000d00       ??_C@_05GKKHEGJL@frexp?$AA@ 00498d00     LIBCMT:fpexcept.obj
 0002:00000d08       ??_C@_04KEPJIHGP@fmod?$AA@ 00498d08     LIBCMT:fpexcept.obj
 0002:00000d10       ??_C@_06MEIMCGCF@_hypot?$AA@ 00498d10     LIBCMT:fpexcept.obj
 0002:00000d18       ??_C@_05KBKMEMPO@_cabs?$AA@ 00498d18     LIBCMT:fpexcept.obj
 0002:00000d20       ??_C@_05CEJMAHNP@ldexp?$AA@ 00498d20     LIBCMT:fpexcept.obj
 0002:00000d28       ??_C@_04EHEDPDJG@modf?$AA@ 00498d28     LIBCMT:fpexcept.obj
 0002:00000d30       ??_C@_04ODHECPBC@fabs?$AA@ 00498d30     LIBCMT:fpexcept.obj
 0002:00000d38       ??_C@_05PBJFFIGL@floor?$AA@ 00498d38     LIBCMT:fpexcept.obj
 0002:00000d40       ??_C@_04GFPJNGEK@ceil?$AA@ 00498d40     LIBCMT:fpexcept.obj
 0002:00000d48       ??_C@_03IIINPABG@tan?$AA@  00498d48     LIBCMT:fpexcept.obj
 0002:00000d4c       ??_C@_03LALBNOCG@cos?$AA@  00498d4c     LIBCMT:fpexcept.obj
 0002:00000d50       ??_C@_03BLEJJJBH@sin?$AA@  00498d50     LIBCMT:fpexcept.obj
 0002:00000d54       ??_C@_04EIAKFFMI@sqrt?$AA@ 00498d54     LIBCMT:fpexcept.obj
 0002:00000d5c       ??_C@_05KNGEOGJB@atan2?$AA@ 00498d5c     LIBCMT:fpexcept.obj
 0002:00000d64       ??_C@_04MLLJIGOK@atan?$AA@ 00498d64     LIBCMT:fpexcept.obj
 0002:00000d6c       ??_C@_04PDIFKINK@acos?$AA@ 00498d6c     LIBCMT:fpexcept.obj
 0002:00000d74       ??_C@_04FIHNOPOL@asin?$AA@ 00498d74     LIBCMT:fpexcept.obj
 0002:00000d7c       ??_C@_04FJHINJAO@tanh?$AA@ 00498d7c     LIBCMT:fpexcept.obj
 0002:00000d84       ??_C@_04HPJJNFIM@cosh?$AA@ 00498d84     LIBCMT:fpexcept.obj
 0002:00000d8c       ??_C@_04COOMCNPB@sinh?$AA@ 00498d8c     LIBCMT:fpexcept.obj
 0002:00000d94       ??_C@_05HGHHAHAP@log10?$AA@ 00498d94     LIBCMT:fpexcept.obj
 0002:00000d9c       ??_C@_03MGHMBJCF@log?$AA@  00498d9c     LIBCMT:fpexcept.obj
 0002:00000da0       ??_C@_03JGHBODFD@pow?$AA@  00498da0     LIBCMT:fpexcept.obj
 0002:00000da4       ??_C@_03KHJOGHMM@exp?$AA@  00498da4     LIBCMT:fpexcept.obj
 0002:00000e10       ??_C@_05EOHGHCHD@exp10?$AA@ 00498e10     LIBCMT:libm_error.obj
 0002:00000e18       ___lookuptable_s           00498e18     LIBCMT:outputs.obj
 0002:00000ef8       ??_C@_13NOLLCAOD@?$AA?$AA?$AA?$AA@ 00498ef8     LIBCMT:a_map.obj
 0002:00000efc       ??_C@_0BI@DFKBFLJE@GetProcessWindowStation?$AA@ 00498efc     LIBCMT:crtmbox.obj
 0002:00000f14       ??_C@_0BK@CIDNPOGP@GetUserObjectInformationA?$AA@ 00498f14     LIBCMT:crtmbox.obj
 0002:00000f30       ??_C@_0BD@HHGDFDBJ@GetLastActivePopup?$AA@ 00498f30     LIBCMT:crtmbox.obj
 0002:00000f44       ??_C@_0BA@HNOPNCHB@GetActiveWindow?$AA@ 00498f44     LIBCMT:crtmbox.obj
 0002:00000f54       ??_C@_0M@CHKKJDAI@MessageBoxA?$AA@ 00498f54     LIBCMT:crtmbox.obj
 0002:00000f60       ??_C@_0L@NDEGIDAG@USER32?4DLL?$AA@ 00498f60     LIBCMT:crtmbox.obj
 0002:00000f6c       ??_C@_05KLBDPFGC@e?$CL000?$AA@ 00498f6c     LIBCMT:cvt.obj
 0002:00000f78       __real@4150017ec0000000    00498f78     LIBCMT:testfdiv.obj
 0002:00000f80       __real@4147ffff80000000    00498f80     LIBCMT:testfdiv.obj
 0002:00000f88       ??_C@_0BK@NHEOCAHP@IsProcessorFeaturePresent?$AA@ 00498f88     LIBCMT:testfdiv.obj
 0002:00000fa4       ??_C@_08CPNIBGIE@KERNEL32?$AA@ 00498fa4     LIBCMT:testfdiv.obj
 0002:00000fb0       ___newctype                00498fb0     LIBCMT:ctype.obj
 0002:000012b0       __wctype                   004992b0     LIBCMT:ctype.obj
 0002:000014b8       ___newclmap                004994b8     LIBCMT:ctype.obj
 0002:00001638       ___newcumap                00499638     LIBCMT:ctype.obj
 0002:000017b8       ??_C@_08JCCMCCIL@HH?3mm?3ss?$AA@ 004997b8     LIBCMT:strftime.obj
 0002:000017c4       ??_C@_0BE@CKGJFCPC@dddd?0?5MMMM?5dd?0?5yyyy?$AA@ 004997c4     LIBCMT:strftime.obj
 0002:000017d8       ??_C@_08BPBNCDIB@MM?1dd?1yy?$AA@ 004997d8     LIBCMT:strftime.obj
 0002:000017e4       ??_C@_02CJNFDJBF@PM?$AA@   004997e4     LIBCMT:strftime.obj
 0002:000017e8       ??_C@_02DEDBPAFC@AM?$AA@   004997e8     LIBCMT:strftime.obj
 0002:000017ec       ??_C@_08EDHMEBNP@December?$AA@ 004997ec     LIBCMT:strftime.obj
 0002:000017f8       ??_C@_08HCHEGEOA@November?$AA@ 004997f8     LIBCMT:strftime.obj
 0002:00001804       ??_C@_07JJNFCEND@October?$AA@ 00499804     LIBCMT:strftime.obj
 0002:0000180c       ??_C@_09BHHEALKD@September?$AA@ 0049980c     LIBCMT:strftime.obj
 0002:00001818       ??_C@_06LBBHFDDG@August?$AA@ 00499818     LIBCMT:strftime.obj
 0002:00001820       ??_C@_04MIEPOIFP@July?$AA@ 00499820     LIBCMT:strftime.obj
 0002:00001828       ??_C@_04CNLMGBGM@June?$AA@ 00499828     LIBCMT:strftime.obj
 0002:00001830       ??_C@_05DMJDNLEJ@April?$AA@ 00499830     LIBCMT:strftime.obj
 0002:00001838       ??_C@_05HPCKOFNC@March?$AA@ 00499838     LIBCMT:strftime.obj
 0002:00001840       ??_C@_08GNJGEPFN@February?$AA@ 00499840     LIBCMT:strftime.obj
 0002:0000184c       ??_C@_07CGJPFGJA@January?$AA@ 0049984c     LIBCMT:strftime.obj
 0002:00001854       ??_C@_03MKABNOCG@Dec?$AA@  00499854     LIBCMT:strftime.obj
 0002:00001858       ??_C@_03JPJOFNIA@Nov?$AA@  00499858     LIBCMT:strftime.obj
 0002:0000185c       ??_C@_03BMAOKBAD@Oct?$AA@  0049985c     LIBCMT:strftime.obj
 0002:00001860       ??_C@_03GGCAPAJC@Sep?$AA@  00499860     LIBCMT:strftime.obj
 0002:00001864       ??_C@_03IFJFEIGA@Aug?$AA@  00499864     LIBCMT:strftime.obj
 0002:00001868       ??_C@_03LBGABGKK@Jul?$AA@  00499868     LIBCMT:strftime.obj
 0002:0000186c       ??_C@_03IDFGHECI@Jun?$AA@  0049986c     LIBCMT:strftime.obj
 0002:00001870       ??_C@_03CNMDKL@May?$AA@    00499870     LIBCMT:strftime.obj
 0002:00001874       ??_C@_03LEOLGMJP@Apr?$AA@  00499874     LIBCMT:strftime.obj
 0002:00001878       ??_C@_03ODNJBKGA@Mar?$AA@  00499878     LIBCMT:strftime.obj
 0002:0000187c       ??_C@_03HJBDCHOM@Feb?$AA@  0049987c     LIBCMT:strftime.obj
 0002:00001880       ??_C@_03JIHJHPIE@Jan?$AA@  00499880     LIBCMT:strftime.obj
 0002:00001884       ??_C@_08INBOOONO@Saturday?$AA@ 00499884     LIBCMT:strftime.obj
 0002:00001890       ??_C@_06JECMNKMI@Friday?$AA@ 00499890     LIBCMT:strftime.obj
 0002:00001898       ??_C@_08HACCIKIA@Thursday?$AA@ 00499898     LIBCMT:strftime.obj
 0002:000018a4       ??_C@_09DLIGFAKA@Wednesday?$AA@ 004998a4     LIBCMT:strftime.obj
 0002:000018b0       ??_C@_07BAAGCFCM@Tuesday?$AA@ 004998b0     LIBCMT:strftime.obj
 0002:000018b8       ??_C@_06JLEDEDGH@Monday?$AA@ 004998b8     LIBCMT:strftime.obj
 0002:000018c0       ??_C@_06OOPIFAJ@Sunday?$AA@ 004998c0     LIBCMT:strftime.obj
 0002:000018c8       ??_C@_03FEFJNEK@Sat?$AA@   004998c8     LIBCMT:strftime.obj
 0002:000018cc       ??_C@_03IDIOELNC@Fri?$AA@  004998cc     LIBCMT:strftime.obj
 0002:000018d0       ??_C@_03IOFIKPDN@Thu?$AA@  004998d0     LIBCMT:strftime.obj
 0002:000018d4       ??_C@_03MHOMLAJA@Wed?$AA@  004998d4     LIBCMT:strftime.obj
 0002:000018d8       ??_C@_03NAGEINEP@Tue?$AA@  004998d8     LIBCMT:strftime.obj
 0002:000018dc       ??_C@_03PDAGKDH@Mon?$AA@   004998dc     LIBCMT:strftime.obj
 0002:000018e0       ??_C@_03KOEHGMDN@Sun?$AA@  004998e0     LIBCMT:strftime.obj
 0002:000018e4       ??_C@_07GPDNMNG@CONOUT$?$AA@ 004998e4     LIBCMT:initcon.obj
 0002:000018ec       ??_C@_06IMKFLFPG@1?$CDQNAN?$AA@ 004998ec     LIBCMT:x10fout.obj
 0002:000018f4       ??_C@_05DNEBIAHO@1?$CDINF?$AA@ 004998f4     LIBCMT:x10fout.obj
 0002:000018fc       ??_C@_05PHHOCPM@1?$CDIND?$AA@ 004998fc     LIBCMT:x10fout.obj
 0002:00001904       ??_C@_06PGGFOGJG@1?$CDSNAN?$AA@ 00499904     LIBCMT:x10fout.obj
 0002:00001918       __DEFAULT_CW_in_mem        00499918     LIBCMT:common.obj
 0002:0000191a       __pi_by_2_to_61            0049991a     LIBCMT:common.obj
 0002:000ca868       _pdf_font_NimbusRomNo9L_Regu_cff_buf 00562868     font_serif.obj
 0002:000d0b18       _pdf_font_NimbusRomNo9L_Regu_cff_len 00568b18     font_serif.obj
 0002:000d0b1c       _pdf_font_NimbusRomNo9L_Medi_cff_len 00568b1c     font_serif.obj
 0002:000d0b20       _pdf_font_NimbusRomNo9L_Medi_cff_buf 00568b20     font_serif.obj
 0002:000d6a24       _pdf_font_NimbusRomNo9L_ReguItal_cff_len 0056ea24     font_serif.obj
 0002:000d6a28       _pdf_font_NimbusRomNo9L_ReguItal_cff_buf 0056ea28     font_serif.obj
 0002:000dd618       _pdf_font_NimbusRomNo9L_MediItal_cff_buf 00575618     font_serif.obj
 0002:000e4008       _pdf_font_NimbusRomNo9L_MediItal_cff_len 0057c008     font_serif.obj
 0002:000e400c       _pdf_font_NimbusSanL_Regu_cff_len 0057c00c     font_sans.obj
 0002:000e4010       _pdf_font_NimbusSanL_Regu_cff_buf 0057c010     font_sans.obj
 0002:000e80f0       _pdf_font_NimbusSanL_Bold_cff_buf 005800f0     font_sans.obj
 0002:000ec534       _pdf_font_NimbusSanL_Bold_cff_len 00584534     font_sans.obj
 0002:000ec538       _pdf_font_NimbusSanL_ReguItal_cff_buf 00584538     font_sans.obj
 0002:000f13f8       _pdf_font_NimbusSanL_ReguItal_cff_len 005893f8     font_sans.obj
 0002:000f13fc       _pdf_font_NimbusSanL_BoldItal_cff_len 005893fc     font_sans.obj
 0002:000f1400       _pdf_font_NimbusSanL_BoldItal_cff_buf 00589400     font_sans.obj
 0002:000f6200       _pdf_font_NimbusMonL_Regu_cff_buf 0058e200     font_mono.obj
 0002:000fc610       _pdf_font_NimbusMonL_Regu_cff_len 00594610     font_mono.obj
 0002:000fc614       _pdf_font_NimbusMonL_Bold_cff_len 00594614     font_mono.obj
 0002:000fc618       _pdf_font_NimbusMonL_Bold_cff_buf 00594618     font_mono.obj
 0002:00104674       _pdf_font_NimbusMonL_ReguObli_cff_len 0059c674     font_mono.obj
 0002:00104678       _pdf_font_NimbusMonL_ReguObli_cff_buf 0059c678     font_mono.obj
 0002:0010b578       _pdf_font_NimbusMonL_BoldObli_cff_buf 005a3578     font_mono.obj
 0002:001138a8       _pdf_font_NimbusMonL_BoldObli_cff_len 005ab8a8     font_mono.obj
 0002:001138ac       _pdf_font_StandardSymL_cff_len 005ab8ac     font_misc.obj
 0002:001138b0       _pdf_font_StandardSymL_cff_buf 005ab8b0     font_misc.obj
 0002:001182b0       _pdf_font_Dingbats_cff_buf 005b02b0     font_misc.obj
 0002:0011f5e4       _pdf_font_Dingbats_cff_len 005b75e4     font_misc.obj
 0002:0011f5e8       _pdf_font_URWChanceryL_MediItal_cff_buf 005b75e8     font_misc.obj
 0002:00127c6c       _pdf_font_URWChanceryL_MediItal_cff_len 005bfc6c     font_misc.obj
 0002:00127da8       _pdf_docencoding           005bfda8     pdf_fontenc.obj
 0002:00127fa8       _pdf_macroman              005bffa8     pdf_fontenc.obj
 0002:001283a8       _pdf_macexpert             005c03a8     pdf_fontenc.obj
 0002:001287a8       _pdf_winansi               005c07a8     pdf_fontenc.obj
 0002:00128ba8       _pdf_standard              005c0ba8     pdf_fontenc.obj
 0002:001337f0       _cf_run_eol                005cb7f0     filt_faxetab.obj
 0002:001337f4       _cf2_run_pass              005cb7f4     filt_faxetab.obj
 0002:001337f8       _cf2_run_vertical          005cb7f8     filt_faxetab.obj
 0002:00133814       _cf2_run_horizontal        005cb814     filt_faxetab.obj
 0002:00133818       _cf2_run_eol_1d            005cb818     filt_faxetab.obj
 0002:0013381c       _cf2_run_eol_2d            005cb81c     filt_faxetab.obj
 0002:00133820       _cf_white_runs             005cb820     filt_faxetab.obj
 0002:001339c4       _jbig2_huffman_lines_A     005cb9c4     jbig2_huffman.obj
 0002:00133a00       _cf_black_runs             005cba00     filt_faxetab.obj
 0002:00133ba4       _cf_uncompressed           005cbba4     filt_faxetab.obj
 0002:00133bbc       _cf_uncompressed_exit      005cbbbc     filt_faxetab.obj
 0002:00133bf4       _jbig2_huffman_params_A    005cbbf4     jbig2_huffman.obj
 0002:00133c00       _cf_white_decode           005cbc00     filt_faxdtab.obj
 0002:001340c0       _cf_black_decode           005cc0c0     filt_faxdtab.obj
 0002:001345c0       _cf_2d_decode              005cc5c0     filt_faxdtab.obj
 0002:00134820       _cf_uncompressed_decode    005cc820     filt_faxdtab.obj
 0002:00136120       _jbig2_mmr_white_decode    005ce120     jbig2_mmr.obj
 0002:001365e0       _jbig2_mmr_black_decode    005ce5e0     jbig2_mmr.obj
 0002:00136af0       _jbig2_huffman_lines_B     005ceaf0     jbig2_huffman.obj
 0002:00136b50       _jbig2_huffman_params_B    005ceb50     jbig2_huffman.obj
 0002:00136b5c       _jbig2_huffman_params_C    005ceb5c     jbig2_huffman.obj
 0002:00136b68       _jbig2_huffman_lines_C     005ceb68     jbig2_huffman.obj
 0002:00136bd4       _jbig2_huffman_params_D    005cebd4     jbig2_huffman.obj
 0002:00136be0       _jbig2_huffman_lines_D     005cebe0     jbig2_huffman.obj
 0002:00136c34       _jbig2_huffman_params_E    005cec34     jbig2_huffman.obj
 0002:00136c40       _jbig2_huffman_lines_E     005cec40     jbig2_huffman.obj
 0002:00136ca0       _jbig2_huffman_lines_F     005ceca0     jbig2_huffman.obj
 0002:00136d48       _jbig2_huffman_params_F    005ced48     jbig2_huffman.obj
 0002:00136d54       _jbig2_huffman_params_G    005ced54     jbig2_huffman.obj
 0002:00136d60       _jbig2_huffman_lines_G     005ced60     jbig2_huffman.obj
 0002:00136e14       _jbig2_huffman_params_H    005cee14     jbig2_huffman.obj
 0002:00136e20       _jbig2_huffman_lines_H     005cee20     jbig2_huffman.obj
 0002:00136f1c       _jbig2_huffman_params_I    005cef1c     jbig2_huffman.obj
 0002:00136f28       _jbig2_huffman_lines_I     005cef28     jbig2_huffman.obj
 0002:00137030       _jbig2_huffman_lines_J     005cf030     jbig2_huffman.obj
 0002:0013712c       _jbig2_huffman_params_J    005cf12c     jbig2_huffman.obj
 0002:00137138       _jbig2_huffman_lines_K     005cf138     jbig2_huffman.obj
 0002:001371d4       _jbig2_huffman_params_K    005cf1d4     jbig2_huffman.obj
 0002:001371e0       _jbig2_huffman_lines_L     005cf1e0     jbig2_huffman.obj
 0002:0013727c       _jbig2_huffman_params_L    005cf27c     jbig2_huffman.obj
 0002:00137288       _jbig2_huffman_lines_M     005cf288     jbig2_huffman.obj
 0002:00137324       _jbig2_huffman_params_M    005cf324     jbig2_huffman.obj
 0002:00137330       _jbig2_huffman_lines_N     005cf330     jbig2_huffman.obj
 0002:00137384       _jbig2_huffman_params_N    005cf384     jbig2_huffman.obj
 0002:00137390       _jbig2_huffman_lines_O     005cf390     jbig2_huffman.obj
 0002:0013742c       _jbig2_huffman_params_O    005cf42c     jbig2_huffman.obj
 0002:00137438       _jbig2_arith_Qe            005cf438     jbig2_arith.obj
 0002:00137510       _jpeg_natural_order        005cf510     jutils.obj
 0002:00137750       _jpeg_std_message_table    005cf750     jerror.obj
 0002:00137f78       _winfnt_driver_class       005cff78     winfnt.obj
 0002:00138188       _t42_driver_class          005d0188     type42.obj
 0002:00138508       _t1_driver_class           005d0508     type1.obj
 0002:00138c88       _tt_driver_class           005d0c88     truetype.obj
 0002:00138d40       _tt_default_graphics_state 005d0d40     truetype.obj
 0002:00138fec       _ft_grays_raster           005d0fec     smooth.obj
 0002:00139004       _ft_smooth_renderer_class  005d1004     smooth.obj
 0002:00139040       _ft_smooth_lcd_renderer_class 005d1040     smooth.obj
 0002:0013907c       _ft_smooth_lcdv_renderer_class 005d107c     smooth.obj
 0002:00139170       _sfnt_module_class         005d1170     sfnt.obj
 0002:00139274       _tt_cmap0_class_rec        005d1274     sfnt.obj
 0002:001392e8       _tt_cmap2_class_rec        005d12e8     sfnt.obj
 0002:0013931c       _tt_cmap4_class_rec        005d131c     sfnt.obj
 0002:00139350       _tt_cmap6_class_rec        005d1350     sfnt.obj
 0002:00139384       _tt_cmap8_class_rec        005d1384     sfnt.obj
 0002:001393b8       _tt_cmap10_class_rec       005d13b8     sfnt.obj
 0002:001393ec       _tt_cmap12_class_rec       005d13ec     sfnt.obj
 0002:00139420       _tt_cmap14_class_rec       005d1420     sfnt.obj
 0002:00139608       _ft_standard_raster        005d1608     raster.obj
 0002:00139620       _ft_raster1_renderer_class 005d1620     raster.obj
 0002:0013965c       _ft_raster5_renderer_class 005d165c     raster.obj
 0002:00139ab8       _psnames_module_class      005d1ab8     psnames.obj
 0002:0013ab5c       _pshinter_module_class     005d2b5c     pshinter.obj
 0002:00148550       _ps_table_funcs            005e0550     psaux.obj
 0002:00148560       _ps_parser_funcs           005e0560     psaux.obj
 0002:00148594       _t1_builder_funcs          005e0594     psaux.obj
 0002:001485b4       _t1_decoder_funcs          005e05b4     psaux.obj
 0002:001485c0       _t1_cmap_standard_class_rec 005e05c0     psaux.obj
 0002:001485e8       _t1_cmap_expert_class_rec  005e05e8     psaux.obj
 0002:00148610       _t1_cmap_custom_class_rec  005e0610     psaux.obj
 0002:00148638       _t1_cmap_unicode_class_rec 005e0638     psaux.obj
 0002:00148660       _t1_cmap_classes           005e0660     psaux.obj
 0002:00148670       _afm_parser_funcs          005e0670     psaux.obj
 0002:00148698       _psaux_module_class        005e0698     psaux.obj
 0002:001486bc       _pfr_metrics_service_rec   005e06bc     pfr.obj
 0002:001488f8       _pfr_driver_class          005e08f8     pfr.obj
 0002:001489fc       _pfr_cmap_class_rec        005e09fc     pfr.obj
 0002:00148a50       _pcf_driver_class          005e0a50     pcf.obj
 0002:00148b9c       _pcf_cmap_class            005e0b9c     pcf.obj
 0002:00148c60       _t1cid_driver_class        005e0c60     type1cid.obj
 0002:00149a10       _cff_driver_class          005e1a10     cff.obj
 0002:00149b04       _ftc_size_list_class       005e1b04     ftcache.obj
 0002:0014a3e4       _ftc_face_list_class       005e23e4     ftcache.obj
 0002:0014a8f8       _cff_cmap_encoding_class_rec 005e28f8     cff.obj
 0002:0014a920       _cff_cmap_unicode_class_rec 005e2920     cff.obj
 0002:0014a948       _ftc_cmap_cache_class      005e2948     ftcache.obj
 0002:0014a968       _ftc_basic_image_family_class 005e2968     ftcache.obj
 0002:0014a980       _ftc_basic_image_cache_class 005e2980     ftcache.obj
 0002:0014a9a4       _ftc_basic_sbit_family_class 005e29a4     ftcache.obj
 0002:0014a9c0       _ftc_basic_sbit_cache_class 005e29c0     ftcache.obj
 0002:0014a9e8       _bdf_driver_class          005e29e8     bdf.obj
 0002:0014b078       _bdf_cmap_class            005e3078     bdf.obj
 0002:0014b0d4       _autofit_module_class      005e30d4     autofit.obj
 0002:0014b158       _af_autofitter_service     005e3158     autofit.obj
 0002:0014b168       _af_dummy_script_class     005e3168     autofit.obj
 0002:0014b1a0       _af_latin2_script_class    005e31a0     autofit.obj
 0002:0014b298       _af_latin_script_class     005e3298     autofit.obj
 0002:0014b360       _af_cjk_script_class       005e3360     autofit.obj
 0002:0014b390       _af_indic_script_class     005e3390     autofit.obj
 0002:0014b484       _ft_bitmap_glyph_class     005e3484     ftglyph.obj
 0002:0014b4a4       _ft_outline_glyph_class    005e34a4     ftglyph.obj
 0002:0014bb18       __dist_code                005e3b18     trees.obj
 0002:0014bd18       __length_code              005e3d18     trees.obj
 0002:0014bf08       _deflate_copyright         005e3f08     deflate.obj
 0002:0014bfc0       _inflate_copyright         005e3fc0     inftrees.obj
 0002:0014c0f0       _z_errmsg                  005e40f0     zutil.obj
 0002:0014e9c0       __real@408f400000000000    005e69c0      CIL library: CIL module
 0002:0014e9c8       __real@3ffc5a1ca0000000    005e69c8      CIL library: CIL module
 0002:0014e9d0       __real@3fe6da3c20000000    005e69d0      CIL library: CIL module
 0002:0014e9d8       __real@3fd60639e0000000    005e69d8      CIL library: CIL module
 0002:0014e9e0       __real@3ff66e9780000000    005e69e0      CIL library: CIL module
 0002:0014e9e8       __real@409f400000000000    005e69e8      CIL library: CIL module
 0002:0014e9f0       __real@3fc4cccccccccccd    005e69f0      CIL library: CIL module
 0002:0014e9f8       __real@3fe0000000000000    005e69f8      CIL library: CIL module
 0002:0014ea00       __real@4008000000000000    005e6a00      CIL library: CIL module
 0002:0014ea08       __real@3fc1a7b9611a7b96    005e6a08      CIL library: CIL module
 0002:0014ea10       __real@401f25e353f7ced9    005e6a10      CIL library: CIL module
 0002:0014ea18       __real@3fd5555555555555    005e6a18      CIL library: CIL module
 0002:0014ea20       __real@3f82231832fcac8e    005e6a20      CIL library: CIL module
 0002:0014ea28       __real@3fc07004ded20922    005e6a28      CIL library: CIL module
 0002:0014ea30       __real@3fca7b9611a7b961    005e6a30      CIL library: CIL module
 0002:0014ea38       __real@3ff0000000000000    005e6a38      CIL library: CIL module
 0002:0014ea40       __real@3fbc28f5c28f5c29    005e6a40      CIL library: CIL module
 0002:0014ea48       __real@3fd3333333333333    005e6a48      CIL library: CIL module
 0002:0014ea50       __real@3fe2e147ae147ae1    005e6a50      CIL library: CIL module
 0002:0014ea58       __real@0000000000000000    005e6a58      CIL library: CIL module
 0002:0014ea60       __real@3e80000000000000    005e6a60      CIL library: CIL module
 0002:0014ea68       __real@4000000000000000    005e6a68      CIL library: CIL module
 0002:0014ea70       __real@406fe00000000000    005e6a70      CIL library: CIL module
 0002:0014ea78       __real@3ff1517a80000000    005e6a78      CIL library: CIL module
 0002:0014ea80       __real@4004e7aea0000000    005e6a80      CIL library: CIL module
 0002:0014ea88       __real@3ffd906bc0000000    005e6a88      CIL library: CIL module
 0002:0014ea90       __real@3ff6a09e60000000    005e6a90      CIL library: CIL module
 0002:0014ea98       __real@3f40000000000000    005e6a98      CIL library: CIL module
 0002:0014eaa0       __real@3fc6571840000000    005e6aa0      CIL library: CIL module
 0002:0014eaa8       __real@400921fb54442d18    005e6aa8      CIL library: CIL module
 0002:0014eab0       __real@3ff921fb54442d18    005e6ab0      CIL library: CIL module
 0002:0014eab8       __real@4059000000000000    005e6ab8      CIL library: CIL module
 0002:0014eac0       __real@4069000000000000    005e6ac0      CIL library: CIL module
 0002:0014eac8       __real@407f400000000000    005e6ac8      CIL library: CIL module
 0002:0014ead0       __real@408c3a6666666666    005e6ad0      CIL library: CIL module
 0002:0014ead8       __real@4030000000000000    005e6ad8      CIL library: CIL module
 0002:0014eae0       __real@405d000000000000    005e6ae0      CIL library: CIL module
 0002:0014eae8       __real@bf800000            005e6ae8      CIL library: CIL module
 0002:0014eaec       __real@41200000            005e6aec      CIL library: CIL module
 0002:0014eaf0       __real@402e000000000000    005e6af0      CIL library: CIL module
 0002:0014eaf8       __real@4031000000000000    005e6af8      CIL library: CIL module
 0002:0014eb00       __real@404ca5dc1a47a9e3    005e6b00      CIL library: CIL module
 0002:0014eb08       __real@3f50624dd2f1a9fc    005e6b08      CIL library: CIL module
 0002:0014eb10       __real@40f0000000000000    005e6b10      CIL library: CIL module
 0002:0014eb18       __real@bff0000000000000    005e6b18      CIL library: CIL module
 0002:0014eb20       __real@3fc0000000000000    005e6b20      CIL library: CIL module
 0002:0014eb28       __real@3fd0000000000000    005e6b28      CIL library: CIL module
 0002:0014eb30       __real@401921fb54442d18    005e6b30      CIL library: CIL module
 0002:0014eb38       __real@3ff6a09e667f3bcd    005e6b38      CIL library: CIL module
 0002:0014eb40       __real@4006a09e667f3bcd    005e6b40      CIL library: CIL module
 0002:0014eb48       __real@4024000000000000    005e6b48      CIL library: CIL module
 0002:0014eb50       __real@4050000000000000    005e6b50      CIL library: CIL module
 0002:0014eb58       __real@3f70000000000000    005e6b58      CIL library: CIL module
 0002:0014eb60       __real@4070000000000000    005e6b60      CIL library: CIL module
 0002:0014eb68       __real@4014000000000000    005e6b68      CIL library: CIL module
 0002:0014eb70       __real@3dcccccd            005e6b70      CIL library: CIL module
 0002:0014eb78       __real@3fb999999999999a    005e6b78      CIL library: CIL module
 0002:0014eb80       __real@3fa0000000000000    005e6b80      CIL library: CIL module
 0002:0014eb88       __real@447a0000            005e6b88      CIL library: CIL module
 0002:0014eb8c       __real@c47a0000            005e6b8c      CIL library: CIL module
 0002:0014eb90       __real@c08f400000000000    005e6b90      CIL library: CIL module
 0002:0014eb98       __real@4f800000            005e6b98      CIL library: CIL module
 0002:0014eba0       __real@41f0000000000000    005e6ba0      CIL library: CIL module
 0002:0014eba8       __real@4038000000000000    005e6ba8      CIL library: CIL module
 0002:0014ebb0       __real@c6fa0000            005e6bb0      CIL library: CIL module
 0002:0014ebb8       __real@40df400000000000    005e6bb8      CIL library: CIL module
 0002:0014ebc0       __real@34000000            005e6bc0      CIL library: CIL module
 0002:001560e0       __load_config_used         005ee0e0     LIBCMT:loadcfg.obj
 0002:00156180       ___safe_se_handler_table   005ee180     <linker-defined>
 0002:0015618c       ___rtc_iaa                 005ee18c     LIBCMT:initsect.obj
 0002:00156190       ___rtc_izz                 005ee190     LIBCMT:initsect.obj
 0002:00156194       ___rtc_taa                 005ee194     LIBCMT:initsect.obj
 0002:00156198       ___rtc_tzz                 005ee198     LIBCMT:initsect.obj
 0002:00156774       __IMPORT_DESCRIPTOR_KERNEL32 005ee774     kernel32:KERNEL32.dll
 0002:00156788       __NULL_IMPORT_DESCRIPTOR   005ee788     kernel32:KERNEL32.dll
 0003:00000170       __iob                      005ef170     LIBCMT:_file.obj
 0003:000003f0       __aexit_rtn                005ef3f0     LIBCMT:crt0dat.obj
 0003:00000400       __timezone                 005ef400     LIBCMT:timeset.obj
 0003:00000404       __daylight                 005ef404     LIBCMT:timeset.obj
 0003:00000408       __dstbias                  005ef408     LIBCMT:timeset.obj
 0003:00000490       __tzname                   005ef490     LIBCMT:timeset.obj
 0003:000004b0       ___app_type                005ef4b0     LIBCMT:crt0.obj
 0003:000004b4       ___security_cookie         005ef4b4     LIBCMT:gs_cookie.obj
 0003:000004b8       ___security_cookie_complement 005ef4b8     LIBCMT:gs_cookie.obj
 0003:000004bc       __amblksiz                 005ef4bc     LIBCMT:heapinit.obj
 0003:00000698       ___badioinfo               005ef698     LIBCMT:ioinit.obj
 0003:000006d0       ___nullstring              005ef6d0     LIBCMT:output.obj
 0003:000006d4       ___wnullstring             005ef6d4     LIBCMT:output.obj
 0003:000006d8       __sys_errlist              005ef6d8     LIBCMT:syserr.obj
 0003:00000788       __sys_nerr                 005ef788     LIBCMT:syserr.obj
 0003:0000078c       ___flsindex                005ef78c     LIBCMT:tidtable.obj
 0003:00000790       ___getvalueindex           005ef790     LIBCMT:tidtable.obj
 0003:00000798       __lookuptrailbytes         005ef798     LIBCMT:read.obj
 0003:000008a0       __NLG_Destination          005ef8a0     LIBCMT:exsup.obj
 0003:000008b0       __cfltcvt_tab              005ef8b0     LIBCMT:cmiscdat.obj
 0003:000008d8       __XcptActTab               005ef8d8     LIBCMT:winxfltr.obj
 0003:00000950       __First_FPE_Indx           005ef950     LIBCMT:winxfltr.obj
 0003:00000954       __Num_FPE                  005ef954     LIBCMT:winxfltr.obj
 0003:00000958       __XcptActTabSize           005ef958     LIBCMT:winxfltr.obj
 0003:0000095c       __XcptActTabCount          005ef95c     LIBCMT:winxfltr.obj
 0003:00000960       __fltused                  005ef960     LIBCMT:fpinit.obj
 0003:00000964       __ldused                   005ef964     LIBCMT:fpinit.obj
 0003:00000968       __d_inf                    005ef968     LIBCMT:util.obj
 0003:00000970       __d_ind                    005ef970     LIBCMT:util.obj
 0003:00000978       __d_max                    005ef978     LIBCMT:util.obj
 0003:00000980       __d_min                    005ef980     LIBCMT:util.obj
 0003:00000988       __d_mzero                  005ef988     LIBCMT:util.obj
 0003:00000aa0       __lpdays                   005efaa0     LIBCMT:days.obj
 0003:00000ad4       __days                     005efad4     LIBCMT:days.obj
 0003:00000b08       ___initialmbcinfo          005efb08     LIBCMT:mbctype.obj
 0003:00000d28       __mbctype                  005efd28     LIBCMT:mbctype.obj
 0003:00000e30       __mbcasemap                005efe30     LIBCMT:mbctype.obj
 0003:00000f30       ___ptmbcinfo               005eff30     LIBCMT:mbctype.obj
 0003:0000102c       ___globallocalestatus      005f002c     LIBCMT:glstatus.obj
 0003:00001030       ___clocalestr              005f0030     LIBCMT:nlsdata2.obj
 0003:00001038       ___initiallocinfo          005f0038     LIBCMT:nlsdata2.obj
 0003:00001110       ___ptlocinfo               005f0110     LIBCMT:nlsdata2.obj
 0003:00001114       ___lc_clike                005f0114     LIBCMT:nlsdata2.obj
 0003:00001118       ___initiallocalestructinfo 005f0118     LIBCMT:nlsdata2.obj
 0003:00001130       ___abort_behavior          005f0130     LIBCMT:abort.obj
 0003:00001134       __matherr_flag             005f0134     LIBCMT:matherr.obj
 0003:00001138       __pctype                   005f0138     LIBCMT:ctype.obj
 0003:0000113c       __pwctype                  005f013c     LIBCMT:ctype.obj
 0003:00001140       ___lc_time_c               005f0140     LIBCMT:strftime.obj
 0003:000011f8       ___lc_time_curr            005f01f8     LIBCMT:strftime.obj
 0003:000011fc       ___lconv_static_decimal    005f01fc     LIBCMT:lconv.obj
 0003:00001200       ___lconv_c                 005f0200     LIBCMT:lconv.obj
 0003:00001230       ___lconv                   005f0230     LIBCMT:lconv.obj
 0003:00001234       ___mb_cur_max              005f0234     LIBCMT:nlsdata1.obj
 0003:00001238       ___decimal_point           005f0238     LIBCMT:nlsdata1.obj
 0003:0000123c       ___decimal_point_length    005f023c     LIBCMT:nlsdata1.obj
 0003:00001270       __pow10pos                 005f0270     LIBCMT:constpow.obj
 0003:000013d0       __pow10neg                 005f03d0     LIBCMT:constpow.obj
 0003:00001530       __coninpfh                 005f0530     LIBCMT:initcon.obj
 0003:00001534       __confh                    005f0534     LIBCMT:initcon.obj
 0003:00001550       __indefinite               005f0550     LIBCMT:87disp.obj
 0003:0000155a       __piby2                    005f055a     LIBCMT:87disp.obj
 0003:00001580       _pagetobench               005f0580     pdfbench.obj
 0003:00002e68       _j2k_prog_order_list       005f1e68     j2k.obj
 0003:00003190       _j2k_dec_mstab             005f2190     j2k.obj
 0003:000034c8       _pdf_cmap_Adobe_Korea1_2   005f24c8     cmap_korean.obj
 0003:00003620       _pdf_cmap_Adobe_Korea1_UCS2 005f2620     cmap_korean.obj
 0003:00003778       _pdf_cmap_KSC_EUC_H        005f2778     cmap_korean.obj
 0003:000038d0       _pdf_cmap_KSC_EUC_V        005f28d0     cmap_korean.obj
 0003:00003a28       _pdf_cmap_KSCms_UHC_H      005f2a28     cmap_korean.obj
 0003:00003b80       _pdf_cmap_KSCms_UHC_HW_H   005f2b80     cmap_korean.obj
 0003:00003cd8       _pdf_cmap_KSCms_UHC_HW_V   005f2cd8     cmap_korean.obj
 0003:00003e30       _pdf_cmap_KSCms_UHC_UCS2   005f2e30     cmap_korean.obj
 0003:00003f88       _pdf_cmap_KSCms_UHC_V      005f2f88     cmap_korean.obj
 0003:000040e0       _pdf_cmap_KSCpc_EUC_H      005f30e0     cmap_korean.obj
 0003:00004238       _pdf_cmap_KSCpc_EUC_UCS2   005f3238     cmap_korean.obj
 0003:00004390       _pdf_cmap_KSCpc_EUC_UCS2C  005f3390     cmap_korean.obj
 0003:000044e8       _pdf_cmap_UniKS_UCS2_H     005f34e8     cmap_korean.obj
 0003:00004640       _pdf_cmap_UniKS_UCS2_V     005f3640     cmap_korean.obj
 0003:00004798       _pdf_cmap_83pv_RKSJ_H      005f3798     cmap_japanese.obj
 0003:000048f0       _pdf_cmap_90ms_RKSJ_H      005f38f0     cmap_japanese.obj
 0003:00004a48       _pdf_cmap_90ms_RKSJ_UCS2   005f3a48     cmap_japanese.obj
 0003:00004ba0       _pdf_cmap_90ms_RKSJ_V      005f3ba0     cmap_japanese.obj
 0003:00004cf8       _pdf_cmap_90msp_RKSJ_H     005f3cf8     cmap_japanese.obj
 0003:00004e50       _pdf_cmap_90msp_RKSJ_V     005f3e50     cmap_japanese.obj
 0003:00004fa8       _pdf_cmap_90pv_RKSJ_H      005f3fa8     cmap_japanese.obj
 0003:00005100       _pdf_cmap_90pv_RKSJ_UCS2   005f4100     cmap_japanese.obj
 0003:00005258       _pdf_cmap_90pv_RKSJ_UCS2C  005f4258     cmap_japanese.obj
 0003:000053b0       _pdf_cmap_Add_RKSJ_H       005f43b0     cmap_japanese.obj
 0003:00005508       _pdf_cmap_Add_RKSJ_V       005f4508     cmap_japanese.obj
 0003:00005660       _pdf_cmap_Adobe_Japan1_4   005f4660     cmap_japanese.obj
 0003:000057b8       _pdf_cmap_Adobe_Japan1_UCS2 005f47b8     cmap_japanese.obj
 0003:00005910       _pdf_cmap_EUC_H            005f4910     cmap_japanese.obj
 0003:00005a68       _pdf_cmap_EUC_V            005f4a68     cmap_japanese.obj
 0003:00005bc0       _pdf_cmap_Ext_RKSJ_H       005f4bc0     cmap_japanese.obj
 0003:00005d18       _pdf_cmap_Ext_RKSJ_V       005f4d18     cmap_japanese.obj
 0003:00005e70       _pdf_cmap_H                005f4e70     cmap_japanese.obj
 0003:00005fc8       _pdf_cmap_UniJIS_UCS2_H    005f4fc8     cmap_japanese.obj
 0003:00006120       _pdf_cmap_UniJIS_UCS2_HW_H 005f5120     cmap_japanese.obj
 0003:00006278       _pdf_cmap_UniJIS_UCS2_HW_V 005f5278     cmap_japanese.obj
 0003:000063d0       _pdf_cmap_UniJIS_UCS2_V    005f53d0     cmap_japanese.obj
 0003:00006528       _pdf_cmap_V                005f5528     cmap_japanese.obj
 0003:00006680       _pdf_cmap_Adobe_CNS1_3     005f5680     cmap_chinese_t.obj
 0003:000067d8       _pdf_cmap_Adobe_CNS1_UCS2  005f57d8     cmap_chinese_t.obj
 0003:00006930       _pdf_cmap_B5pc_H           005f5930     cmap_chinese_t.obj
 0003:00006a88       _pdf_cmap_B5pc_UCS2        005f5a88     cmap_chinese_t.obj
 0003:00006be0       _pdf_cmap_B5pc_UCS2C       005f5be0     cmap_chinese_t.obj
 0003:00006d38       _pdf_cmap_B5pc_V           005f5d38     cmap_chinese_t.obj
 0003:00006e90       _pdf_cmap_CNS_EUC_H        005f5e90     cmap_chinese_t.obj
 0003:00006fe8       _pdf_cmap_CNS_EUC_V        005f5fe8     cmap_chinese_t.obj
 0003:00007140       _pdf_cmap_ETen_B5_H        005f6140     cmap_chinese_t.obj
 0003:00007298       _pdf_cmap_ETen_B5_UCS2     005f6298     cmap_chinese_t.obj
 0003:000073f0       _pdf_cmap_ETen_B5_V        005f63f0     cmap_chinese_t.obj
 0003:00007548       _pdf_cmap_ETenms_B5_H      005f6548     cmap_chinese_t.obj
 0003:000076a0       _pdf_cmap_ETenms_B5_V      005f66a0     cmap_chinese_t.obj
 0003:000077f8       _pdf_cmap_HKscs_B5_H       005f67f8     cmap_chinese_t.obj
 0003:00007950       _pdf_cmap_HKscs_B5_V       005f6950     cmap_chinese_t.obj
 0003:00007aa8       _pdf_cmap_UniCNS_UCS2_H    005f6aa8     cmap_chinese_t.obj
 0003:00007c00       _pdf_cmap_UniCNS_UCS2_V    005f6c00     cmap_chinese_t.obj
 0003:00007d58       _pdf_cmap_Adobe_GB1_4      005f6d58     cmap_chinese_s.obj
 0003:00007eb0       _pdf_cmap_Adobe_GB1_UCS2   005f6eb0     cmap_chinese_s.obj
 0003:00008008       _pdf_cmap_GB_EUC_H         005f7008     cmap_chinese_s.obj
 0003:00008160       _pdf_cmap_GB_EUC_V         005f7160     cmap_chinese_s.obj
 0003:000082b8       _pdf_cmap_GBK_EUC_H        005f72b8     cmap_chinese_s.obj
 0003:00008410       _pdf_cmap_GBK_EUC_UCS2     005f7410     cmap_chinese_s.obj
 0003:00008568       _pdf_cmap_GBK_EUC_V        005f7568     cmap_chinese_s.obj
 0003:000086c0       _pdf_cmap_GBK2K_H          005f76c0     cmap_chinese_s.obj
 0003:00008818       _pdf_cmap_GBK2K_V          005f7818     cmap_chinese_s.obj
 0003:00008970       _pdf_cmap_GBKp_EUC_H       005f7970     cmap_chinese_s.obj
 0003:00008ac8       _pdf_cmap_GBKp_EUC_V       005f7ac8     cmap_chinese_s.obj
 0003:00008c20       _pdf_cmap_GBT_EUC_H        005f7c20     cmap_chinese_s.obj
 0003:00008d78       _pdf_cmap_GBT_EUC_V        005f7d78     cmap_chinese_s.obj
 0003:00008ed0       _pdf_cmap_GBpc_EUC_H       005f7ed0     cmap_chinese_s.obj
 0003:00009028       _pdf_cmap_GBpc_EUC_UCS2    005f8028     cmap_chinese_s.obj
 0003:00009180       _pdf_cmap_GBpc_EUC_UCS2C   005f8180     cmap_chinese_s.obj
 0003:000092d8       _pdf_cmap_GBpc_EUC_V       005f82d8     cmap_chinese_s.obj
 0003:00009430       _pdf_cmap_UniGB_UCS2_H     005f8430     cmap_chinese_s.obj
 0003:00009588       _pdf_cmap_UniGB_UCS2_V     005f8588     cmap_chinese_s.obj
 0003:000096e0       _pdf_cmaptable             005f86e0     pdf_cmap_table.obj
 0003:0002b7e4       _pdf_devicegray            0061a7e4     pdf_colorspace1.obj
 0003:0002b7e8       _pdf_devicergb             0061a7e8     pdf_colorspace1.obj
 0003:0002b7ec       _pdf_devicecmyk            0061a7ec     pdf_colorspace1.obj
 0003:0002b7f0       _pdf_devicelab             0061a7f0     pdf_colorspace1.obj
 0003:0002b7f4       _pdf_devicepattern         0061a7f4     pdf_colorspace1.obj
 0003:00031a9c       _fz_infiniterect           00620a9c     base_rect.obj
 0003:00032170       _fz_img_1c1                00621170     imagedraw.obj
 0003:00032174       _fz_img_4c4                00621174     imagedraw.obj
 0003:00032178       _fz_img_1o1                00621178     imagedraw.obj
 0003:0003217c       _fz_img_4o4                0062117c     imagedraw.obj
 0003:00032180       _fz_img_w4i1o4             00621180     imagedraw.obj
 0003:00032184       _fz_duff_non               00621184     porterduff.obj
 0003:00032188       _fz_duff_nimcn             00621188     porterduff.obj
 0003:0003218c       _fz_duff_nimon             0062118c     porterduff.obj
 0003:00032190       _fz_duff_1o1               00621190     porterduff.obj
 0003:00032194       _fz_duff_4o4               00621194     porterduff.obj
 0003:00032198       _fz_duff_1i1c1             00621198     porterduff.obj
 0003:0003219c       _fz_duff_4i1c4             0062119c     porterduff.obj
 0003:000321a0       _fz_duff_1i1o1             006211a0     porterduff.obj
 0003:000321a4       _fz_duff_4i1o4             006211a4     porterduff.obj
 0003:000321a8       _fz_path_1c1               006211a8     porterduff.obj
 0003:000321ac       _fz_path_1o1               006211ac     porterduff.obj
 0003:000321b0       _fz_path_w4i1o4            006211b0     porterduff.obj
 0003:000321b4       _fz_text_1o1               006211b4     porterduff.obj
 0003:000321b8       _fz_text_w4i1o4            006211b8     porterduff.obj
 0003:00032330       _fz_decodetile             00621330     imageunpack.obj
 0003:00032334       _fz_loadtile1              00621334     imageunpack.obj
 0003:00032338       _fz_loadtile2              00621338     imageunpack.obj
 0003:0003233c       _fz_loadtile4              0062133c     imageunpack.obj
 0003:00032340       _fz_loadtile8              00621340     imageunpack.obj
 0003:000325d4       _fz_srown                  006215d4     imagescale.obj
 0003:000325d8       _fz_srow1                  006215d8     imagescale.obj
 0003:000325dc       _fz_srow2                  006215dc     imagescale.obj
 0003:000325e0       _fz_srow4                  006215e0     imagescale.obj
 0003:000325e4       _fz_srow5                  006215e4     imagescale.obj
 0003:000325e8       _fz_scoln                  006215e8     imagescale.obj
 0003:000325ec       _fz_scol1                  006215ec     imagescale.obj
 0003:000325f0       _fz_scol2                  006215f0     imagescale.obj
 0003:000325f4       _fz_scol4                  006215f4     imagescale.obj
 0003:000325f8       _fz_scol5                  006215f8     imagescale.obj
 0003:00037670       __half                     00626670     LIBCMT:pow.obj
 0003:000376d0       __infinity                 006266d0     LIBCMT:87tran.obj
 0003:000376da       __minfinity                006266da     LIBCMT:87tran.obj
 0003:000376e4       __logemax                  006266e4     LIBCMT:87tran.obj
 0003:0003770a       __OP_EXPjmptab             0062670a     LIBCMT:87tran.obj
 0003:00037730       __OP_ATAN2jmptab           00626730     LIBCMT:87triga.obj
 0003:000378e0       __cflush                   006268e0     LIBCMT:_file.obj
 0003:000378e4       __umaskval                 006268e4     LIBCMT:crt0dat.obj
 0003:000378e8       __osplatform               006268e8     LIBCMT:crt0dat.obj
 0003:000378ec       __osver                    006268ec     LIBCMT:crt0dat.obj
 0003:000378f0       __winver                   006268f0     LIBCMT:crt0dat.obj
 0003:000378f4       __winmajor                 006268f4     LIBCMT:crt0dat.obj
 0003:000378f8       __winminor                 006268f8     LIBCMT:crt0dat.obj
 0003:000378fc       ___argc                    006268fc     LIBCMT:crt0dat.obj
 0003:00037900       ___argv                    00626900     LIBCMT:crt0dat.obj
 0003:00037904       ___wargv                   00626904     LIBCMT:crt0dat.obj
 0003:00037908       __environ                  00626908     LIBCMT:crt0dat.obj
 0003:0003790c       ___initenv                 0062690c     LIBCMT:crt0dat.obj
 0003:00037910       __wenviron                 00626910     LIBCMT:crt0dat.obj
 0003:00037914       ___winitenv                00626914     LIBCMT:crt0dat.obj
 0003:00037918       __pgmptr                   00626918     LIBCMT:crt0dat.obj
 0003:0003791c       __wpgmptr                  0062691c     LIBCMT:crt0dat.obj
 0003:00037920       __exitflag                 00626920     LIBCMT:crt0dat.obj
 0003:00037924       __C_Termination_Done       00626924     LIBCMT:crt0dat.obj
 0003:00037928       __C_Exit_Done              00626928     LIBCMT:crt0dat.obj
 0003:000379e8       __aenvptr                  006269e8     LIBCMT:crt0.obj
 0003:000379ec       __wenvptr                  006269ec     LIBCMT:crt0.obj
 0003:000379f0       ___error_mode              006269f0     LIBCMT:crt0.obj
 0003:00037d1c       __crtheap                  00626d1c     LIBCMT:heapinit.obj
 0003:00037e70       ___sbh_pHeaderDefer        00626e70     LIBCMT:sbheap.obj
 0003:0003818c       ?_pnhHeap@@3P6AHI@ZA       0062718c     LIBCMT:handler.obj
 0003:00038190       __newmode                  00627190     LIBCMT:_newmode.obj
 0003:00038194       ___pInvalidArgHandler      00627194     LIBCMT:invarg.obj
 0003:00038198       __maxwait                  00627198     LIBCMT:crtheap.obj
 0003:0003819c       _gpFlsAlloc                0062719c     LIBCMT:tidtable.obj
 0003:000381a0       _gpFlsGetValue             006271a0     LIBCMT:tidtable.obj
 0003:000381a4       _gpFlsSetValue             006271a4     LIBCMT:tidtable.obj
 0003:000381a8       _gpFlsFree                 006271a8     LIBCMT:tidtable.obj
 0003:000381ac       __stdbuf                   006271ac     LIBCMT:_sftbuf.obj
 0003:000381b4       __commode                  006271b4     LIBCMT:ncommode.obj
 0003:000381b8       ?__pInconsistency@@3P6AXXZA 006271b8     LIBCMT:hooks.obj
 0003:000381dc       ___pPurecall               006271dc     LIBCMT:inithelp.obj
 0003:000381e4       ___fastflag                006271e4     LIBCMT:fpinit.obj
 0003:000381e8       __adjust_fdiv              006271e8     LIBCMT:fpinit.obj
 0003:000381f4       ___mbulinfo                006271f4     LIBCMT:mbctype.obj
 0003:00038200       ___mbcodepage              00627200     LIBCMT:mbctype.obj
 0003:00038204       ___ismbcodepage            00627204     LIBCMT:mbctype.obj
 0003:00038208       ___mblcid                  00627208     LIBCMT:mbctype.obj
 0003:0003820c       ___locale_changed          0062720c     LIBCMT:setlocal.obj
 0003:00038210       ___lc_handle               00627210     LIBCMT:nlsdata2.obj
 0003:00038228       ___lc_codepage             00627228     LIBCMT:nlsdata2.obj
 0003:0003822c       ___lc_collate_cp           0062722c     LIBCMT:nlsdata2.obj
 0003:00038360       ___lconv_static_null       00627360     LIBCMT:lconv.obj
 0003:00038364       __fmode                    00627364     LIBCMT:txtmode.obj
 0003:00038368       __outputformat             00627368     LIBCMT:outputformat.obj
 0003:00039b98       _fz_emptyrect              00628b98     base_rect.obj
 0003:00039bdc       _loadonly                  00628bdc     pdfbench.obj
 0003:00039be0       _xref                      00628be0     pdfbench.obj
 0003:00039be4       _pagecount                 00628be4     pdfbench.obj
 0003:00039be8       _drawgc                    00628be8     pdfbench.obj
 0003:00039bec       _drawpage                  00628bec     pdfbench.obj
 0003:00039bf0       __debugger_hook_dummy      00628bf0     <common>
 0003:00039bf4       __pmatherr                 00628bf4     <common>
 0003:00039bf8       ___use_sse2_mathfcns       00628bf8     <common>
 0003:00039bfc       ___sse2_available          00628bfc     <common>
 0003:00039c00       __nhandle                  00628c00     <common>
 0003:00039c20       ___pioinfo                 00628c20     <common>
 0003:00039d20       __pDestructExceptionObject 00628d20     <common>
 0003:00039d24       ___sbh_cntHeaderList       00628d24     <common>
 0003:00039d28       ___sbh_pHeaderList         00628d28     <common>
 0003:00039d2c       ___sbh_threshold           00628d2c     <common>
 0003:00039d30       ___sbh_pHeaderScan         00628d30     <common>
 0003:00039d34       ___sbh_sizeHeaderList      00628d34     <common>
 0003:00039d38       ___sbh_indGroupDefer       00628d38     <common>
 0003:00039d3c       ___active_heap             00628d3c     <common>
 0003:00039d40       __acmdln                   00628d40     <common>
 0003:00039d44       ___env_initialized         00628d44     <common>
 0003:00039d48       ___onexitend               00628d48     <common>
 0003:00039d4c       ___onexitbegin             00628d4c     <common>
 0003:00039d50       ___mbctype_initialized     00628d50     <common>
 0003:00039d54       ___dyn_tls_init_callback   00628d54     <common>
 0003:00039d58       ___piob                    00628d58     <common>
 0003:00039d60       __bufin                    00628d60     <common>
 0003:0003ad60       __nstream                  00629d60     <common>
 0003:0003ad80       _defaultSubstitute         00629d80     <common>

 entry point at        0001:00083f3c

 Static symbols

 0001:00000230       _crc32_little              00401230 f    CIL library: CIL module
 0001:00000575       _updatewindow              00401575 f    CIL library: CIL module
 0001:0000188d       _jbig2_default_free        0040288d f    CIL library: CIL module
 0001:0000188d       _zfree                     0040288d f    CIL library: CIL module
 0001:0000188d       _ft_free                   0040288d f    CIL library: CIL module
 0001:0000203e       _flush_pending             0040303e f    CIL library: CIL module
 0001:0000208b       _longest_match             0040308b f    CIL library: CIL module
 0001:000021d0       _longest_match_fast        004031d0 f    CIL library: CIL module
 0001:0000225a       _fill_window               0040325a f    CIL library: CIL module
 0001:000023a8       _deflate_stored            004033a8 f    CIL library: CIL module
 0001:000024d2       _deflate_fast              004034d2 f    CIL library: CIL module
 0001:000027bc       _deflate_slow              004037bc f    CIL library: CIL module
 0001:00002b77       _init_block                00403b77 f    CIL library: CIL module
 0001:00002bd5       _pqdownheap                00403bd5 f    CIL library: CIL module
 0001:00002c85       _gen_bitlen                00403c85 f    CIL library: CIL module
 0001:00002e42       _gen_codes                 00403e42 f    CIL library: CIL module
 0001:00002ec4       _build_tree                00403ec4 f    CIL library: CIL module
 0001:000030aa       _scan_tree                 004040aa f    CIL library: CIL module
 0001:00003166       _send_tree                 00404166 f    CIL library: CIL module
 0001:00003600       _build_bl_tree             00404600 f    CIL library: CIL module
 0001:00003661       _send_all_trees            00404661 f    CIL library: CIL module
 0001:00003b66       _compress_block            00404b66 f    CIL library: CIL module
 0001:00003f18       _set_data_type             00404f18 f    CIL library: CIL module
 0001:00003f5a       _bi_windup                 00404f5a f    CIL library: CIL module
 0001:00003fb1       _ft_realloc                00404fb1 f    CIL library: CIL module
 0001:00003fc1       _ft_ansi_stream_close      00404fc1 f    CIL library: CIL module
 0001:00003fdb       _ft_ansi_stream_io         00404fdb f    CIL library: CIL module
 0001:00004066       _ft_bitmap_glyph_init      00405066 f    CIL library: CIL module
 0001:000040da       _ft_bitmap_glyph_copy      004050da f    CIL library: CIL module
 0001:00004102       _ft_bitmap_glyph_done      00405102 f    CIL library: CIL module
 0001:00004110       _ft_bitmap_glyph_bbox      00405110 f    CIL library: CIL module
 0001:00004142       _ft_outline_glyph_init     00405142 f    CIL library: CIL module
 0001:00004186       _ft_outline_glyph_done     00405186 f    CIL library: CIL module
 0001:0000419b       _ft_outline_glyph_copy     0040519b f    CIL library: CIL module
 0001:000041d1       _ft_outline_glyph_transform 004051d1 f    CIL library: CIL module
 0001:00004200       _ft_outline_glyph_bbox     00405200 f    CIL library: CIL module
 0001:00004213       _ft_outline_glyph_prepare  00405213 f    CIL library: CIL module
 0001:00004238       _ft_new_glyph              00405238 f    CIL library: CIL module
 0001:000044b8       _af_sort_pos               004054b8 f    CIL library: CIL module
 0001:000044f3       _af_sort_widths            004054f3 f    CIL library: CIL module
 0001:0000454a       _af_face_globals_compute_script_coverage 0040554a f    CIL library: CIL module
 0001:00004644       _af_face_globals_new       00405644 f    CIL library: CIL module
 0001:00004695       _af_face_globals_free      00405695 f    CIL library: CIL module
 0001:000046f8       _af_face_globals_get_metrics 004056f8 f    CIL library: CIL module
 0001:00004797       _af_axis_hints_new_segment 00405797 f    CIL library: CIL module
 0001:00004811       _af_axis_hints_new_edge    00405811 f    CIL library: CIL module
 0001:000048e3       _af_direction_compute      004058e3 f    CIL library: CIL module
 0001:00004925       _af_glyph_hints_done       00405925 f    CIL library: CIL module
 0001:000049a5       _af_glyph_hints_reload     004059a5 f    CIL library: CIL module
 0001:00004cbf       _af_glyph_hints_save       00405cbf f    CIL library: CIL module
 0001:00004d04       _af_glyph_hints_align_edge_points 00405d04 f    CIL library: CIL module
 0001:00004d98       _af_glyph_hints_align_strong_points 00405d98 f    CIL library: CIL module
 0001:00004f20       _af_iup_interp             00405f20 f    CIL library: CIL module
 0001:00005029       _af_glyph_hints_align_weak_points 00406029 f    CIL library: CIL module
 0001:00005213       _af_dummy_hints_init       00406213 f    CIL library: CIL module
 0001:00005227       _af_latin_metrics_init_widths 00406227 f    CIL library: CIL module
 0001:00005401       _af_latin_metrics_init_blues 00406401 f    CIL library: CIL module
 0001:000056b2       _af_latin_metrics_init     004066b2 f    CIL library: CIL module
 0001:00005712       _af_latin_metrics_scale_dim 00406712 f    CIL library: CIL module
 0001:0000590c       _af_latin_metrics_scale    0040690c f    CIL library: CIL module
 0001:0000593b       _af_latin_hints_compute_segments 0040693b f    CIL library: CIL module
 0001:00005bc8       _af_latin_hints_link_segments 00406bc8 f    CIL library: CIL module
 0001:00005d21       _af_latin_hints_compute_edges 00406d21 f    CIL library: CIL module
 0001:00005fac       _af_latin_hints_detect_features 00406fac f    CIL library: CIL module
 0001:00005fd8       _af_latin_hints_compute_blue_edges 00406fd8 f    CIL library: CIL module
 0001:000060ed       _af_latin_snap_width       004070ed f    CIL library: CIL module
 0001:000060ed       _af_latin2_snap_width      004070ed f    CIL library: CIL module
 0001:000060ed       _af_cjk_snap_width         004070ed f    CIL library: CIL module
 0001:00006141       _af_latin_compute_stem_width 00407141 f    CIL library: CIL module
 0001:00006294       _af_latin_align_linked_edge 00407294 f    CIL library: CIL module
 0001:000062b7       _af_latin_hint_edges       004072b7 f    CIL library: CIL module
 0001:00006754       _af_latin_hints_apply      00407754 f    CIL library: CIL module
 0001:000067f4       _af_latin2_metrics_init_widths 004077f4 f    CIL library: CIL module
 0001:000069cd       _af_latin2_metrics_init_blues 004079cd f    CIL library: CIL module
 0001:00006c7b       _af_latin2_metrics_init    00407c7b f    CIL library: CIL module
 0001:00006cd8       _af_latin2_metrics_scale_dim 00407cd8 f    CIL library: CIL module
 0001:00006eee       _af_latin2_metrics_scale   00407eee f    CIL library: CIL module
 0001:00006f1b       _af_latin2_hints_compute_segments 00407f1b f    CIL library: CIL module
 0001:00007191       _af_latin2_hints_link_segments 00408191 f    CIL library: CIL module
 0001:000072e5       _af_latin2_hints_compute_edges 004082e5 f    CIL library: CIL module
 0001:000075ac       _af_latin2_hints_detect_features 004085ac f    CIL library: CIL module
 0001:000075d8       _af_latin2_hints_compute_blue_edges 004085d8 f    CIL library: CIL module
 0001:000076ab       _af_latin2_hints_init      004086ab f    CIL library: CIL module
 0001:000076ab       _af_latin_hints_init       004086ab f    CIL library: CIL module
 0001:0000772a       _af_latin2_compute_stem_width 0040872a f    CIL library: CIL module
 0001:0000785e       _af_latin2_hint_edges      0040885e f    CIL library: CIL module
 0001:00007d53       _af_latin2_hints_apply     00408d53 f    CIL library: CIL module
 0001:00007df2       _af_cjk_metrics_init       00408df2 f    CIL library: CIL module
 0001:00007e32       _af_cjk_metrics_scale      00408e32 f    CIL library: CIL module
 0001:00007e66       _af_cjk_hints_compute_segments 00408e66 f    CIL library: CIL module
 0001:00007ece       _af_cjk_hints_link_segments 00408ece f    CIL library: CIL module
 0001:00008178       _af_cjk_hints_compute_edges 00409178 f    CIL library: CIL module
 0001:0000845c       _af_cjk_hints_detect_features 0040945c f    CIL library: CIL module
 0001:00008489       _af_cjk_hints_init         00409489 f    CIL library: CIL module
 0001:000084f8       _af_cjk_compute_stem_width 004094f8 f    CIL library: CIL module
 0001:0000860e       _af_hint_normal_stem       0040960e f    CIL library: CIL module
 0001:00008792       _af_cjk_hint_edges         00409792 f    CIL library: CIL module
 0001:00008a2e       _af_cjk_align_edge_points  00409a2e f    CIL library: CIL module
 0001:00008ae8       _af_cjk_hints_apply        00409ae8 f    CIL library: CIL module
 0001:00008b7c       _af_indic_metrics_init     00409b7c f    CIL library: CIL module
 0001:00008b81       _af_indic_metrics_scale    00409b81 f    CIL library: CIL module
 0001:00008b86       _af_indic_hints_init       00409b86 f    CIL library: CIL module
 0001:00008b8b       _af_indic_hints_apply      00409b8b f    CIL library: CIL module
 0001:00008b90       _af_loader_load_g          00409b90 f    CIL library: CIL module
 0001:000092a9       _af_loader_load_glyph      0040a2a9 f    CIL library: CIL module
 0001:000093b1       _af_autofitter_init        0040a3b1 f    CIL library: CIL module
 0001:000093ec       _af_autofitter_done        0040a3ec f    CIL library: CIL module
 0001:00009410       _af_autofitter_load_glyph  0040a410 f    CIL library: CIL module
 0001:000098d1       _FT_GlyphLoader_Adjust_Points 0040a8d1 f    CIL library: CIL module
 0001:00009d95       _ft_glyphslot_init         0040ad95 f    CIL library: CIL module
 0001:00009e79       _ft_glyphslot_clear        0040ae79 f    CIL library: CIL module
 0001:00009edc       _ft_glyphslot_done         0040aedc f    CIL library: CIL module
 0001:0000a06f       _ft_glyphslot_grid_fit_metrics 0040b06f f    CIL library: CIL module
 0001:0000a3b9       _destroy_size              0040b3b9 f    CIL library: CIL module
 0001:0000a3f9       _destroy_charmaps          0040b3f9 f    CIL library: CIL module
 0001:0000a436       _destroy_face              0040b436 f    CIL library: CIL module
 0001:0000a4da       _find_unicode_charmap      0040b4da f    CIL library: CIL module
 0001:0000a54a       _open_face                 0040b54a f    CIL library: CIL module
 0001:0000aaee       _ft_recompute_scaled_metrics 0040baee f    CIL library: CIL module
 0001:0000af77       _ft_cmap_done_internal     0040bf77 f    CIL library: CIL module
 0001:0000b26b       _ft_add_renderer           0040c26b f    CIL library: CIL module
 0001:0000b30e       _ft_remove_renderer        0040c30e f    CIL library: CIL module
 0001:0000b479       _Destroy_Module            0040c479 f    CIL library: CIL module
 0001:0000c704       _ft_trig_downscale         0040d704 f    CIL library: CIL module
 0001:0000c75d       _ft_trig_prenorm           0040d75d f    CIL library: CIL module
 0001:0000c7d0       _ft_trig_pseudo_polarize   0040d7d0 f    CIL library: CIL module
 0001:0000cad4       _hash_bucket               0040dad4 f    CIL library: CIL module
 0001:0000cb49       _hash_rehash               0040db49 f    CIL library: CIL module
 0001:0000cbc4       _hash_init                 0040dbc4 f    CIL library: CIL module
 0001:0000cbfc       _hash_free                 0040dbfc f    CIL library: CIL module
 0001:0000cc37       _hash_insert               0040dc37 f    CIL library: CIL module
 0001:0000cc9d       __bdf_list_done            0040dc9d f    CIL library: CIL module
 0001:0000ccba       __bdf_list_ensure          0040dcba f    CIL library: CIL module
 0001:0000cd0c       __bdf_list_shift           0040dd0c f    CIL library: CIL module
 0001:0000cd38       __bdf_list_join            0040dd38 f    CIL library: CIL module
 0001:0000cd8c       __bdf_list_split           0040dd8c f    CIL library: CIL module
 0001:0000cf42       __bdf_readstream           0040df42 f    CIL library: CIL module
 0001:0000d153       __bdf_atoul                0040e153 f    CIL library: CIL module
 0001:0000d1b9       __bdf_atol                 0040e1b9 f    CIL library: CIL module
 0001:0000d244       __bdf_atos                 0040e244 f    CIL library: CIL module
 0001:0000d2dd       _by_encoding               0040e2dd f    CIL library: CIL module
 0001:0000d2fd       _bdf_create_property       0040e2fd f    CIL library: CIL module
 0001:0000d3e8       __bdf_add_comment          0040e3e8 f    CIL library: CIL module
 0001:0000d43c       __bdf_set_default_spacing  0040e43c f    CIL library: CIL module
 0001:0000d533       __bdf_is_atom              0040e533 f    CIL library: CIL module
 0001:0000d612       __bdf_add_property         0040e612 f    CIL library: CIL module
 0001:0000d8c1       __bdf_parse_glyphs         0040e8c1 f    CIL library: CIL module
 0001:0000e05d       __bdf_parse_properties     0040f05d f    CIL library: CIL module
 0001:0000e220       __bdf_parse_start          0040f220 f    CIL library: CIL module
 0001:0000e684       _bdf_load_font             0040f684 f    CIL library: CIL module
 0001:0000e8a5       _bdf_free_font             0040f8a5 f    CIL library: CIL module
 0001:0000ea7d       _bdf_get_font_property     0040fa7d f    CIL library: CIL module
 0001:0000eab0       _bdf_cmap_init             0040fab0 f    CIL library: CIL module
 0001:0000eace       _pcf_cmap_done             0040face f    CIL library: CIL module
 0001:0000eace       _bdf_cmap_done             0040face f    CIL library: CIL module
 0001:0000eace       _pfr_cmap_done             0040face f    CIL library: CIL module
 0001:0000eadb       _pcf_cmap_char_index       0040fadb f    CIL library: CIL module
 0001:0000eadb       _bdf_cmap_char_index       0040fadb f    CIL library: CIL module
 0001:0000eb17       _bdf_interpret_style       0040fb17 f    CIL library: CIL module
 0001:0000ecd9       _BDF_Face_Done             0040fcd9 f    CIL library: CIL module
 0001:0000ed6e       _BDF_Face_Init             0040fd6e f    CIL library: CIL module
 0001:0000f1e2       _BDF_Size_Select           004101e2 f    CIL library: CIL module
 0001:0000f21c       _BDF_Size_Request          0041021c f    CIL library: CIL module
 0001:0000f293       _BDF_Glyph_Load            00410293 f    CIL library: CIL module
 0001:0000f39a       _bdf_get_bdf_property      0041039a f    CIL library: CIL module
 0001:0000f3ee       _bdf_get_charset_id        004103ee f    CIL library: CIL module
 0001:0000f40d       _bdf_driver_requester      0041040d f    CIL library: CIL module
 0001:0000f41d       _FTC_MruNode_Prepend       0041041d f    CIL library: CIL module
 0001:0000f43a       _FTC_MruNode_Up            0041043a f    CIL library: CIL module
 0001:0000f45c       _FTC_MruNode_Remove        0041045c f    CIL library: CIL module
 0001:0000f47a       _FTC_MruList_Init          0041047a f    CIL library: CIL module
 0001:0000f4a1       _FTC_MruList_Reset         004104a1 f    CIL library: CIL module
 0001:0000f4b6       _FTC_MruList_New           004104b6 f    CIL library: CIL module
 0001:0000f580       _FTC_MruList_Remove        00410580 f    CIL library: CIL module
 0001:0000f5af       _FTC_MruList_RemoveSelection 004105af f    CIL library: CIL module
 0001:0000f601       _ftc_scaler_lookup_size    00410601 f    CIL library: CIL module
 0001:0000f67f       _ftc_size_node_done        0041067f f    CIL library: CIL module
 0001:0000f692       _ftc_size_node_compare     00410692 f    CIL library: CIL module
 0001:0000f6ee       _ftc_size_node_init        004106ee f    CIL library: CIL module
 0001:0000f715       _ftc_size_node_reset       00410715 f    CIL library: CIL module
 0001:0000f746       _ftc_size_node_compare_faceid 00410746 f    CIL library: CIL module
 0001:0000f7dc       _ftc_face_node_init        004107dc f    CIL library: CIL module
 0001:0000f81e       _ftc_face_node_done        0041081e f    CIL library: CIL module
 0001:0000f848       _ftc_face_node_compare     00410848 f    CIL library: CIL module
 0001:0000f8cd       _FTC_Manager_FlushN        004108cd f    CIL library: CIL module
 0001:0000f917       _ftc_cache_resize          00410917 f    CIL library: CIL module
 0001:0000fab2       _ftc_cache_init            00410ab2 f    CIL library: CIL module
 0001:0000fae9       _FTC_Cache_Clear           00410ae9 f    CIL library: CIL module
 0001:0000fb70       _ftc_cache_done            00410b70 f    CIL library: CIL module
 0001:0000fba2       _ftc_cmap_node_free        00410ba2 f    CIL library: CIL module
 0001:0000fbb4       _ftc_cmap_node_new         00410bb4 f    CIL library: CIL module
 0001:0000fc06       _ftc_cmap_node_weight      00410c06 f    CIL library: CIL module
 0001:0000fc0a       _ftc_cmap_node_compare     00410c0a f    CIL library: CIL module
 0001:0000fc34       _ftc_cmap_node_remove_faceid 00410c34 f    CIL library: CIL module
 0001:0000fc43       _FTC_GNode_UnselectFamily  00410c43 f    CIL library: CIL module
 0001:0000fc62       _ftc_gnode_compare         00410c62 f    CIL library: CIL module
 0001:0000fc7f       _ftc_gcache_init           00410c7f f    CIL library: CIL module
 0001:0000fcab       _ftc_gcache_done           00410cab f    CIL library: CIL module
 0001:0000fcc0       _ftc_inode_free            00410cc0 f    CIL library: CIL module
 0001:0000fcfe       _ftc_inode_new             00410cfe f    CIL library: CIL module
 0001:0000fd61       _ftc_inode_weight          00410d61 f    CIL library: CIL module
 0001:0000fda1       _ftc_sbit_copy_bitmap      00410da1 f    CIL library: CIL module
 0001:0000fddf       _ftc_snode_free            00410ddf f    CIL library: CIL module
 0001:0000fe2c       _ftc_snode_load            00410e2c f    CIL library: CIL module
 0001:0000ff6c       _FTC_SNode_New             00410f6c f    CIL library: CIL module
 0001:00010016       _ftc_snode_new             00411016 f    CIL library: CIL module
 0001:0001002b       _ftc_snode_weight          0041102b f    CIL library: CIL module
 0001:00010063       _ftc_snode_compare         00411063 f    CIL library: CIL module
 0001:0001011f       _ftc_basic_family_compare  0041111f f    CIL library: CIL module
 0001:0001017c       _ftc_basic_family_init     0041117c f    CIL library: CIL module
 0001:000101aa       _ftc_basic_family_get_count 004111aa f    CIL library: CIL module
 0001:000101d3       _ftc_basic_family_load_bitmap 004111d3 f    CIL library: CIL module
 0001:00010217       _ftc_basic_family_load_glyph 00411217 f    CIL library: CIL module
 0001:00010286       _ftc_basic_gnode_compare_faceid 00411286 f    CIL library: CIL module
 0001:000102a9       _Load_Glyph                004112a9 f    CIL library: CIL module
 0001:000102f1       _cff_get_advances          004112f1 f    CIL library: CIL module
 0001:00010345       _cff_get_glyph_name        00411345 f    CIL library: CIL module
 0001:000103ac       _cff_get_name_index        004113ac f    CIL library: CIL module
 0001:00010473       _cff_ps_has_glyph_names    00411473 f    CIL library: CIL module
 0001:00010485       _cff_ps_get_font_info      00411485 f    CIL library: CIL module
 0001:00010573       _cff_get_ps_name           00411573 f    CIL library: CIL module
 0001:00010584       _cff_get_cmap_info         00411584 f    CIL library: CIL module
 0001:000105e8       _cff_get_ros               004115e8 f    CIL library: CIL module
 0001:00010681       _cff_get_is_cid            00411681 f    CIL library: CIL module
 0001:000106a8       _cff_get_cid_from_glyph_index 004116a8 f    CIL library: CIL module
 0001:000106e8       _cff_get_interface         004116e8 f    CIL library: CIL module
 0001:00010721       _cff_parser_init           00411721 f   cffparse.obj
 0001:0001074f       _cff_parse_integer         0041174f f    CIL library: CIL module
 0001:0001074f       _cff_parse_integer         0041174f f    CIL library: CIL module
 0001:000107de       _cff_parse_real            004117de f    CIL library: CIL module
 0001:00010a1f       _cff_parse_num             00411a1f f    CIL library: CIL module
 0001:00010a43       _cff_parse_fixed           00411a43 f    CIL library: CIL module
 0001:00010a68       _cff_parse_fixed_scaled    00411a68 f    CIL library: CIL module
 0001:00010a94       _cff_parse_fixed_dynamic   00411a94 f    CIL library: CIL module
 0001:00010b1b       _cff_parse_font_matrix     00411b1b f    CIL library: CIL module
 0001:00010bd1       _cff_parse_font_bbox       00411bd1 f    CIL library: CIL module
 0001:00010c42       _cff_parse_private_dict    00411c42 f    CIL library: CIL module
 0001:00010c7b       _cff_parse_cid_ros         00411c7b f    CIL library: CIL module
 0001:00010cca       _cff_parser_run            00411cca f   cffparse.obj
 0001:00010ed5       _cff_index_read_offset     00411ed5 f    CIL library: CIL module
 0001:00010f19       _cff_index_init            00411f19 f    CIL library: CIL module
 0001:00011032       _cff_index_done            00412032 f    CIL library: CIL module
 0001:00011067       _cff_index_load_offsets    00412067 f    CIL library: CIL module
 0001:00011198       _cff_index_get_pointers    00412198 f    CIL library: CIL module
 0001:00011229       _cff_index_access_element  00412229 f    CIL library: CIL module
 0001:00011326       _cff_index_get_name        00412326 f    CIL library: CIL module
 0001:0001139a       _cff_index_get_sid_string  0041239a f    CIL library: CIL module
 0001:000113ed       _CFF_Load_FD_Select        004123ed f    CIL library: CIL module
 0001:0001145c       _cff_fd_select_get         0041245c f    CIL library: CIL module
 0001:000114e3       _cff_charset_compute_cids  004124e3 f    CIL library: CIL module
 0001:0001155a       _cff_charset_load          0041255a f    CIL library: CIL module
 0001:000117c5       _cff_encoding_load         004127c5 f    CIL library: CIL module
 0001:00011a83       _cff_subfont_load          00412a83 f    CIL library: CIL module
 0001:00011c87       _cff_subfont_done          00412c87 f    CIL library: CIL module
 0001:00011cb0       _cff_font_load             00412cb0 f    CIL library: CIL module
 0001:0001200e       _cff_font_done             0041300e f    CIL library: CIL module
 0001:000121f8       _cff_size_get_globals_funcs 004131f8 f    CIL library: CIL module
 0001:00012230       _cff_size_done             00413230 f    CIL library: CIL module
 0001:0001226f       _cff_make_private_dict     0041326f f    CIL library: CIL module
 0001:000123c1       _cff_size_init             004133c1 f    CIL library: CIL module
 0001:000124be       _cff_size_select           004134be f    CIL library: CIL module
 0001:00012582       _cff_size_request          00413582 f    CIL library: CIL module
 0001:0001267a       _cff_slot_init             0041367a f    CIL library: CIL module
 0001:000126bb       _cff_face_init             004136bb f    CIL library: CIL module
 0001:00012e70       _cff_face_done             00413e70 f    CIL library: CIL module
 0001:00012ead       _cff_compute_bias          00413ead f    CIL library: CIL module
 0001:00012ed0       _cff_decoder_init          00413ed0 f    CIL library: CIL module
 0001:00012f91       _cff_decoder_prepare       00413f91 f    CIL library: CIL module
 0001:0001303b       _check_points              0041403b f    CIL library: CIL module
 0001:0001306e       _cff_builder_add_point     0041406e f    CIL library: CIL module
 0001:000130b5       _cff_builder_add_point1    004140b5 f    CIL library: CIL module
 0001:000130df       _cff_builder_add_contour   004140df f    CIL library: CIL module
 0001:00013139       _cff_builder_start_point   00414139 f    CIL library: CIL module
 0001:00013157       _cff_builder_close_contour 00414157 f    CIL library: CIL module
 0001:000131cd       _cff_lookup_glyph_by_stdcharcode 004141cd f    CIL library: CIL module
 0001:0001320c       _cff_get_glyph_data        0041420c f    CIL library: CIL module
 0001:0001322e       _cff_free_glyph_data       0041422e f    CIL library: CIL module
 0001:00013247       _cff_operator_seac         00414247 f    CIL library: CIL module
 0001:000133d2       _cff_decoder_parse_charstrings 004143d2 f    CIL library: CIL module
 0001:00014886       _cff_slot_load             00415886 f    CIL library: CIL module
 0001:00014e12       _cff_cmap_encoding_init    00415e12 f    CIL library: CIL module
 0001:00014e2a       _cff_cmap_encoding_done    00415e2a f    CIL library: CIL module
 0001:00014e33       _cff_cmap_encoding_char_index 00415e33 f    CIL library: CIL module
 0001:00014e4d       _cff_cmap_encoding_char_next 00415e4d f    CIL library: CIL module
 0001:00014e8a       _cff_sid_to_glyph_name     00415e8a f    CIL library: CIL module
 0001:00014eb2       _cff_sid_free_glyph_name   00415eb2 f    CIL library: CIL module
 0001:00014ec4       _cff_cmap_unicode_init     00415ec4 f    CIL library: CIL module
 0001:00014f02       _t1_cmap_unicode_done      00415f02 f    CIL library: CIL module
 0001:00014f02       _cff_cmap_unicode_done     00415f02 f    CIL library: CIL module
 0001:00014f1f       _cff_cmap_unicode_char_index 00415f1f f    CIL library: CIL module
 0001:00014f3c       _cff_cmap_unicode_char_next 00415f3c f    CIL library: CIL module
 0001:00014f59       _cff_parse_real            00415f59 f    CIL library: CIL module
 0001:0001519a       _cff_parse_num             0041619a f    CIL library: CIL module
 0001:000151be       _cff_parse_fixed           004161be f    CIL library: CIL module
 0001:000151e3       _cff_parse_fixed_scaled    004161e3 f    CIL library: CIL module
 0001:0001520f       _cff_parse_fixed_dynamic   0041620f f    CIL library: CIL module
 0001:00015296       _cff_parse_font_matrix     00416296 f    CIL library: CIL module
 0001:0001534c       _cff_parse_font_bbox       0041634c f    CIL library: CIL module
 0001:000153bd       _cff_parse_private_dict    004163bd f    CIL library: CIL module
 0001:000153f6       _cff_parse_cid_ros         004163f6 f    CIL library: CIL module
 0001:00015445       _cid_parser_new            00416445 f    CIL library: CIL module
 0001:000156d3       _cid_get_offset            004166d3 f    CIL library: CIL module
 0001:000156f4       _cid_load_keyword          004166f4 f    CIL library: CIL module
 0001:00015785       _parse_font_matrix         00416785 f    CIL library: CIL module
 0001:00015871       _parse_fd_array            00416871 f    CIL library: CIL module
 0001:000158ee       _parse_expansion_factor    004168ee f    CIL library: CIL module
 0001:00015924       _cid_parse_dict            00416924 f    CIL library: CIL module
 0001:00015a4b       _cid_read_subrs            00416a4b f    CIL library: CIL module
 0001:00015d13       _cid_hex_to_binary         00416d13 f    CIL library: CIL module
 0001:00015e48       _cid_face_open             00416e48 f    CIL library: CIL module
 0001:00015f85       _T1_GlyphSlot_Done         00416f85 f    CIL library: CIL module
 0001:00015f85       _cid_slot_done             00416f85 f    CIL library: CIL module
 0001:00015f85       _cff_slot_done             00416f85 f    CIL library: CIL module
 0001:00015f94       _cid_slot_init             00416f94 f    CIL library: CIL module
 0001:00015fcf       _cid_size_get_globals_funcs 00416fcf f    CIL library: CIL module
 0001:00016001       _cid_size_done             00417001 f    CIL library: CIL module
 0001:00016024       _cid_size_init             00417024 f    CIL library: CIL module
 0001:00016069       _cid_size_request          00417069 f    CIL library: CIL module
 0001:0001609e       _cid_face_done             0041709e f    CIL library: CIL module
 0001:00016206       _cid_face_init             00417206 f    CIL library: CIL module
 0001:00016433       _cid_get_postscript_name   00417433 f    CIL library: CIL module
 0001:00016448       _cid_ps_get_font_info      00417448 f    CIL library: CIL module
 0001:00016462       _cid_ps_get_font_extra     00417462 f    CIL library: CIL module
 0001:00016477       _cid_get_ros               00417477 f    CIL library: CIL module
 0001:000164ae       _cid_get_is_cid            004174ae f    CIL library: CIL module
 0001:000164bc       _cid_get_cid_from_glyph_index 004174bc f    CIL library: CIL module
 0001:000164cd       _cid_get_interface         004174cd f    CIL library: CIL module
 0001:000164dd       _cid_load_glyph            004174dd f    CIL library: CIL module
 0001:0001669d       _cid_slot_load_glyph       0041769d f    CIL library: CIL module
 0001:0001697b       _gxv_feat_registry_validate 0041797b f    CIL library: CIL module
 0001:00016a00       _gxv_feat_name_index_validate 00417a00 f    CIL library: CIL module
 0001:00016a40       _gxv_feat_setting_validate 00417a40 f    CIL library: CIL module
 0001:00016a86       _gxv_feat_name_validate    00417a86 f    CIL library: CIL module
 0001:00016b9a       _gxv_feat_validate         00417b9a f    CIL library: CIL module
 0001:00016ca7       _gxv_compare_ushort_offset 00417ca7 f    CIL library: CIL module
 0001:00016cc3       _gxv_set_length_by_ushort_offset 00417cc3 f    CIL library: CIL module
 0001:00016d76       _gxv_compare_ulong_offset  00417d76 f    CIL library: CIL module
 0001:00016d8f       _gxv_set_length_by_ulong_offset 00417d8f f    CIL library: CIL module
 0001:00016e39       _gxv_array_getlimits_byte  00417e39 f    CIL library: CIL module
 0001:00016e9c       _gxv_array_getlimits_ushort 00417e9c f    CIL library: CIL module
 0001:00016f26       _gxv_BinSrchHeader_check_consistency 00417f26 f    CIL library: CIL module
 0001:00016fd4       _gxv_BinSrchHeader_validate 00417fd4 f    CIL library: CIL module
 0001:000170b3       _gxv_LookupTable_fmt0_validate 004180b3 f    CIL library: CIL module
 0001:0001715e       _gxv_LookupTable_fmt2_skip_endmarkers 0041815e f    CIL library: CIL module
 0001:00017199       _gxv_LookupTable_fmt2_validate 00418199 f    CIL library: CIL module
 0001:00017323       _gxv_LookupTable_fmt4_validate 00418323 f    CIL library: CIL module
 0001:000174c5       _gxv_LookupTable_fmt6_validate 004184c5 f    CIL library: CIL module
 0001:00017602       _gxv_LookupTable_fmt8_validate 00418602 f    CIL library: CIL module
 0001:000176cc       _gxv_LookupTable_validate  004186cc f    CIL library: CIL module
 0001:00017769       _gxv_glyphid_validate      00418769 f    CIL library: CIL module
 0001:000177a4       _gxv_ctlPoint_validate     004187a4 f    CIL library: CIL module
 0001:00017806       _gxv_sfntName_validate     00418806 f    CIL library: CIL module
 0001:0001788f       _gxv_ClassTable_validate   0041888f f    CIL library: CIL module
 0001:000179e0       _gxv_StateArray_validate   004189e0 f    CIL library: CIL module
 0001:00017a80       _gxv_EntryTable_validate   00418a80 f    CIL library: CIL module
 0001:00017c36       _gxv_StateTable_subtable_setup 00418c36 f    CIL library: CIL module
 0001:00017ca0       _gxv_StateTable_validate   00418ca0 f    CIL library: CIL module
 0001:00017df9       _gxv_XStateTable_subtable_setup 00418df9 f    CIL library: CIL module
 0001:00017e44       _gxv_XClassTable_lookupval_validate 00418e44 f    CIL library: CIL module
 0001:00017e74       _gxv_XStateArray_validate  00418e74 f    CIL library: CIL module
 0001:00017f31       _gxv_XEntryTable_validate  00418f31 f    CIL library: CIL module
 0001:000180cb       _gxv_XStateTable_validate  004190cb f    CIL library: CIL module
 0001:0001827e       _gxv_odtect_add_range      0041927e f    CIL library: CIL module
 0001:000182b2       _gxv_odtect_validate       004192b2 f    CIL library: CIL module
 0001:0001833c       _gxv_bsln_LookupValue_validate 0041933c f    CIL library: CIL module
 0001:0001837b       _gxv_bsln_parts_fmt0_validate 0041937b f    CIL library: CIL module
 0001:000183b0       _gxv_bsln_parts_fmt1_validate 004193b0 f    CIL library: CIL module
 0001:000183ed       _gxv_bsln_parts_fmt2_validate 004193ed f    CIL library: CIL module
 0001:0001847e       _gxv_bsln_parts_fmt3_validate 0041947e f    CIL library: CIL module
 0001:000184bb       _gxv_bsln_validate         004194bb f    CIL library: CIL module
 0001:0001856f       _gxv_trak_trackTable_validate 0041956f f    CIL library: CIL module
 0001:00018623       _gxv_trak_trackData_validate 00419623 f    CIL library: CIL module
 0001:00018771       _gxv_trak_validate         00419771 f    CIL library: CIL module
 0001:000188f5       _gxv_just_wdc_entry_validate 004198f5 f    CIL library: CIL module
 0001:00018979       _gxv_just_widthDeltaClusters_validate 00419979 f    CIL library: CIL module
 0001:000189c4       _gxv_just_actSubrecord_type0_validate 004199c4 f    CIL library: CIL module
 0001:00018a42       _gxv_just_actSubrecord_validate 00419a42 f    CIL library: CIL module
 0001:00018b58       _gxv_just_pcActionRecord_validate 00419b58 f    CIL library: CIL module
 0001:00018bc9       _gxv_just_pcTable_LookupValue_entry_validate 00419bc9 f    CIL library: CIL module
 0001:00018bed       _gxv_just_postcompTable_validate 00419bed f    CIL library: CIL module
 0001:00018c33       _gxv_just_justClassTable_validate 00419c33 f    CIL library: CIL module
 0001:00018c8c       _gxv_just_wdcTable_LookupValue_validate 00419c8c f    CIL library: CIL module
 0001:00018cae       _gxv_just_justData_validate 00419cae f    CIL library: CIL module
 0001:00018e02       _gxv_just_validate         00419e02 f    CIL library: CIL module
 0001:00018f33       _gxv_mort_featurearray_validate 00419f33 f    CIL library: CIL module
 0001:00019052       _gxv_mort_subtables_validate 0041a052 f    CIL library: CIL module
 0001:0001911d       _gxv_mort_chain_validate   0041a11d f    CIL library: CIL module
 0001:000191b5       _gxv_mort_validate         0041a1b5 f    CIL library: CIL module
 0001:0001927b       _gxv_morx_subtable_type0_entry_validate 0041a27b f    CIL library: CIL module
 0001:0001927b       _gxv_mort_subtable_type0_entry_validate 0041a27b f    CIL library: CIL module
 0001:0001929d       _gxv_mort_subtable_type0_validate 0041a29d f    CIL library: CIL module
 0001:000192f7       _gxv_kern_subtable_fmt1_valueTable_load 0041a2f7 f    CIL library: CIL module
 0001:000192f7       _gxv_mort_subtable_type1_substitutionTable_load 0041a2f7 f    CIL library: CIL module
 0001:00019338       _gxv_mort_subtable_type1_entry_validate 0041a338 f    CIL library: CIL module
 0001:00019364       _gxv_mort_subtable_type1_substTable_validate 0041a364 f    CIL library: CIL module
 0001:000193e7       _gxv_mort_subtable_type1_validate 0041a3e7 f    CIL library: CIL module
 0001:00019469       _gxv_mort_subtable_type2_opttable_load 0041a469 f    CIL library: CIL module
 0001:000194ca       _gxv_mort_subtable_type2_subtable_setup 0041a4ca f    CIL library: CIL module
 0001:00019560       _gxv_mort_subtable_type2_ligActionOffset_validate 0041a560 f    CIL library: CIL module
 0001:000195b0       _gxv_mort_subtable_type2_entry_validate 0041a5b0 f    CIL library: CIL module
 0001:000195ca       _gxv_mort_subtable_type2_ligatureTable_validate 0041a5ca f    CIL library: CIL module
 0001:00019620       _gxv_mort_subtable_type2_validate 0041a620 f    CIL library: CIL module
 0001:0001969c       _gxv_mort_subtable_type4_lookupval_validate 0041a69c f    CIL library: CIL module
 0001:000196ab       _gxv_mort_subtable_type4_validate 0041a6ab f    CIL library: CIL module
 0001:000196d2       _gxv_mort_subtable_type5_subtable_setup 0041a6d2 f    CIL library: CIL module
 0001:00019726       _gxv_mort_subtable_type5_InsertList_validate 0041a726 f    CIL library: CIL module
 0001:00019773       _gxv_mort_subtable_type5_entry_validate 0041a773 f    CIL library: CIL module
 0001:000197cf       _gxv_mort_subtable_type5_validate 0041a7cf f    CIL library: CIL module
 0001:00019834       _gxv_morx_subtables_validate 0041a834 f    CIL library: CIL module
 0001:00019929       _gxv_morx_chain_validate   0041a929 f    CIL library: CIL module
 0001:000199eb       _gxv_morx_validate         0041a9eb f    CIL library: CIL module
 0001:00019a98       _gxv_morx_subtable_type0_validate 0041aa98 f    CIL library: CIL module
 0001:00019af0       _gxv_morx_subtable_type1_substitutionTable_load 0041aaf0 f    CIL library: CIL module
 0001:00019b30       _gxv_morx_subtable_type1_entry_validate 0041ab30 f    CIL library: CIL module
 0001:00019b8e       _gxv_morx_subtable_type1_LookupValue_validate 0041ab8e f    CIL library: CIL module
 0001:00019bb4       _gxv_morx_subtable_type1_substitutionTable_validate 0041abb4 f    CIL library: CIL module
 0001:00019c51       _gxv_morx_subtable_type1_validate 0041ac51 f    CIL library: CIL module
 0001:00019cd7       _gxv_morx_subtable_type2_opttable_load 0041acd7 f    CIL library: CIL module
 0001:00019d6d       _gxv_morx_subtable_type2_subtable_setup 0041ad6d f    CIL library: CIL module
 0001:00019ddf       _gxv_morx_subtable_type2_entry_validate 0041addf f    CIL library: CIL module
 0001:00019e1f       _gxv_morx_subtable_type2_ligatureTable_validate 0041ae1f f    CIL library: CIL module
 0001:00019e6b       _gxv_morx_subtable_type2_validate 0041ae6b f    CIL library: CIL module
 0001:00019eda       _gxv_morx_subtable_type4_validate 0041aeda f    CIL library: CIL module
 0001:00019edf       _gxv_morx_subtable_type5_insertionGlyphList_load 0041aedf f    CIL library: CIL module
 0001:00019f31       _gxv_morx_subtable_type5_subtable_setup 0041af31 f    CIL library: CIL module
 0001:00019f31       _gxv_morx_subtable_type1_subtable_setup 0041af31 f    CIL library: CIL module
 0001:00019f8b       _gxv_morx_subtable_type5_InsertList_validate 0041af8b f    CIL library: CIL module
 0001:00019fd8       _gxv_morx_subtable_type5_entry_validate 0041afd8 f    CIL library: CIL module
 0001:0001a037       _gxv_morx_subtable_type5_validate 0041b037 f    CIL library: CIL module
 0001:0001a09c       _gxv_kern_subtable_fmt0_pairs_validate 0041b09c f    CIL library: CIL module
 0001:0001a13e       _gxv_kern_subtable_fmt0_validate 0041b13e f    CIL library: CIL module
 0001:0001a1b4       _gxv_mort_subtable_type1_subtable_setup 0041b1b4 f    CIL library: CIL module
 0001:0001a1b4       _gxv_kern_subtable_fmt1_subtable_setup 0041b1b4 f    CIL library: CIL module
 0001:0001a22e       _gxv_kern_subtable_fmt1_entry_validate 0041b22e f    CIL library: CIL module
 0001:0001a28c       _gxv_kern_subtable_fmt2_clstbl_validate 0041b28c f    CIL library: CIL module
 0001:0001a347       _gxv_kern_subtable_fmt2_validate 0041b347 f    CIL library: CIL module
 0001:0001a50e       _gxv_kern_subtable_fmt3_validate 0041b50e f    CIL library: CIL module
 0001:0001a693       _gxv_kern_coverage_validate 0041b693 f    CIL library: CIL module
 0001:0001a716       _gxv_kern_subtable_validate 0041b716 f    CIL library: CIL module
 0001:0001a848       _gxv_kern_validate_generic 0041b848 f    CIL library: CIL module
 0001:0001a910       _gxv_opbd_LookupValue_validate 0041b910 f    CIL library: CIL module
 0001:0001a99d       _gxv_opbd_LookupFmt4_transit 0041b99d f    CIL library: CIL module
 0001:0001a9a9       _gxv_opbd_validate         0041b9a9 f    CIL library: CIL module
 0001:0001aa5f       _gxv_prop_zero_advance_validate 0041ba5f f    CIL library: CIL module
 0001:0001aaa9       _gxv_prop_property_validate 0041baa9 f    CIL library: CIL module
 0001:0001ab49       _gxv_prop_LookupValue_validate 0041bb49 f    CIL library: CIL module
 0001:0001ab5e       _gxv_prop_LookupFmt4_transit 0041bb5e f    CIL library: CIL module
 0001:0001ab5e       _gxv_XClassTable_lookupfmt4_transit 0041bb5e f    CIL library: CIL module
 0001:0001ab5e       _gxv_mort_subtable_type4_lookupfmt4_transit 0041bb5e f    CIL library: CIL module
 0001:0001ab5e       _gxv_morx_subtable_type1_LookupFmt4_transit 0041bb5e f    CIL library: CIL module
 0001:0001ab5e       _gxv_bsln_LookupFmt4_transit 0041bb5e f    CIL library: CIL module
 0001:0001aba7       _gxv_prop_validate         0041bba7 f    CIL library: CIL module
 0001:0001ac71       _gxv_lcar_LookupValue_validate 0041bc71 f    CIL library: CIL module
 0001:0001ad13       _gxv_lcar_LookupFmt4_transit 0041bd13 f    CIL library: CIL module
 0001:0001ad63       _gxv_lcar_validate         0041bd63 f    CIL library: CIL module
 0001:0001adf2       _gxv_load_table            0041bdf2 f    CIL library: CIL module
 0001:0001adf2       _otv_load_table            0041bdf2 f    CIL library: CIL module
 0001:0001ae4a       _gxv_validate              0041be4a f    CIL library: CIL module
 0001:0001b4e9       _classic_kern_validate     0041c4e9 f    CIL library: CIL module
 0001:0001b5ac       _otv_BaseCoord_validate    0041c5ac f    CIL library: CIL module
 0001:0001b60c       _otv_BaseValues_validate   0041c60c f    CIL library: CIL module
 0001:0001b673       _otv_MinMax_validate       0041c673 f    CIL library: CIL module
 0001:0001b81f       _otv_BaseScript_validate   0041c81f f    CIL library: CIL module
 0001:0001b95b       _otv_BaseScriptList_validate 0041c95b f    CIL library: CIL module
 0001:0001b9c6       _otv_Axis_validate         0041c9c6 f    CIL library: CIL module
 0001:0001ba6f       _otv_BASE_validate         0041ca6f f    CIL library: CIL module
 0001:0001bb4b       _otv_Coverage_validate     0041cb4b f    CIL library: CIL module
 0001:0001bc8c       _otv_Coverage_get_count    0041cc8c f    CIL library: CIL module
 0001:0001bce9       _otv_ClassDef_validate     0041cce9 f    CIL library: CIL module
 0001:0001bdf2       _otv_Device_validate       0041cdf2 f    CIL library: CIL module
 0001:0001be74       _otv_Lookup_validate       0041ce74 f    CIL library: CIL module
 0001:0001bef5       _otv_LookupList_validate   0041cef5 f    CIL library: CIL module
 0001:0001bf6b       _otv_Feature_validate      0041cf6b f    CIL library: CIL module
 0001:0001bfd3       _otv_FeatureList_validate  0041cfd3 f    CIL library: CIL module
 0001:0001c050       _otv_LangSys_validate      0041d050 f    CIL library: CIL module
 0001:0001c0e9       _otv_Script_validate       0041d0e9 f    CIL library: CIL module
 0001:0001c173       _otv_ScriptList_validate   0041d173 f    CIL library: CIL module
 0001:0001c1e8       _otv_x_Ox                  0041d1e8 f    CIL library: CIL module
 0001:0001c258       _otv_u_C_x_Ox              0041d258 f    CIL library: CIL module
 0001:0001c2ea       _otv_x_ux                  0041d2ea f    CIL library: CIL module
 0001:0001c35c       _otv_x_y_ux_sy             0041d35c f    CIL library: CIL module
 0001:0001c40b       _otv_x_ux_y_uy_z_uz_p_sp   0041d40b f    CIL library: CIL module
 0001:0001c4cb       _otv_u_O_O_x_Onx           0041d4cb f    CIL library: CIL module
 0001:0001c589       _otv_u_x_y_Ox_sy           0041d589 f    CIL library: CIL module
 0001:0001c641       _otv_u_O_O_O_O_x_Onx       0041d641 f    CIL library: CIL module
 0001:0001c73a       _otv_u_x_Ox_y_Oy_z_Oz_p_sp 0041d73a f    CIL library: CIL module
 0001:0001c876       _otv_GSUBGPOS_have_MarkAttachmentType_flag 0041d876 f    CIL library: CIL module
 0001:0001c8c4       _otv_O_x_Ox                0041d8c4 f    CIL library: CIL module
 0001:0001c969       _otv_CaretValue_validate   0041d969 f    CIL library: CIL module
 0001:0001c9c2       _otv_GDEF_validate         0041d9c2 f    CIL library: CIL module
 0001:0001cbb0       _otv_x_sxy                 0041dbb0 f    CIL library: CIL module
 0001:0001cc76       _otv_u_O_O_u_O_O           0041dc76 f    CIL library: CIL module
 0001:0001cd2c       _otv_value_length          0041dd2c f    CIL library: CIL module
 0001:0001cd55       _otv_ValueRecord_validate  0041dd55 f    CIL library: CIL module
 0001:0001ce11       _otv_Anchor_validate       0041de11 f    CIL library: CIL module
 0001:0001cf1f       _otv_MarkArray_validate    0041df1f f    CIL library: CIL module
 0001:0001cf94       _otv_SinglePos_validate    0041df94 f    CIL library: CIL module
 0001:0001d087       _otv_PairSet_validate      0041e087 f    CIL library: CIL module
 0001:0001d123       _otv_PairPos_validate      0041e123 f    CIL library: CIL module
 0001:0001d309       _otv_CursivePos_validate   0041e309 f    CIL library: CIL module
 0001:0001d439       _otv_MarkBasePos_validate  0041e439 f    CIL library: CIL module
 0001:0001d492       _otv_MarkLigPos_validate   0041e492 f    CIL library: CIL module
 0001:0001d4f2       _otv_MarkMarkPos_validate  0041e4f2 f    CIL library: CIL module
 0001:0001d547       _otv_ContextPos_validate   0041e547 f    CIL library: CIL module
 0001:0001d547       _otv_ContextSubst_validate 0041e547 f    CIL library: CIL module
 0001:0001d5e2       _otv_ChainContextPos_validate 0041e5e2 f    CIL library: CIL module
 0001:0001d5e2       _otv_ChainContextSubst_validate 0041e5e2 f    CIL library: CIL module
 0001:0001d67d       _otv_ExtensionPos_validate 0041e67d f    CIL library: CIL module
 0001:0001d714       _otv_GPOS_subtable_validate 0041e714 f    CIL library: CIL module
 0001:0001d731       _otv_GPOS_validate         0041e731 f    CIL library: CIL module
 0001:0001d7e4       _otv_SingleSubst_validate  0041e7e4 f    CIL library: CIL module
 0001:0001d919       _otv_AlternateSubst_validate 0041e919 f    CIL library: CIL module
 0001:0001d919       _otv_MultipleSubst_validate 0041e919 f    CIL library: CIL module
 0001:0001d972       _otv_Ligature_validate     0041e972 f    CIL library: CIL module
 0001:0001d9c8       _otv_LigatureSubst_validate 0041e9c8 f    CIL library: CIL module
 0001:0001da21       _otv_ExtensionSubst_validate 0041ea21 f    CIL library: CIL module
 0001:0001dac6       _otv_ReverseChainSingleSubst_validate 0041eac6 f    CIL library: CIL module
 0001:0001dbe2       _otv_GSUB_validate         0041ebe2 f    CIL library: CIL module
 0001:0001dc95       _otv_JstfPriority_validate 0041ec95 f    CIL library: CIL module
 0001:0001dfbb       _otv_JstfScript_validate   0041efbb f    CIL library: CIL module
 0001:0001e118       _otv_JSTF_validate         0041f118 f    CIL library: CIL module
 0001:0001e1ee       _otv_MathConstants_validate 0041f1ee f    CIL library: CIL module
 0001:0001e274       _otv_MathItalicsCorrectionInfo_validate 0041f274 f    CIL library: CIL module
 0001:0001e36f       _otv_MathKern_validate     0041f36f f    CIL library: CIL module
 0001:0001e478       _otv_MathKernInfo_validate 0041f478 f    CIL library: CIL module
 0001:0001e582       _otv_MathGlyphInfo_validate 0041f582 f    CIL library: CIL module
 0001:0001e625       _otv_GlyphAssembly_validate 0041f625 f    CIL library: CIL module
 0001:0001e702       _otv_MathGlyphConstruction_validate 0041f702 f    CIL library: CIL module
 0001:0001e7e4       _otv_MathVariants_validate 0041f7e4 f    CIL library: CIL module
 0001:0001e98e       _otv_MATH_validate         0041f98e f    CIL library: CIL module
 0001:0001ea37       _otv_validate              0041fa37 f    CIL library: CIL module
 0001:0001edff       _pcf_read_TOC              0041fdff f    CIL library: CIL module
 0001:0001ef70       _pcf_get_metric            0041ff70 f    CIL library: CIL module
 0001:0001eff8       _pcf_seek_to_table_type    0041fff8 f    CIL library: CIL module
 0001:0001f05f       _pcf_find_property         0042005f f    CIL library: CIL module
 0001:0001f0d8       _pcf_get_properties        004200d8 f    CIL library: CIL module
 0001:0001f374       _pcf_get_metrics           00420374 f    CIL library: CIL module
 0001:0001f4af       _pcf_get_bitmaps           004204af f    CIL library: CIL module
 0001:0001f608       _pcf_get_encodings         00420608 f    CIL library: CIL module
 0001:0001f80e       _pcf_get_accel             0042080e f    CIL library: CIL module
 0001:0001f90c       _pcf_interpret_style       0042090c f    CIL library: CIL module
 0001:0001fac8       _pcf_load_font             00420ac8 f    CIL library: CIL module
 0001:0001fdaa       _pcf_cmap_init             00420daa f    CIL library: CIL module
 0001:0001fdc5       _pcf_cmap_char_next        00420dc5 f    CIL library: CIL module
 0001:0001fdc5       _bdf_cmap_char_next        00420dc5 f    CIL library: CIL module
 0001:0001fe27       _PCF_Face_Done             00420e27 f    CIL library: CIL module
 0001:0001ff5f       _PCF_Face_Init             00420f5f f    CIL library: CIL module
 0001:000200b9       _PCF_Size_Select           004210b9 f    CIL library: CIL module
 0001:000200f8       _PCF_Size_Request          004210f8 f    CIL library: CIL module
 0001:0002016f       _PCF_Glyph_Load            0042116f f    CIL library: CIL module
 0001:0002039d       _pcf_get_bdf_property      0042139d f    CIL library: CIL module
 0001:000203d4       _pcf_get_charset_id        004213d4 f    CIL library: CIL module
 0001:000203f3       _pcf_driver_requester      004213f3 f    CIL library: CIL module
 0001:00020403       _pfr_extra_items_parse     00421403 f    CIL library: CIL module
 0001:0002047f       _pfr_log_font_load         0042147f f    CIL library: CIL module
 0001:000206e7       _pfr_extra_item_load_bitmap_info 004216e7 f    CIL library: CIL module
 0001:00020871       _pfr_extra_item_load_font_id 00421871 f    CIL library: CIL module
 0001:000208bf       _pfr_extra_item_load_stem_snaps 004218bf f    CIL library: CIL module
 0001:00020950       _pfr_extra_item_load_kerning_pairs 00421950 f    CIL library: CIL module
 0001:00020aa2       _pfr_aux_name_load         00421aa2 f    CIL library: CIL module
 0001:00020b17       _pfr_phy_font_done         00421b17 f    CIL library: CIL module
 0001:00020bcf       _pfr_phy_font_load         00421bcf f    CIL library: CIL module
 0001:00020ff8       _pfr_glyph_close_contour   00421ff8 f    CIL library: CIL module
 0001:0002106d       _pfr_glyph_line_to         0042206d f    CIL library: CIL module
 0001:000210c6       _pfr_glyph_curve_to        004220c6 f    CIL library: CIL module
 0001:00021153       _pfr_glyph_move_to         00422153 f    CIL library: CIL module
 0001:000211a1       _pfr_glyph_load_simple     004221a1 f    CIL library: CIL module
 0001:000215e5       _pfr_glyph_load_compound   004225e5 f    CIL library: CIL module
 0001:00021883       _pfr_glyph_load_rec        00422883 f    CIL library: CIL module
 0001:000219ff       _pfr_cmap_init             004229ff f    CIL library: CIL module
 0001:00021a3e       _pfr_cmap_char_index       00422a3e f    CIL library: CIL module
 0001:00021a7c       _pfr_cmap_char_next        00422a7c f    CIL library: CIL module
 0001:00021af1       _pfr_face_done             00422af1 f    CIL library: CIL module
 0001:00021b2c       _pfr_face_init             00422b2c f    CIL library: CIL module
 0001:00021e3a       _pfr_slot_init             00422e3a f    CIL library: CIL module
 0001:00021e69       _pfr_slot_done             00422e69 f    CIL library: CIL module
 0001:00021ec8       _pfr_slot_load             00422ec8 f    CIL library: CIL module
 0001:000220c1       _pfr_face_get_kerning      004230c1 f    CIL library: CIL module
 0001:0002229e       _pfr_get_kerning           0042329e f    CIL library: CIL module
 0001:000222fb       _pfr_get_advance           004232fb f    CIL library: CIL module
 0001:00022332       _pfr_get_metrics           00423332 f    CIL library: CIL module
 0001:000223a4       _pfr_get_service           004233a4 f    CIL library: CIL module
 0001:000223b4       _pfr_bitwriter_decode_bytes 004233b4 f    CIL library: CIL module
 0001:00022455       _pfr_bitwriter_decode_rle1 00423455 f    CIL library: CIL module
 0001:00022529       _pfr_bitwriter_decode_rle2 00423529 f    CIL library: CIL module
 0001:000225d0       _pfr_lookup_bitmap_data    004235d0 f    CIL library: CIL module
 0001:000226a7       _pfr_load_bitmap_metrics   004236a7 f    CIL library: CIL module
 0001:000228ab       _pfr_load_bitmap_bits      004238ab f    CIL library: CIL module
 0001:00022936       _pfr_slot_load_bitmap      00423936 f   pfrsbit.obj
 0001:00022b88       _ps_table_new              00423b88 f    CIL library: CIL module
 0001:00022c11       _shift_elements            00423c11 f    CIL library: CIL module
 0001:00022c36       _reallocate_t1_table       00423c36 f    CIL library: CIL module
 0001:00022c8d       _ps_table_add              00423c8d f    CIL library: CIL module
 0001:00022d36       _ps_table_done             00423d36 f    CIL library: CIL module
 0001:00022d88       _ps_table_release          00423d88 f    CIL library: CIL module
 0001:00022dcc       _skip_spaces               00423dcc f    CIL library: CIL module
 0001:00022e0f       _skip_literal_string       00423e0f f    CIL library: CIL module
 0001:00022e98       _skip_string               00423e98 f    CIL library: CIL module
 0001:00022ef8       _skip_procedure            00423ef8 f    CIL library: CIL module
 0001:00022f7c       _ps_parser_skip_PS_token   00423f7c f    CIL library: CIL module
 0001:0002307b       _ps_parser_skip_spaces     0042407b f    CIL library: CIL module
 0001:0002308a       _ps_parser_to_token        0042408a f    CIL library: CIL module
 0001:000231a5       _ps_parser_to_token_array  004241a5 f    CIL library: CIL module
 0001:0002324f       _ps_tocoordarray           0042424f f    CIL library: CIL module
 0001:00023307       _ps_tofixedarray           00424307 f    CIL library: CIL module
 0001:000233bc       _ps_tobool                 004243bc f    CIL library: CIL module
 0001:00023417       _ps_parser_load_field      00424417 f    CIL library: CIL module
 0001:00023644       _ps_parser_load_field_table 00424644 f    CIL library: CIL module
 0001:00023723       _ps_parser_to_int          00424723 f    CIL library: CIL module
 0001:0002373a       _ps_parser_to_bytes        0042473a f    CIL library: CIL module
 0001:0002379f       _ps_parser_to_fixed        0042479f f    CIL library: CIL module
 0001:000237be       _ps_parser_to_coord_array  004247be f    CIL library: CIL module
 0001:000237df       _ps_parser_to_fixed_array  004247df f    CIL library: CIL module
 0001:00023804       _ps_parser_init            00424804 f    CIL library: CIL module
 0001:00023835       _t1_builder_init           00424835 f    CIL library: CIL module
 0001:000238b9       _t1_builder_done           004248b9 f    CIL library: CIL module
 0001:000238d4       _t1_builder_check_points   004248d4 f    CIL library: CIL module
 0001:0002390b       _t1_builder_add_point      0042490b f    CIL library: CIL module
 0001:00023962       _t1_builder_add_point1     00424962 f    CIL library: CIL module
 0001:00023990       _t1_builder_add_contour    00424990 f    CIL library: CIL module
 0001:000239ee       _t1_builder_start_point    004249ee f    CIL library: CIL module
 0001:00023a27       _t1_builder_close_contour  00424a27 f    CIL library: CIL module
 0001:00023ab9       _t1_decrypt                00424ab9 f    CIL library: CIL module
 0001:00023ad8       _t1_lookup_glyph_by_stdcharcode 00424ad8 f    CIL library: CIL module
 0001:00023b5c       _t1operator_seac           00424b5c f    CIL library: CIL module
 0001:00023c85       _t1_decoder_parse_charstrings 00424c85 f    CIL library: CIL module
 0001:00024701       _t1_decoder_init           00425701 f    CIL library: CIL module
 0001:0002478e       _t1_decoder_done           0042578e f    CIL library: CIL module
 0001:00024793       _t1_cmap_std_init          00425793 f    CIL library: CIL module
 0001:000247c8       _t1_cmap_std_done          004257c8 f    CIL library: CIL module
 0001:000247db       _t1_cmap_std_char_index    004257db f    CIL library: CIL module
 0001:0002485f       _t1_cmap_std_char_next     0042585f f    CIL library: CIL module
 0001:0002488e       _t1_cmap_standard_init     0042588e f    CIL library: CIL module
 0001:0002489d       _t1_cmap_expert_init       0042589d f    CIL library: CIL module
 0001:000248ac       _t1_cmap_custom_init       004258ac f    CIL library: CIL module
 0001:000248d4       _t1_cmap_custom_done       004258d4 f    CIL library: CIL module
 0001:000248e4       _t1_cmap_custom_char_index 004258e4 f    CIL library: CIL module
 0001:0002490a       _t1_cmap_custom_char_next  0042590a f    CIL library: CIL module
 0001:00024948       _t1_get_glyph_name         00425948 f    CIL library: CIL module
 0001:0002495a       _t1_cmap_unicode_init      0042595a f    CIL library: CIL module
 0001:00024982       _t1_cmap_unicode_char_index 00425982 f    CIL library: CIL module
 0001:00024999       _t1_cmap_unicode_char_next 00425999 f    CIL library: CIL module
 0001:000249b0       _afm_stream_skip_spaces    004259b0 f    CIL library: CIL module
 0001:00024a0b       _afm_stream_read_one       00425a0b f    CIL library: CIL module
 0001:00024a71       _afm_stream_read_string    00425a71 f    CIL library: CIL module
 0001:00024abf       _afm_parser_read_vals      00425abf f    CIL library: CIL module
 0001:00024bd8       _afm_parser_next_key       00425bd8 f    CIL library: CIL module
 0001:00024c14       _afm_tokenize              00425c14 f    CIL library: CIL module
 0001:00024c5a       _afm_parser_init           00425c5a f    CIL library: CIL module
 0001:00024ca5       _afm_parser_done           00425ca5 f    CIL library: CIL module
 0001:00024cbb       _afm_parser_read_int       00425cbb f    CIL library: CIL module
 0001:00024cee       _afm_parse_track_kern      00425cee f    CIL library: CIL module
 0001:00024e1c       _compare_kern_pairs        00425e1c f    CIL library: CIL module
 0001:00024e1c       _afm_compare_kern_pairs    00425e1c f    CIL library: CIL module
 0001:00024e3f       _afm_parse_kern_pairs      00425e3f f    CIL library: CIL module
 0001:00024f8a       _afm_parse_kern_data       00425f8a f    CIL library: CIL module
 0001:00024fec       _afm_parser_skip_section   00425fec f    CIL library: CIL module
 0001:0002503d       _afm_parser_parse          0042603d f    CIL library: CIL module
 0001:0002528d       _PS_Conv_Strtol            0042628d f    CIL library: CIL module
 0001:0002530f       _PS_Conv_ToInt             0042630f f    CIL library: CIL module
 0001:00025335       _PS_Conv_ToFixed           00426335 f    CIL library: CIL module
 0001:00025483       _PS_Conv_ASCIIHexDecode    00426483 f    CIL library: CIL module
 0001:00025519       _PS_Conv_EexecDecode       00426519 f    CIL library: CIL module
 0001:00025591       _ps_mask_ensure            00426591 f    CIL library: CIL module
 0001:000255df       _ps_mask_test_bit          004265df f    CIL library: CIL module
 0001:000255ff       _ps_mask_set_bit           004265ff f    CIL library: CIL module
 0001:00025636       _ps_mask_table_done        00426636 f    CIL library: CIL module
 0001:0002567e       _ps_mask_table_ensure      0042667e f    CIL library: CIL module
 0001:000256bb       _ps_mask_table_alloc       004266bb f    CIL library: CIL module
 0001:000256f6       _ps_mask_table_last        004266f6 f    CIL library: CIL module
 0001:00025727       _ps_mask_table_set_bits    00426727 f    CIL library: CIL module
 0001:000257b1       _ps_mask_table_merge       004267b1 f    CIL library: CIL module
 0001:000258a4       _ps_mask_table_merge_all   004268a4 f    CIL library: CIL module
 0001:00025977       _ps_dimension_done         00426977 f    CIL library: CIL module
 0001:000259ab       _ps_dimension_reset_mask   004269ab f    CIL library: CIL module
 0001:000259d1       _ps_dimension_set_mask_bits 004269d1 f    CIL library: CIL module
 0001:000259ee       _ps_dimension_add_t1stem   004269ee f    CIL library: CIL module
 0001:00025b08       _ps_dimension_add_counter  00426b08 f    CIL library: CIL module
 0001:00025b9c       _ps_dimension_end          00426b9c f    CIL library: CIL module
 0001:00025bbd       _ps_hints_stem             00426bbd f    CIL library: CIL module
 0001:00025c19       _ps_hints_t1stem3          00426c19 f    CIL library: CIL module
 0001:00025cb2       _ps_hints_t1reset          00426cb2 f    CIL library: CIL module
 0001:00025cf3       _ps_hints_t2mask           00426cf3 f    CIL library: CIL module
 0001:00025d55       _ps_hints_t2counter        00426d55 f    CIL library: CIL module
 0001:00025dcd       _ps_hints_close            00426dcd f    CIL library: CIL module
 0001:00025dff       _t1_hints_open             00426dff f    CIL library: CIL module
 0001:00025e22       _t1_hints_stem             00426e22 f    CIL library: CIL module
 0001:00025e39       _t2_hints_open             00426e39 f    CIL library: CIL module
 0001:00025e5c       _t2_hints_stems            00426e5c f    CIL library: CIL module
 0001:00025edd       _psh_globals_scale_widths  00426edd f    CIL library: CIL module
 0001:00025f55       _psh_blues_set_zones_0     00426f55 f    CIL library: CIL module
 0001:00026059       _psh_blues_set_zones       00427059 f    CIL library: CIL module
 0001:0002618c       _psh_blues_scale_zones     0042718c f    CIL library: CIL module
 0001:0002630c       _psh_blues_snap_stem       0042730c f    CIL library: CIL module
 0001:000263e2       _psh_globals_destroy       004273e2 f    CIL library: CIL module
 0001:00026417       _psh_globals_new           00427417 f    CIL library: CIL module
 0001:0002652f       _psh_globals_set_scale     0042752f f    CIL library: CIL module
 0001:000265a1       _psh_hint_table_done       004275a1 f    CIL library: CIL module
 0001:000265e4       _psh_hint_table_record     004275e4 f    CIL library: CIL module
 0001:00026659       _psh_hint_table_init       00427659 f    CIL library: CIL module
 0001:00026795       _psh_hint_table_activate_mask 00427795 f    CIL library: CIL module
 0001:0002686d       _psh_dimension_quantize_len 0042786d f    CIL library: CIL module
 0001:000268c0       _psh_hint_align            004278c0 f    CIL library: CIL module
 0001:00026b33       _psh_glyph_compute_inflections 00427b33 f    CIL library: CIL module
 0001:00026c70       _psh_glyph_done            00427c70 f    CIL library: CIL module
 0001:00026cb1       _psh_compute_dir           00427cb1 f    CIL library: CIL module
 0001:00026cf1       _psh_glyph_load_points     00427cf1 f    CIL library: CIL module
 0001:00026d33       _psh_glyph_save_points     00427d33 f    CIL library: CIL module
 0001:00026d8e       _psh_glyph_init            00427d8e f    CIL library: CIL module
 0001:00026fd1       _psh_glyph_compute_extrema 00427fd1 f    CIL library: CIL module
 0001:000270b8       _psh_hint_table_find_strong_points 004280b8 f    CIL library: CIL module
 0001:00027269       _psh_glyph_find_strong_points 00428269 f    CIL library: CIL module
 0001:0002736e       _psh_glyph_find_blue_points 0042836e f    CIL library: CIL module
 0001:00027478       _psh_glyph_interpolate_strong_points 00428478 f    CIL library: CIL module
 0001:00027517       _psh_glyph_interpolate_normal_points 00428517 f    CIL library: CIL module
 0001:000276ef       _psh_glyph_interpolate_other_points 004286ef f    CIL library: CIL module
 0001:00027a5d       _ps_hinter_done            00428a5d f    CIL library: CIL module
 0001:00027a92       _ps_hinter_init            00428a92 f    CIL library: CIL module
 0001:00027b37       _pshinter_get_globals_funcs 00428b37 f    CIL library: CIL module
 0001:00027b3f       _pshinter_get_t1_funcs     00428b3f f    CIL library: CIL module
 0001:00027b47       _pshinter_get_t2_funcs     00428b47 f    CIL library: CIL module
 0001:00027b51       _ft_get_adobe_glyph_index  00428b51 f    CIL library: CIL module
 0001:00027c15       _ps_unicode_value          00428c15 f    CIL library: CIL module
 0001:00027cf0       _compare_uni_maps          00428cf0 f    CIL library: CIL module
 0001:00027d21       _ps_unicodes_init          00428d21 f    CIL library: CIL module
 0001:00027ed5       _ps_unicodes_char_index    00428ed5 f    CIL library: CIL module
 0001:00027f33       _ps_unicodes_char_next     00428f33 f    CIL library: CIL module
 0001:00027fb9       _ps_get_macintosh_name     00428fb9 f    CIL library: CIL module
 0001:00027fd4       _ps_get_standard_strings   00428fd4 f    CIL library: CIL module
 0001:00027ff0       _psnames_get_service       00428ff0 f    CIL library: CIL module
 0001:00028000       _New_Profile               00429000 f    CIL library: CIL module
 0001:00028087       _End_Profile               00429087 f    CIL library: CIL module
 0001:000280e6       _Insert_Y_Turn             004290e6 f    CIL library: CIL module
 0001:0002814a       _Finalize_Profile_Table    0042914a f    CIL library: CIL module
 0001:000281e5       _Split_Conic               004291e5 f    CIL library: CIL module
 0001:00028245       _Split_Cubic               00429245 f    CIL library: CIL module
 0001:000282d1       _Line_Up                   004292d1 f    CIL library: CIL module
 0001:00028426       _Bezier_Up                 00429426 f    CIL library: CIL module
 0001:00028578       _Bezier_Down               00429578 f    CIL library: CIL module
 0001:000285bf       _Line_To                   004295bf f    CIL library: CIL module
 0001:000286a0       _Conic_To                  004296a0 f    CIL library: CIL module
 0001:000287a7       _Cubic_To                  004297a7 f    CIL library: CIL module
 0001:000288dd       _Decompose_Curve           004298dd f    CIL library: CIL module
 0001:00028bb4       _Convert_Glyph             00429bb4 f    CIL library: CIL module
 0001:00028ca3       _InsNew                    00429ca3 f    CIL library: CIL module
 0001:00028cbc       _DelOld                    00429cbc f    CIL library: CIL module
 0001:00028cd4       _Sort                      00429cd4 f    CIL library: CIL module
 0001:00028d2f       _Vertical_Sweep_Init       00429d2f f    CIL library: CIL module
 0001:00028d79       _Vertical_Sweep_Span       00429d79 f    CIL library: CIL module
 0001:00028e4a       _Vertical_Sweep_Drop       00429e4a f    CIL library: CIL module
 0001:00028f7c       _Vertical_Sweep_Step       00429f7c f    CIL library: CIL module
 0001:00028f8e       _Horizontal_Sweep_Span     00429f8e f    CIL library: CIL module
 0001:00028ffa       _Horizontal_Sweep_Drop     00429ffa f    CIL library: CIL module
 0001:00029128       _Draw_Sweep                0042a128 f    CIL library: CIL module
 0001:000293e6       _Render_Single_Pass        0042a3e6 f    CIL library: CIL module
 0001:000294e7       _Render_Glyph              0042a4e7 f    CIL library: CIL module
 0001:00029644       _ft_black_new              0042a644 f    CIL library: CIL module
 0001:00029673       _ft_black_done             0042a673 f    CIL library: CIL module
 0001:00029682       _ft_black_reset            0042a682 f    CIL library: CIL module
 0001:000296c2       _ft_black_render           0042a6c2 f    CIL library: CIL module
 0001:00029795       _ft_raster1_init           0042a795 f    CIL library: CIL module
 0001:00029795       _ft_smooth_init            0042a795 f    CIL library: CIL module
 0001:000297ba       _ft_smooth_get_cbox        0042a7ba f    CIL library: CIL module
 0001:000297ba       _ft_raster1_get_cbox       0042a7ba f    CIL library: CIL module
 0001:000297e3       _ft_raster1_render         0042a7e3 f    CIL library: CIL module
 0001:00029970       _tt_face_lookup_table      0042a970 f    CIL library: CIL module
 0001:0002999c       _tt_face_goto_table        0042a99c f    CIL library: CIL module
 0001:000299cd       _check_table_dir           0042a9cd f    CIL library: CIL module
 0001:00029aff       _tt_face_load_font_dir     0042aaff f    CIL library: CIL module
 0001:00029c15       _tt_face_load_any          0042ac15 f    CIL library: CIL module
 0001:00029c74       _tt_face_load_head         0042ac74 f    CIL library: CIL module
 0001:00029cab       _tt_face_load_bhed         0042acab f    CIL library: CIL module
 0001:00029ce2       _tt_face_load_maxp         0042ace2 f    CIL library: CIL module
 0001:00029e88       _tt_face_load_name         0042ae88 f    CIL library: CIL module
 0001:00029fc8       _tt_face_free_name         0042afc8 f    CIL library: CIL module
 0001:0002a03c       _tt_face_load_cmap         0042b03c f    CIL library: CIL module
 0001:0002a07f       _tt_face_load_os2          0042b07f f    CIL library: CIL module
 0001:0002a3fb       _tt_face_load_post         0042b3fb f    CIL library: CIL module
 0001:0002a432       _tt_face_load_pclt         0042b432 f    CIL library: CIL module
 0001:0002a469       _tt_face_load_gasp         0042b469 f    CIL library: CIL module
 0001:0002a555       _tt_face_load_hmtx         0042b555 f    CIL library: CIL module
 0001:0002a75b       _tt_face_load_hhea         0042b75b f    CIL library: CIL module
 0001:0002a8c4       _tt_face_get_metrics       0042b8c4 f    CIL library: CIL module
 0001:0002a948       _tt_cmap_init              0042b948 f    CIL library: CIL module
 0001:0002a956       _tt_cmap0_validate         0042b956 f    CIL library: CIL module
 0001:0002a9bb       _tt_cmap0_char_index       0042b9bb f    CIL library: CIL module
 0001:0002a9d6       _tt_cmap0_char_next        0042b9d6 f    CIL library: CIL module
 0001:0002aa0b       _tt_cmap0_get_info         0042ba0b f    CIL library: CIL module
 0001:0002aa29       _tt_cmap2_validate         0042ba29 f    CIL library: CIL module
 0001:0002ab78       _tt_cmap2_get_subheader    0042bb78 f    CIL library: CIL module
 0001:0002abc4       _tt_cmap2_char_index       0042bbc4 f    CIL library: CIL module
 0001:0002ac42       _tt_cmap2_char_next        0042bc42 f    CIL library: CIL module
 0001:0002ad2d       _tt_cmap2_get_info         0042bd2d f    CIL library: CIL module
 0001:0002ad4e       _tt_cmap4_init             0042bd4e f    CIL library: CIL module
 0001:0002ad71       _tt_cmap4_set_range        0042bd71 f    CIL library: CIL module
 0001:0002ae88       _tt_cmap4_next             0042be88 f    CIL library: CIL module
 0001:0002af0c       _tt_cmap4_validate         0042bf0c f    CIL library: CIL module
 0001:0002b207       _tt_cmap4_char_map_linear  0042c207 f    CIL library: CIL module
 0001:0002b36b       _tt_cmap4_char_map_binary  0042c36b f    CIL library: CIL module
 0001:0002b77c       _tt_cmap4_char_index       0042c77c f    CIL library: CIL module
 0001:0002b7ab       _tt_cmap4_char_next        0042c7ab f    CIL library: CIL module
 0001:0002b7fc       _tt_cmap4_get_info         0042c7fc f    CIL library: CIL module
 0001:0002b81b       _tt_cmap6_validate         0042c81b f    CIL library: CIL module
 0001:0002b8a7       _tt_cmap6_char_index       0042c8a7 f    CIL library: CIL module
 0001:0002b8e0       _tt_cmap6_char_next        0042c8e0 f    CIL library: CIL module
 0001:0002b957       _tt_cmap6_get_info         0042c957 f    CIL library: CIL module
 0001:0002b978       _tt_cmap8_validate         0042c978 f    CIL library: CIL module
 0001:0002bbd1       _tt_cmap8_char_index       0042cbd1 f    CIL library: CIL module
 0001:0002bca8       _tt_cmap8_char_next        0042cca8 f    CIL library: CIL module
 0001:0002bdbc       _tt_cmap8_get_info         0042cdbc f    CIL library: CIL module
 0001:0002bdef       _tt_cmap10_validate        0042cdef f    CIL library: CIL module
 0001:0002be9d       _tt_cmap10_char_index      0042ce9d f    CIL library: CIL module
 0001:0002befd       _tt_cmap10_char_next       0042cefd f    CIL library: CIL module
 0001:0002bf84       _tt_cmap10_get_info        0042cf84 f    CIL library: CIL module
 0001:0002bfb9       _tt_cmap12_init            0042cfb9 f    CIL library: CIL module
 0001:0002bfec       _tt_cmap12_validate        0042cfec f    CIL library: CIL module
 0001:0002c177       _tt_cmap12_next            0042d177 f    CIL library: CIL module
 0001:0002c231       _tt_cmap12_char_map_binary 0042d231 f    CIL library: CIL module
 0001:0002c36b       _tt_cmap12_char_index      0042d36b f    CIL library: CIL module
 0001:0002c380       _tt_cmap12_char_next       0042d380 f    CIL library: CIL module
 0001:0002c3cb       _tt_cmap12_get_info        0042d3cb f    CIL library: CIL module
 0001:0002c400       _tt_cmap14_done            0042d400 f    CIL library: CIL module
 0001:0002c424       _tt_cmap14_ensure          0042d424 f    CIL library: CIL module
 0001:0002c45c       _tt_cmap14_init            0042d45c f    CIL library: CIL module
 0001:0002c493       _tt_cmap14_validate        0042d493 f    CIL library: CIL module
 0001:0002c730       _af_dummy_hints_apply      0042d730 f    CIL library: CIL module
 0001:0002c730       _cid_driver_init           0042d730 f    CIL library: CIL module
 0001:0002c730       _T1_Driver_Init            0042d730 f    CIL library: CIL module
 0001:0002c730       _dummy_consume_data        0042d730 f    CIL library: CIL module
 0001:0002c730       _tt_cmap14_char_index      0042d730 f    CIL library: CIL module
 0001:0002c730       _cff_driver_init           0042d730 f    CIL library: CIL module
 0001:0002c730       _tt_face_free_charmap_stub 0042d730 f    CIL library: CIL module
 0001:0002c733       _tt_cmap14_char_next       0042d733 f    CIL library: CIL module
 0001:0002c73d       _tt_cmap14_get_info        0042d73d f    CIL library: CIL module
 0001:0002c74e       _tt_cmap14_char_map_def_binary 0042d74e f    CIL library: CIL module
 0001:0002c7bf       _tt_cmap14_char_map_nondef_binary 0042d7bf f    CIL library: CIL module
 0001:0002c833       _tt_cmap14_find_variant    0042d833 f    CIL library: CIL module
 0001:0002c89c       _tt_cmap14_char_var_index  0042d89c f    CIL library: CIL module
 0001:0002c92b       _tt_cmap14_char_var_isdefault 0042d92b f    CIL library: CIL module
 0001:0002c9bf       _tt_cmap14_variants        0042d9bf f    CIL library: CIL module
 0001:0002ca33       _tt_cmap14_char_variants   0042da33 f    CIL library: CIL module
 0001:0002cb46       _tt_cmap14_def_char_count  0042db46 f    CIL library: CIL module
 0001:0002cb7b       _tt_cmap14_get_def_chars   0042db7b f    CIL library: CIL module
 0001:0002cbfa       _tt_cmap14_get_nondef_chars 0042dbfa f    CIL library: CIL module
 0001:0002cc8e       _tt_cmap14_variant_chars   0042dc8e f    CIL library: CIL module
 0001:0002cf1f       _tt_face_build_cmaps       0042df1f f    CIL library: CIL module
 0001:0002d107       _tt_get_cmap_info          0042e107 f    CIL library: CIL module
 0001:0002d119       _tt_face_load_kern         0042e119 f    CIL library: CIL module
 0001:0002d2e8       _tt_face_get_kerning       0042e2e8 f    CIL library: CIL module
 0001:0002d48b       _tt_name_entry_ascii_from_utf16 0042e48b f    CIL library: CIL module
 0001:0002d4eb       _tt_name_entry_ascii_from_other 0042e4eb f    CIL library: CIL module
 0001:0002d543       _tt_face_get_name          0042e543 f    CIL library: CIL module
 0001:0002d710       _sfnt_open_font            0042e710 f    CIL library: CIL module
 0001:0002d856       _sfnt_init_face            0042e856 f    CIL library: CIL module
 0001:0002d902       _sfnt_load_face            0042e902 f    CIL library: CIL module
 0001:0002dea1       _sfnt_done_face            0042eea1 f    CIL library: CIL module
 0001:0002e03a       _get_sfnt_table            0042f03a f    CIL library: CIL module
 0001:0002e0bf       _sfnt_table_info           0042f0bf f    CIL library: CIL module
 0001:0002e10c       _sfnt_get_glyph_name       0042f10c f    CIL library: CIL module
 0001:0002e13d       _sfnt_get_name_index       0042f13d f    CIL library: CIL module
 0001:0002e19b       _sfnt_get_ps_name          0042f19b f    CIL library: CIL module
 0001:0002e397       _sfnt_get_charset_id       0042f397 f    CIL library: CIL module
 0001:0002e3f0       _sfnt_get_interface        0042f3f0 f    CIL library: CIL module
 0001:0002e400       _tt_face_set_sbit_strike_stub 0042f400 f    CIL library: CIL module
 0001:0002e438       _tt_face_load_sbit_stub    0042f438 f    CIL library: CIL module
 0001:0002e438       _tt_face_load_directory_stub 0042f438 f    CIL library: CIL module
 0001:0002e438       _tt_face_load_charmap_stub 0042f438 f    CIL library: CIL module
 0001:0002e438       _tt_face_load_sfnt_header_stub 0042f438 f    CIL library: CIL module
 0001:0002e438       _tt_face_load_hdmx_stub    0042f438 f    CIL library: CIL module
 0001:0002e43c       _blit_sbit                 0042f43c f    CIL library: CIL module
 0001:0002e570       _Load_SBit_Const_Metrics   0042f570 f    CIL library: CIL module
 0001:0002e5ac       _Load_SBit_Range_Codes     0042f5ac f    CIL library: CIL module
 0001:0002e67f       _Load_SBit_Range           0042f67f f    CIL library: CIL module
 0001:0002e780       _tt_face_load_eblc         0042f780 f    CIL library: CIL module
 0001:0002ea02       _tt_face_free_eblc         0042fa02 f    CIL library: CIL module
 0001:0002eaa8       _tt_face_set_sbit_strike   0042faa8 f    CIL library: CIL module
 0001:0002eabc       _tt_face_load_strike_metrics 0042fabc f    CIL library: CIL module
 0001:0002eb26       _find_sbit_range           0042fb26 f    CIL library: CIL module
 0001:0002ec03       _tt_find_sbit_image        0042fc03 f    CIL library: CIL module
 0001:0002ec5d       _tt_load_sbit_metrics      0042fc5d f    CIL library: CIL module
 0001:0002ed0e       _crop_bitmap               0042fd0e f    CIL library: CIL module
 0001:0002ee99       _Load_SBit_Single          0042fe99 f    CIL library: CIL module
 0001:0002ef74       _Load_SBit_Image           0042ff74 f    CIL library: CIL module
 0001:0002f1fe       _tt_face_load_sbit_image   004301fe f    CIL library: CIL module
 0001:0002f2d9       _load_format_20            004302d9 f    CIL library: CIL module
 0001:0002f4a0       _load_format_25            004304a0 f    CIL library: CIL module
 0001:0002f550       _load_post_names           00430550 f    CIL library: CIL module
 0001:0002f5b3       _tt_face_free_ps_names     004305b3 f    CIL library: CIL module
 0001:0002f677       _tt_face_get_ps_name       00430677 f    CIL library: CIL module
 0001:0002f76d       _tt_face_load_bdf_props    0043076d f    CIL library: CIL module
 0001:0002f87e       _tt_face_find_bdf_prop     0043087e f    CIL library: CIL module
 0001:0002fa33       _gray_compute_cbox         00430a33 f    CIL library: CIL module
 0001:0002fabf       _gray_find_cell            00430abf f    CIL library: CIL module
 0001:0002fb21       _gray_record_cell          00430b21 f    CIL library: CIL module
 0001:0002fb43       _gray_set_cell             00430b43 f    CIL library: CIL module
 0001:0002fb99       _gray_render_scanline      00430b99 f    CIL library: CIL module
 0001:0002fcd5       _gray_render_line          00430cd5 f    CIL library: CIL module
 0001:0002ff05       _gray_split_conic          00430f05 f    CIL library: CIL module
 0001:0002ff61       _gray_render_conic         00430f61 f    CIL library: CIL module
 0001:0003010c       _gray_split_cubic          0043110c f    CIL library: CIL module
 0001:000301bc       _gray_render_cubic         004311bc f    CIL library: CIL module
 0001:000303f3       _gray_move_to              004313f3 f    CIL library: CIL module
 0001:00030468       _gray_line_to              00431468 f    CIL library: CIL module
 0001:00030487       _gray_conic_to             00431487 f    CIL library: CIL module
 0001:0003049e       _gray_cubic_to             0043149e f    CIL library: CIL module
 0001:000304ba       _gray_render_span          004314ba f    CIL library: CIL module
 0001:0003055d       _gray_hline                0043155d f    CIL library: CIL module
 0001:0003067f       _gray_sweep                0043167f f    CIL library: CIL module
 0001:00030757       _gray_convert_glyph_inner  00431757 f    CIL library: CIL module
 0001:000307a2       _gray_convert_glyph        004317a2 f    CIL library: CIL module
 0001:00030a92       _gray_raster_render        00431a92 f    CIL library: CIL module
 0001:00030c4a       _gray_raster_new           00431c4a f    CIL library: CIL module
 0001:00030c79       _gray_raster_done          00431c79 f    CIL library: CIL module
 0001:00030c88       _gray_raster_reset         00431c88 f    CIL library: CIL module
 0001:00030cca       _ft_raster1_set_mode       00431cca f    CIL library: CIL module
 0001:00030cca       _ft_smooth_set_mode        00431cca f    CIL library: CIL module
 0001:00030ce6       _ft_raster1_transform      00431ce6 f    CIL library: CIL module
 0001:00030ce6       _ft_smooth_transform       00431ce6 f    CIL library: CIL module
 0001:00030d2c       _ft_smooth_render_generic  00431d2c f    CIL library: CIL module
 0001:00030f85       _ft_smooth_render          00431f85 f    CIL library: CIL module
 0001:00030fa7       _ft_smooth_render_lcd      00431fa7 f    CIL library: CIL module
 0001:00030fcd       _ft_smooth_render_lcd_v    00431fcd f    CIL library: CIL module
 0001:00030ff3       _cff_get_kerning           00431ff3 f    CIL library: CIL module
 0001:00030ff3       _tt_get_kerning            00431ff3 f    CIL library: CIL module
 0001:00031025       _tt_get_advances           00432025 f    CIL library: CIL module
 0001:000310c9       _tt_size_select            004320c9 f    CIL library: CIL module
 0001:00031112       _tt_size_request           00432112 f    CIL library: CIL module
 0001:00031174       _Load_Glyph                00432174 f    CIL library: CIL module
 0001:000311db       _tt_get_interface          004321db f    CIL library: CIL module
 0001:0003121e       _tt_face_load_loca         0043221e f    CIL library: CIL module
 0001:00031321       _tt_face_get_location      00432321 f    CIL library: CIL module
 0001:000313d1       _tt_face_load_cvt          004323d1 f    CIL library: CIL module
 0001:000314a0       _tt_face_load_fpgm         004324a0 f    CIL library: CIL module
 0001:000314ef       _tt_face_load_prep         004324ef f    CIL library: CIL module
 0001:0003153e       _tt_face_load_hdmx         0043253e f    CIL library: CIL module
 0001:0003168a       _tt_face_get_device_metrics 0043268a f    CIL library: CIL module
 0001:000316e1       _TT_Get_HMetrics           004326e1 f    CIL library: CIL module
 0001:00031717       _translate_array           00432717 f    CIL library: CIL module
 0001:00031741       _TT_Access_Glyph_Frame     00432741 f    CIL library: CIL module
 0001:0003177f       _TT_Forget_Glyph_Frame     0043277f f    CIL library: CIL module
 0001:0003178e       _TT_Load_Glyph_Header      0043278e f    CIL library: CIL module
 0001:00031811       _TT_Load_Simple_Glyph      00432811 f    CIL library: CIL module
 0001:00031b8c       _TT_Load_Composite_Glyph   00432b8c f    CIL library: CIL module
 0001:00031d93       _tt_prepare_zone           00432d93 f    CIL library: CIL module
 0001:00031ddf       _TT_Hint_Glyph             00432ddf f    CIL library: CIL module
 0001:00031fc7       _TT_Process_Simple_Glyph   00432fc7 f    CIL library: CIL module
 0001:000321d8       _TT_Process_Composite_Component 004331d8 f    CIL library: CIL module
 0001:00032342       _TT_Process_Composite_Glyph 00433342 f    CIL library: CIL module
 0001:000324e6       _load_truetype_glyph       004334e6 f    CIL library: CIL module
 0001:00032abc       _compute_glyph_metrics     00433abc f    CIL library: CIL module
 0001:00032c5d       _load_sbit_image           00433c5d f    CIL library: CIL module
 0001:00032d15       _tt_loader_init            00433d15 f    CIL library: CIL module
 0001:00032ea2       _TT_Load_Glyph             00433ea2 f    CIL library: CIL module
 0001:0003301c       _tt_glyphzone_done         0043401c f    CIL library: CIL module
 0001:0003307f       _tt_glyphzone_new          0043407f f    CIL library: CIL module
 0001:00033146       _tt_check_trickyness       00434146 f    CIL library: CIL module
 0001:00033186       _tt_face_init              00434186 f    CIL library: CIL module
 0001:000332b1       _tt_face_done              004342b1 f    CIL library: CIL module
 0001:00033385       _tt_size_run_fpgm          00434385 f    CIL library: CIL module
 0001:00033482       _tt_size_run_prep          00434482 f    CIL library: CIL module
 0001:00033546       _tt_size_done_bytecode     00434546 f    CIL library: CIL module
 0001:000335eb       _tt_size_init_bytecode     004345eb f    CIL library: CIL module
 0001:00033781       _tt_size_ready_bytecode    00434781 f    CIL library: CIL module
 0001:00033869       _tt_size_init              00434869 f    CIL library: CIL module
 0001:00033885       _tt_size_done              00434885 f    CIL library: CIL module
 0001:0003389e       _tt_size_reset             0043489e f    CIL library: CIL module
 0001:000339da       _tt_driver_init            004349da f    CIL library: CIL module
 0001:00033a33       _tt_driver_done            00434a33 f    CIL library: CIL module
 0001:00033a4c       _tt_slot_init              00434a4c f    CIL library: CIL module
 0001:00033a98       _TT_Goto_CodeRange         00434a98 f    CIL library: CIL module
 0001:00033ac2       _TT_Done_Context           00434ac2 f    CIL library: CIL module
 0001:00033b32       _Init_Context              00434b32 f    CIL library: CIL module
 0001:00033b9b       _Update_Max                00434b9b f    CIL library: CIL module
 0001:00033bd6       _TT_Load_Context           00434bd6 f    CIL library: CIL module
 0001:00033d7b       _TT_Save_Context           00434d7b f    CIL library: CIL module
 0001:00033dcf       _TT_Run_Context            00434dcf f    CIL library: CIL module
 0001:00033e5f       _TT_MulFix14               00434e5f f    CIL library: CIL module
 0001:00033eb3       _TT_DotFix14               00434eb3 f    CIL library: CIL module
 0001:00033f3f       _TT_VecLen                 00434f3f f    CIL library: CIL module
 0001:00033fa3       _Current_Ratio             00434fa3 f    CIL library: CIL module
 0001:00034018       _Current_Ppem              00435018 f    CIL library: CIL module
 0001:00034030       _Read_CVT                  00435030 f    CIL library: CIL module
 0001:00034042       _Read_CVT_Stretched        00435042 f    CIL library: CIL module
 0001:00034062       _Write_CVT                 00435062 f    CIL library: CIL module
 0001:00034078       _Write_CVT_Stretched       00435078 f    CIL library: CIL module
 0001:0003409c       _Move_CVT                  0043509c f    CIL library: CIL module
 0001:000340b4       _Move_CVT_Stretched        004350b4 f    CIL library: CIL module
 0001:000340dc       _Ins_Goto_CodeRange        004350dc f    CIL library: CIL module
 0001:00034133       _Direct_Move               00435133 f    CIL library: CIL module
 0001:000341b5       _Direct_Move_Orig          004351b5 f    CIL library: CIL module
 0001:0003421b       _Direct_Move_X             0043521b f    CIL library: CIL module
 0001:0003423b       _Direct_Move_Y             0043523b f    CIL library: CIL module
 0001:0003425c       _Direct_Move_Orig_X        0043525c f    CIL library: CIL module
 0001:00034272       _Direct_Move_Orig_Y        00435272 f    CIL library: CIL module
 0001:00034289       _Round_None                00435289 f    CIL library: CIL module
 0001:000342ae       _Round_To_Grid             004352ae f    CIL library: CIL module
 0001:000342d9       _Round_To_Half_Grid        004352d9 f    CIL library: CIL module
 0001:0003430c       _Round_Down_To_Grid        0043530c f    CIL library: CIL module
 0001:00034334       _Round_Up_To_Grid          00435334 f    CIL library: CIL module
 0001:0003435f       _Round_To_Double_Grid      0043535f f    CIL library: CIL module
 0001:0003438a       _Round_Super               0043538a f    CIL library: CIL module
 0001:000343d7       _Round_Super_45            004353d7 f    CIL library: CIL module
 0001:0003442c       _Compute_Round             0043542c f    CIL library: CIL module
 0001:000344b4       _SetSuperRound             004354b4 f    CIL library: CIL module
 0001:0003459a       _Project                   0043559a f    CIL library: CIL module
 0001:000345be       _Dual_Project              004355be f    CIL library: CIL module
 0001:000345e2       _Project_x                 004355e2 f    CIL library: CIL module
 0001:000345e7       _Project_y                 004355e7 f    CIL library: CIL module
 0001:000345ec       _Compute_Funcs             004355ec f    CIL library: CIL module
 0001:00034728       _Normalize                 00435728 f    CIL library: CIL module
 0001:00034845       _Ins_SxVTL                 00435845 f    CIL library: CIL module
 0001:0003489e       _Ins_MINDEX                0043589e f    CIL library: CIL module
 0001:000348df       _SkipCode                  004358df f    CIL library: CIL module
 0001:00034962       _Ins_FDEF                  00435962 f    CIL library: CIL module
 0001:000349f3       _Ins_ENDF                  004359f3 f    CIL library: CIL module
 0001:00034a35       _Ins_CALL                  00435a35 f    CIL library: CIL module
 0001:00034ae5       _Ins_LOOPCALL              00435ae5 f    CIL library: CIL module
 0001:00034ba0       _Ins_IDEF                  00435ba0 f    CIL library: CIL module
 0001:00034c39       _Ins_NPUSHB                00435c39 f    CIL library: CIL module
 0001:00034ca0       _Ins_NPUSHW                00435ca0 f    CIL library: CIL module
 0001:00034d22       _Ins_PUSHB                 00435d22 f    CIL library: CIL module
 0001:00034d74       _Ins_PUSHW                 00435d74 f    CIL library: CIL module
 0001:00034de7       _Ins_GC                    00435de7 f    CIL library: CIL module
 0001:00034e3b       _Ins_SCFS                  00435e3b f    CIL library: CIL module
 0001:00034eb1       _Ins_MD                    00435eb1 f    CIL library: CIL module
 0001:00034f91       _Ins_SDPVTL                00435f91 f    CIL library: CIL module
 0001:00035034       _Ins_SZP0                  00436034 f    CIL library: CIL module
 0001:00035075       _Ins_SZP1                  00436075 f    CIL library: CIL module
 0001:000350b6       _Ins_SZP2                  004360b6 f    CIL library: CIL module
 0001:000350f7       _Ins_SZPS                  004360f7 f    CIL library: CIL module
 0001:00035164       _Ins_SCANCTRL              00436164 f    CIL library: CIL module
 0001:00035210       _Ins_FLIPPT                00436210 f    CIL library: CIL module
 0001:00035268       _Ins_FLIPRGON              00436268 f    CIL library: CIL module
 0001:000352af       _Ins_FLIPRGOFF             004362af f    CIL library: CIL module
 0001:000352f6       _Compute_Point_Displacement 004362f6 f    CIL library: CIL module
 0001:000353b7       _Move_Zp2_Point            004363b7 f    CIL library: CIL module
 0001:00035413       _Ins_SHP                   00436413 f    CIL library: CIL module
 0001:00035493       _Ins_SHC                   00436493 f    CIL library: CIL module
 0001:00035561       _Ins_SHZ                   00436561 f    CIL library: CIL module
 0001:0003560f       _Ins_SHPIX                 0043660f f    CIL library: CIL module
 0001:000356b2       _Ins_MSIRP                 004366b2 f    CIL library: CIL module
 0001:000357ab       _Ins_MDAP                  004367ab f    CIL library: CIL module
 0001:00035820       _Ins_MIAP                  00436820 f    CIL library: CIL module
 0001:00035925       _Ins_MDRP                  00436925 f    CIL library: CIL module
 0001:00035af7       _Ins_MIRP                  00436af7 f    CIL library: CIL module
 0001:00035d08       _Ins_ALIGNRP               00436d08 f    CIL library: CIL module
 0001:00035db5       _Ins_ISECT                 00436db5 f    CIL library: CIL module
 0001:00035faa       _Ins_ALIGNPTS              00436faa f    CIL library: CIL module
 0001:0003602e       _Ins_IP                    0043702e f    CIL library: CIL module
 0001:000361e5       _Ins_UTP                   004371e5 f    CIL library: CIL module
 0001:00036226       __iup_worker_interpolate   00437226 f    CIL library: CIL module
 0001:0003634a       _Ins_IUP                   0043734a f    CIL library: CIL module
 0001:000364bc       _Ins_DELTAP                004374bc f    CIL library: CIL module
 0001:00036593       _Ins_DELTAC                00437593 f    CIL library: CIL module
 0001:00036667       _Ins_GETINFO               00437667 f    CIL library: CIL module
 0001:000366b0       _Ins_UNKNOWN               004376b0 f    CIL library: CIL module
 0001:000374ae       _ft_var_readpackedpoints   004384ae f    CIL library: CIL module
 0001:00037599       _ft_var_readpackeddeltas   00438599 f    CIL library: CIL module
 0001:0003766e       _ft_var_load_avar          0043866e f    CIL library: CIL module
 0001:000377c7       _ft_var_load_gvar          004387c7 f    CIL library: CIL module
 0001:000379c1       _ft_var_apply_tuple        004389c1 f    CIL library: CIL module
 0001:00037ab7       _TT_Get_MM_Var             00438ab7 f    CIL library: CIL module
 0001:00037e30       _TT_Set_MM_Blend           00438e30 f    CIL library: CIL module
 0001:00037f7e       _TT_Set_Var_Design         00438f7e f    CIL library: CIL module
 0001:0003812f       _tt_face_vary_cvt          0043912f f    CIL library: CIL module
 0001:00038455       _TT_Vary_Get_Glyph_Deltas  00439455 f    CIL library: CIL module
 0001:0003889a       _tt_done_blend             0043989a f    CIL library: CIL module
 0001:00038925       _read_pfb_tag              00439925 f    CIL library: CIL module
 0001:0003897b       _check_type1_format        0043997b f    CIL library: CIL module
 0001:000389f1       _T1_New_Parser             004399f1 f    CIL library: CIL module
 0001:00038b48       _T1_Get_Private_Dict       00439b48 f    CIL library: CIL module
 0001:00038e10       _t1_allocate_blend         00439e10 f    CIL library: CIL module
 0001:00038fe7       _T1_Get_Multi_Master       00439fe7 f    CIL library: CIL module
 0001:00039050       _mm_axis_unmap             0043a050 f    CIL library: CIL module
 0001:000390c1       _mm_weights_unmap          0043a0c1 f    CIL library: CIL module
 0001:0003919f       _T1_Get_MM_Var             0043a19f f    CIL library: CIL module
 0001:000393a6       _T1_Set_MM_Blend           0043a3a6 f    CIL library: CIL module
 0001:00039433       _T1_Set_MM_Design          0043a433 f    CIL library: CIL module
 0001:00039533       _T1_Set_Var_Design         0043a533 f    CIL library: CIL module
 0001:00039583       _T1_Done_Blend             0043a583 f    CIL library: CIL module
 0001:0003969c       _parse_blend_axis_types    0043a69c f    CIL library: CIL module
 0001:00039778       _parse_blend_design_positions 0043a778 f    CIL library: CIL module
 0001:000398b5       _parse_blend_design_map    0043a8b5 f    CIL library: CIL module
 0001:00039a12       _parse_weight_vector       0043aa12 f    CIL library: CIL module
 0001:00039af9       _parse_buildchar           0043aaf9 f    CIL library: CIL module
 0001:00039b14       _t1_load_keyword           0043ab14 f    CIL library: CIL module
 0001:00039bde       _parse_private             0043abde f    CIL library: CIL module
 0001:00039bea       _read_binary_data          0043abea f    CIL library: CIL module
 0001:00039c37       _parse_font_matrix         0043ac37 f    CIL library: CIL module
 0001:00039d1c       _parse_encoding            0043ad1c f    CIL library: CIL module
 0001:0003a06f       _parse_subrs               0043b06f f    CIL library: CIL module
 0001:0003a23a       _parse_charstrings         0043b23a f    CIL library: CIL module
 0001:0003a76d       _parse_dict                0043b76d f    CIL library: CIL module
 0001:0003aab0       _t1_done_loader            0043bab0 f    CIL library: CIL module
 0001:0003ab40       _T1_Open_Face              0043bb40 f    CIL library: CIL module
 0001:0003aef7       _T1_Size_Get_Globals_Funcs 0043bef7 f    CIL library: CIL module
 0001:0003af29       _T1_Size_Done              0043bf29 f    CIL library: CIL module
 0001:0003af4c       _T1_Size_Init              0043bf4c f    CIL library: CIL module
 0001:0003af89       _T1_Size_Request           0043bf89 f    CIL library: CIL module
 0001:0003afc2       _T1_GlyphSlot_Init         0043bfc2 f    CIL library: CIL module
 0001:0003affd       _T1_Face_Done              0043bffd f    CIL library: CIL module
 0001:0003b16d       _T1_Face_Init              0043c16d f    CIL library: CIL module
 0001:0003b4b2       _t42_get_glyph_name        0043c4b2 f    CIL library: CIL module
 0001:0003b4b2       _t1_get_glyph_name         0043c4b2 f    CIL library: CIL module
 0001:0003b4d4       _t1_get_name_index         0043c4d4 f    CIL library: CIL module
 0001:0003b528       _t1_ps_get_font_info       0043c528 f    CIL library: CIL module
 0001:0003b528       _t42_ps_get_font_info      0043c528 f    CIL library: CIL module
 0001:0003b542       _t42_ps_get_font_extra     0043c542 f    CIL library: CIL module
 0001:0003b542       _t1_ps_get_font_extra      0043c542 f    CIL library: CIL module
 0001:0003b557       _t1_ps_has_glyph_names     0043c557 f    CIL library: CIL module
 0001:0003b557       _t42_ps_has_glyph_names    0043c557 f    CIL library: CIL module
 0001:0003b55b       _t42_ps_get_font_private   0043c55b f    CIL library: CIL module
 0001:0003b55b       _t1_ps_get_font_private    0043c55b f    CIL library: CIL module
 0001:0003b575       _Get_Interface             0043c575 f    CIL library: CIL module
 0001:0003b585       _Get_Kerning               0043c585 f    CIL library: CIL module
 0001:0003b5b1       _T1_Parse_Glyph_And_Get_Char_String 0043c5b1 f    CIL library: CIL module
 0001:0003b610       _T1_Parse_Glyph            0043c610 f    CIL library: CIL module
 0001:0003b628       _T1_Compute_Max_Advance    0043c628 f    CIL library: CIL module
 0001:0003b702       _T1_Get_Advances           0043c702 f    CIL library: CIL module
 0001:0003b7e2       _T1_Load_Glyph             0043c7e2 f    CIL library: CIL module
 0001:0003bb63       _T1_Done_Metrics           0043cb63 f    CIL library: CIL module
 0001:0003bb99       _t1_get_index              0043cb99 f    CIL library: CIL module
 0001:0003bbfc       _T1_Read_PFM               0043cbfc f    CIL library: CIL module
 0001:0003bd90       _T1_Read_Metrics           0043cd90 f    CIL library: CIL module
 0001:0003bf42       _T1_Get_Kerning            0043cf42 f    CIL library: CIL module
 0001:0003bf9e       _T1_Get_Track_Kerning      0043cf9e f    CIL library: CIL module
 0001:0003c020       _T42_Open_Face             0043d020 f    CIL library: CIL module
 0001:0003c282       _T42_Face_Init             0043d282 f    CIL library: CIL module
 0001:0003c7a1       _T42_Face_Done             0043d7a1 f    CIL library: CIL module
 0001:0003c8f8       _T42_Driver_Init           0043d8f8 f    CIL library: CIL module
 0001:0003c914       _T42_Size_Init             0043d914 f    CIL library: CIL module
 0001:0003c941       _T42_Size_Request          0043d941 f    CIL library: CIL module
 0001:0003c97b       _T42_Size_Select           0043d97b f    CIL library: CIL module
 0001:0003c9b3       _T42_Size_Done             0043d9b3 f    CIL library: CIL module
 0001:0003c9de       _T42_GlyphSlot_Init        0043d9de f    CIL library: CIL module
 0001:0003ca18       _T42_GlyphSlot_Done        0043da18 f    CIL library: CIL module
 0001:0003ca27       _T42_GlyphSlot_Load        0043da27 f    CIL library: CIL module
 0001:0003cb31       _t42_parser_init           0043db31 f    CIL library: CIL module
 0001:0003cc3c       _t42_is_space              0043dc3c f    CIL library: CIL module
 0001:0003cc5b       _t42_parse_font_matrix     0043dc5b f    CIL library: CIL module
 0001:0003cd22       _t42_parse_encoding        0043dd22 f    CIL library: CIL module
 0001:0003cfdd       _t42_parse_sfnts           0043dfdd f    CIL library: CIL module
 0001:0003d2a8       _t42_parse_charstrings     0043e2a8 f    CIL library: CIL module
 0001:0003d655       _t42_load_keyword          0043e655 f    CIL library: CIL module
 0001:0003d6b9       _t42_parse_dict            0043e6b9 f    CIL library: CIL module
 0001:0003d834       _t42_loader_done           0043e834 f    CIL library: CIL module
 0001:0003d89d       _t42_get_name_index        0043e89d f    CIL library: CIL module
 0001:0003d91b       _t1_get_ps_name            0043e91b f    CIL library: CIL module
 0001:0003d91b       _t42_get_ps_font_name      0043e91b f    CIL library: CIL module
 0001:0003d926       _T42_Get_Interface         0043e926 f    CIL library: CIL module
 0001:0003d936       _fnt_font_done             0043e936 f    CIL library: CIL module
 0001:0003d988       _fnt_font_load             0043e988 f    CIL library: CIL module
 0001:0003da2e       _fnt_face_get_dll_font     0043ea2e f    CIL library: CIL module
 0001:0003e035       _fnt_cmap_init             0043f035 f    CIL library: CIL module
 0001:0003e055       _fnt_cmap_char_index       0043f055 f    CIL library: CIL module
 0001:0003e06b       _fnt_cmap_char_next        0043f06b f    CIL library: CIL module
 0001:0003e09c       _FNT_Face_Done             0043f09c f    CIL library: CIL module
 0001:0003e0c4       _FNT_Face_Init             0043f0c4 f    CIL library: CIL module
 0001:0003e37b       _FNT_Size_Select           0043f37b f    CIL library: CIL module
 0001:0003e3bc       _FNT_Size_Request          0043f3bc f    CIL library: CIL module
 0001:0003e431       _FNT_Load_Glyph            0043f431 f    CIL library: CIL module
 0001:0003e5d8       _winfnt_get_header         0043f5d8 f    CIL library: CIL module
 0001:0003e5f5       _winfnt_get_service        0043f5f5 f    CIL library: CIL module
 0001:0003e76f       _default_decompress_parms  0043f76f f    CIL library: CIL module
 0001:0003eb5b       _output_pass_setup         0043fb5b f    CIL library: CIL module
 0001:0003ec83       _start_iMCU_row            0043fc83 f    CIL library: CIL module
 0001:0003ecc2       _start_input_pass          0043fcc2 f    CIL library: CIL module
 0001:0003ecd2       _start_output_pass         0043fcd2 f    CIL library: CIL module
 0001:0003ed0d       _decompress_onepass        0043fd0d f    CIL library: CIL module
 0001:0003eee9       _consume_data              0043fee9 f    CIL library: CIL module
 0001:0003f088       _decompress_data           00440088 f    CIL library: CIL module
 0001:0003f1ee       _smoothing_ok              004401ee f    CIL library: CIL module
 0001:0003f2ce       _decompress_smooth_data    004402ce f    CIL library: CIL module
 0001:0003f937       _build_ycc_rgb_table       00440937 f    CIL library: CIL module
 0001:0003f9e7       _ycc_rgb_convert           004409e7 f    CIL library: CIL module
 0001:0003faee       _null_convert              00440aee f    CIL library: CIL module
 0001:0003fb54       _grayscale_convert         00440b54 f    CIL library: CIL module
 0001:0003fb77       _gray_rgb_convert          00440b77 f    CIL library: CIL module
 0001:0003fbc9       _ycck_cmyk_convert         00440bc9 f    CIL library: CIL module
 0001:0003fe21       _start_pass                00440e21 f    CIL library: CIL module
 0001:00040049       _start_pass_huff_decoder   00441049 f    CIL library: CIL module
 0001:00040600       _process_restart           00441600 f    CIL library: CIL module
 0001:00040663       _decode_mcu                00441663 f    CIL library: CIL module
 0001:00040a29       _initial_setup             00441a29 f    CIL library: CIL module
 0001:00040bfe       _per_scan_setup            00441bfe f    CIL library: CIL module
 0001:00040d73       _latch_quant_tables        00441d73 f    CIL library: CIL module
 0001:00040e01       _start_input_pass          00441e01 f    CIL library: CIL module
 0001:00040e3b       _finish_input_pass         00441e3b f    CIL library: CIL module
 0001:00040e4c       _consume_markers           00441e4c f    CIL library: CIL module
 0001:00040edf       _reset_input_controller    00441edf f    CIL library: CIL module
 0001:00040f16       _alloc_funny_pointers      00441f16 f    CIL library: CIL module
 0001:00040fbe       _make_funny_pointers       00441fbe f    CIL library: CIL module
 0001:000410ed       _set_wraparound_pointers   004420ed f    CIL library: CIL module
 0001:000411c1       _set_bottom_pointers       004421c1 f    CIL library: CIL module
 0001:00041257       _start_pass_main           00442257 f    CIL library: CIL module
 0001:000412bf       _process_data_simple_main  004422bf f    CIL library: CIL module
 0001:00041327       _process_data_context_main 00442327 f    CIL library: CIL module
 0001:0004142f       _process_data_crank_post   0044242f f    CIL library: CIL module
 0001:00041511       _get_soi                   00442511 f    CIL library: CIL module
 0001:000415ad       _get_sof                   004425ad f    CIL library: CIL module
 0001:0004189d       _get_sos                   0044289d f    CIL library: CIL module
 0001:00041b52       _get_dht                   00442b52 f    CIL library: CIL module
 0001:00041e4a       _get_dqt                   00442e4a f    CIL library: CIL module
 0001:0004207b       _get_dri                   0044307b f    CIL library: CIL module
 0001:00042155       _examine_app0              00443155 f    CIL library: CIL module
 0001:0004233a       _examine_app14             0044333a f    CIL library: CIL module
 0001:000423ea       _get_interesting_appn      004433ea f    CIL library: CIL module
 0001:0004253b       _skip_variable             0044353b f    CIL library: CIL module
 0001:000425de       _next_marker               004435de f    CIL library: CIL module
 0001:000426b5       _first_marker              004436b5 f    CIL library: CIL module
 0001:0004274c       _read_markers              0044374c f    CIL library: CIL module
 0001:00042949       _read_restart_marker       00443949 f    CIL library: CIL module
 0001:00042a9a       _reset_marker_reader       00443a9a f    CIL library: CIL module
 0001:00042ac5       _use_merged_upsample       00443ac5 f    CIL library: CIL module
 0001:00042d2d       _prepare_range_limit_table 00443d2d f    CIL library: CIL module
 0001:00042dab       _master_selection          00443dab f    CIL library: CIL module
 0001:00042f54       _prepare_for_output_pass   00443f54 f    CIL library: CIL module
 0001:00043080       _finish_output_pass        00444080 f    CIL library: CIL module
 0001:000430a1       _build_ycc_rgb_table       004440a1 f    CIL library: CIL module
 0001:00043151       _start_pass_merged_upsample 00444151 f    CIL library: CIL module
 0001:00043166       _merged_2v_upsample        00444166 f    CIL library: CIL module
 0001:0004320c       _merged_1v_upsample        0044420c f    CIL library: CIL module
 0001:0004323d       _h2v1_merged_upsample      0044423d f    CIL library: CIL module
 0001:00043393       _h2v2_merged_upsample      00444393 f    CIL library: CIL module
 0001:000435e8       _start_pass_phuff_decoder  004445e8 f    CIL library: CIL module
 0001:0004381d       _process_restart           0044481d f    CIL library: CIL module
 0001:00043883       _decode_mcu_DC_first       00444883 f    CIL library: CIL module
 0001:00043a6f       _decode_mcu_AC_first       00444a6f f    CIL library: CIL module
 0001:00043c83       _decode_mcu_DC_refine      00444c83 f    CIL library: CIL module
 0001:00043d57       _decode_mcu_AC_refine      00444d57 f    CIL library: CIL module
 0001:00044112       _start_pass_dpost          00445112 f    CIL library: CIL module
 0001:000441b8       _post_process_1pass        004451b8 f    CIL library: CIL module
 0001:0004421d       _post_process_prepass      0044521d f    CIL library: CIL module
 0001:000442ad       _post_process_2pass        004452ad f    CIL library: CIL module
 0001:000443c0       _start_pass_upsample       004453c0 f    CIL library: CIL module
 0001:000443da       _sep_upsample              004453da f    CIL library: CIL module
 0001:000444a0       _fullsize_upsample         004454a0 f    CIL library: CIL module
 0001:000444ab       _noop_upsample             004454ab f    CIL library: CIL module
 0001:000444b3       _int_upsample              004454b3 f    CIL library: CIL module
 0001:00044570       _h2v1_upsample             00445570 f    CIL library: CIL module
 0001:000445c7       _h2v2_upsample             004455c7 f    CIL library: CIL module
 0001:00044634       _h2v1_fancy_upsample       00445634 f    CIL library: CIL module
 0001:000446e3       _h2v2_fancy_upsample       004456e3 f    CIL library: CIL module
 0001:000449b1       _error_exit                004459b1 f    CIL library: CIL module
 0001:000449ca       _output_message            004459ca f    CIL library: CIL module
 0001:00044a18       _emit_message              00445a18 f    CIL library: CIL module
 0001:00044a49       _format_message            00445a49 f    CIL library: CIL module
 0001:00044ae0       _reset_error_mgr           00445ae0 f    CIL library: CIL module
 0001:00045cdf       _select_ncolors            00446cdf f    CIL library: CIL module
 0001:00045daa       _create_colormap           00446daa f    CIL library: CIL module
 0001:00045ed7       _create_colorindex         00446ed7 f    CIL library: CIL module
 0001:00046002       _create_odither_tables     00447002 f    CIL library: CIL module
 0001:000460c7       _color_quantize            004470c7 f    CIL library: CIL module
 0001:0004614f       _color_quantize3           0044714f f    CIL library: CIL module
 0001:000461dc       _quantize_ord_dither       004471dc f    CIL library: CIL module
 0001:000462cb       _quantize3_ord_dither      004472cb f    CIL library: CIL module
 0001:000463ca       _quantize_fs_dither        004473ca f    CIL library: CIL module
 0001:0004654e       _alloc_fs_workspace        0044754e f    CIL library: CIL module
 0001:00046584       _start_pass_1_quant        00447584 f    CIL library: CIL module
 0001:00046651       _new_color_map_1_quant     00447651 f    CIL library: CIL module
 0001:000466ea       _prescan_quantize          004476ea f    CIL library: CIL module
 0001:00046754       _update_box                00447754 f    CIL library: CIL module
 0001:00046a8d       _median_cut                00447a8d f    CIL library: CIL module
 0001:00046bd7       _compute_color             00447bd7 f    CIL library: CIL module
 0001:00046d0f       _select_colors             00447d0f f    CIL library: CIL module
 0001:00046d98       _find_nearby_colors        00447d98 f    CIL library: CIL module
 0001:00046f24       _find_best_colors          00447f24 f    CIL library: CIL module
 0001:00047037       _fill_inverse_cmap         00448037 f    CIL library: CIL module
 0001:00047144       _pass2_no_dither           00448144 f    CIL library: CIL module
 0001:000471ed       _pass2_fs_dither           004481ed f    CIL library: CIL module
 0001:0004745d       _init_error_limit          0044845d f    CIL library: CIL module
 0001:000474e9       _finish_pass1              004484e9 f    CIL library: CIL module
 0001:00047509       _start_pass_2_quant        00448509 f    CIL library: CIL module
 0001:0004760f       _new_color_map_2_quant     0044860f f    CIL library: CIL module
 0001:0004775e       _out_of_memory             0044875e f    CIL library: CIL module
 0001:00047773       _alloc_small               00448773 f    CIL library: CIL module
 0001:0004786b       _alloc_large               0044886b f    CIL library: CIL module
 0001:000478f7       _alloc_sarray              004488f7 f    CIL library: CIL module
 0001:00047989       _alloc_barray              00448989 f    CIL library: CIL module
 0001:00047a27       _request_virt_sarray       00448a27 f    CIL library: CIL module
 0001:00047a88       _request_virt_barray       00448a88 f    CIL library: CIL module
 0001:00047ae9       _realize_virt_arrays       00448ae9 f    CIL library: CIL module
 0001:00047c31       _do_sarray_io              00448c31 f    CIL library: CIL module
 0001:00047cb9       _do_barray_io              00448cb9 f    CIL library: CIL module
 0001:00047d44       _access_virt_sarray        00448d44 f    CIL library: CIL module
 0001:00047e65       _access_virt_barray        00448e65 f    CIL library: CIL module
 0001:00047f8b       _free_pool                 00448f8b f    CIL library: CIL module
 0001:00048060       _self_destruct             00449060 f    CIL library: CIL module
 0001:00048186       _ft_alloc                  00449186 f    CIL library: CIL module
 0001:00048186       _jbig2_default_alloc       00449186 f    CIL library: CIL module
 0001:00048191       _jbig2_default_realloc     00449191 f    CIL library: CIL module
 0001:000481a1       _jbig2_default_error       004491a1 f    CIL library: CIL module
 0001:000486fe       _jbig2_word_stream_buf_get_next_word 004496fe f    CIL library: CIL module
 0001:0004877c       _jbig2_arith_bytein        0044977c f    CIL library: CIL module
 0001:0004887b       _jbig2_arith_renormd       0044987b f    CIL library: CIL module
 0001:00049005       _jbig2_decode_generic_template0 0044a005 f    CIL library: CIL module
 0001:000491ac       _jbig2_decode_generic_template0_unopt 0044a1ac f    CIL library: CIL module
 0001:0004937d       _jbig2_decode_generic_template1 0044a37d f    CIL library: CIL module
 0001:00049526       _jbig2_decode_generic_template2 0044a526 f    CIL library: CIL module
 0001:000496d0       _jbig2_decode_generic_template2a 0044a6d0 f    CIL library: CIL module
 0001:00049897       _jbig2_decode_generic_template3_unopt 0044a897 f    CIL library: CIL module
 0001:00049d1c       _jbig2_decode_refinement_template0_unopt 0044ad1c f    CIL library: CIL module
 0001:00049ee2       _jbig2_decode_refinement_template1_unopt 0044aee2 f    CIL library: CIL module
 0001:0004b0e0       _jbig2_decode_symbol_dict  0044c0e0 f    CIL library: CIL module
 0001:0004d0dc       _jbig2_decode_mmr_consume  0044e0dc f    CIL library: CIL module
 0001:0004d119       _jbig2_set_bits            0044e119 f    CIL library: CIL module
 0001:0004d173       _jbig2_decode_get_run      0044e173 f    CIL library: CIL module
 0001:0004d1df       _jbig2_decode_mmr_line     0044e1df f    CIL library: CIL module
 0001:0004d605       _dump_page_info            0044e605 f    CIL library: CIL module
 0001:0004db34       _jbig2_strndup             0044eb34 f    CIL library: CIL module
 0001:0004dd24       _srown                     0044ed24 f    CIL library: CIL module
 0001:0004ddce       _srowc                     0044edce f    CIL library: CIL module
 0001:0004df25       _srow1                     0044ef25 f    CIL library: CIL module
 0001:0004df40       _srow2                     0044ef40 f    CIL library: CIL module
 0001:0004df5b       _srow4                     0044ef5b f    CIL library: CIL module
 0001:0004df76       _srow5                     0044ef76 f    CIL library: CIL module
 0001:0004df91       _scoln                     0044ef91 f    CIL library: CIL module
 0001:0004e028       _scol1                     0044f028 f    CIL library: CIL module
 0001:0004e043       _scol2                     0044f043 f    CIL library: CIL module
 0001:0004e05e       _scol4                     0044f05e f    CIL library: CIL module
 0001:0004e079       _scol5                     0044f079 f    CIL library: CIL module
 0001:0004e678       _line                      0044f678 f    CIL library: CIL module
 0001:0004e6f7       _bezier                    0044f6f7 f    CIL library: CIL module
 0001:0004ebe5       _hashkey                   0044fbe5 f    CIL library: CIL module
 0001:0004ed2d       _hashinsert                0044fd2d f    CIL library: CIL module
 0001:0004ed95       _bubble                    0044fd95 f    CIL library: CIL module
 0001:0004edf1       _evictall                  0044fdf1 f    CIL library: CIL module
 0001:0004f0f7       _decodetile                004500f7 f    CIL library: CIL module
 0001:0004f295       _init1                     00450295 f    CIL library: CIL module
 0001:0004f306       _loadtile1                 00450306 f    CIL library: CIL module
 0001:0004f462       _loadtile2                 00450462 f    CIL library: CIL module
 0001:0004f516       _loadtile4                 00450516 f    CIL library: CIL module
 0001:0004f5ca       _loadtile8                 004505ca f    CIL library: CIL module
 0001:0004f733       _cliplerpx                 00450733 f    CIL library: CIL module
 0001:0004fb1a       _sortael                   00450b1a f    CIL library: CIL module
 0001:0004fbab       _insertael                 00450bab f    CIL library: CIL module
 0001:0004fc3d       _addspan                   00450c3d f    CIL library: CIL module
 0001:0004fc95       _nonzerowinding            00450c95 f    CIL library: CIL module
 0001:0004fcf3       _evenodd                   00450cf3 f    CIL library: CIL module
 0001:0004fd49       _blit                      00450d49 f    CIL library: CIL module
 0001:0004ffe5       _duff_non                  00450fe5 f    CIL library: CIL module
 0001:0005005c       _duff_nimcn                0045105c f    CIL library: CIL module
 0001:000500d7       _duff_nimon                004510d7 f    CIL library: CIL module
 0001:0005018e       _text_1o1                  0045118e f    CIL library: CIL module
 0001:0005018e       _duff_1o1                  0045118e f    CIL library: CIL module
 0001:000501e4       _duff_4o4                  004511e4 f    CIL library: CIL module
 0001:00050284       _duff_1i1c1                00451284 f    CIL library: CIL module
 0001:000502e2       _duff_4i1c4                004512e2 f    CIL library: CIL module
 0001:00050376       _duff_1i1o1                00451376 f    CIL library: CIL module
 0001:000503ea       _duff_4i1o4                004513ea f    CIL library: CIL module
 0001:000504dd       _path_1c1                  004514dd f    CIL library: CIL module
 0001:00050503       _path_1o1                  00451503 f    CIL library: CIL module
 0001:00050543       _path_w4i1o4               00451543 f    CIL library: CIL module
 0001:00050606       _text_w4i1o4               00451606 f    CIL library: CIL module
 0001:000506fe       _getmask                   004516fe f    CIL library: CIL module
 0001:00050723       _samplemask                00451723 f    CIL library: CIL module
 0001:000507cf       _lerpargb                  004517cf f    CIL library: CIL module
 0001:00050833       _getargb                   00451833 f    CIL library: CIL module
 0001:0005085a       _sampleargb                0045185a f    CIL library: CIL module
 0001:0005090a       _img_1c1                   0045190a f    CIL library: CIL module
 0001:0005096e       _img_4c4                   0045196e f    CIL library: CIL module
 0001:000509d3       _img_1o1                   004519d3 f    CIL library: CIL module
 0001:00050a4c       _img_4o4                   00451a4c f    CIL library: CIL module
 0001:00050b11       _img_w4i1o4                00451b11 f    CIL library: CIL module
 0001:00050c3c       _clipx                     00451c3c f    CIL library: CIL module
 0001:00050d24       _clipy                     00451d24 f    CIL library: CIL module
 0001:00050e0f       _copyvert                  00451e0f f    CIL library: CIL module
 0001:00050e27       _clippoly                  00451e27 f    CIL library: CIL module
 0001:00050f2b       _drawscan                  00451f2b f    CIL library: CIL module
 0001:00050fd9       _findnext                  00451fd9 f    CIL library: CIL module
 0001:00051040       _loadedge                  00452040 f    CIL library: CIL module
 0001:000510b6       _fz_drawtriangle           004520b6 f    CIL library: CIL module
 0001:00051892       _line                      00452892 f    CIL library: CIL module
 0001:00051912       _arc                       00452912 f    CIL library: CIL module
 0001:00051ac5       _linestroke                00452ac5 f    CIL library: CIL module
 0001:00051bb0       _linejoin                  00452bb0 f    CIL library: CIL module
 0001:000520bf       _linecap                   004530bf f    CIL library: CIL module
 0001:0005237a       _linedot                   0045337a f    CIL library: CIL module
 0001:00052494       _strokeflush               00453494 f    CIL library: CIL module
 0001:000524ea       _strokemoveto              004534ea f    CIL library: CIL module
 0001:00052517       _strokelineto              00453517 f    CIL library: CIL module
 0001:000525d3       _strokeclosepath           004535d3 f    CIL library: CIL module
 0001:00052664       _strokebezier              00453664 f    CIL library: CIL module
 0001:00052a34       _dashmoveto                00453a34 f    CIL library: CIL module
 0001:00052aba       _dashlineto                00453aba f    CIL library: CIL module
 0001:00052bd2       _dashbezier                00453bd2 f    CIL library: CIL module
 0001:0005315b       _rendertransform           0045415b f    CIL library: CIL module
 0001:000531a3       _rendersolid               004541a3 f    CIL library: CIL module
 0001:000532ef       _renderpath                004542ef f    CIL library: CIL module
 0001:00053518       _drawglyph                 00454518 f    CIL library: CIL module
 0001:00053644       _rendertext                00454644 f    CIL library: CIL module
 0001:0005381d       _calcimagescale            0045481d f    CIL library: CIL module
 0001:000538e7       _renderimage               004548e7 f    CIL library: CIL module
 0001:00053e6d       _rendershade               00454e6d f    CIL library: CIL module
 0001:00053f11       _blendover                 00454f11 f    CIL library: CIL module
 0001:0005403a       _blendmask                 0045503a f    CIL library: CIL module
 0001:000542a6       _renderover                004552a6 f    CIL library: CIL module
 0001:00054367       _rendermask                00455367 f    CIL library: CIL module
 0001:000546ff       _rendernode                004556ff f    CIL library: CIL module
 0001:00054b0c       _hash                      00455b0c f    CIL library: CIL module
 0001:00055cc3       _iswhitenode               00456cc3 f    CIL library: CIL module
 0001:00055dee       _cleanwhite                00456dee f    CIL library: CIL module
 0001:00055e6a       _cleanovers                00456e6a f    CIL library: CIL module
 0001:00055ef8       _getrect                   00456ef8 f    CIL library: CIL module
 0001:00055ff9       _fitsinside                00456ff9 f    CIL library: CIL module
 0001:000560a1       _cleanmasks                004570a1 f    CIL library: CIL module
 0001:000562cc       _growpath                  004572cc f    CIL library: CIL module
 0001:0005656a       _boundexpand               0045756a f    CIL library: CIL module
 0001:00056e21       _fz_newfont                00457e21 f    CIL library: CIL module
 0001:00056f52       _fz_initfreetype           00457f52 f    CIL library: CIL module
 0001:000576e4       _setup_mix                 004586e4 f    CIL library: CIL module
 0001:00057731       _setup_mix2                00458731 f    CIL library: CIL module
 0001:00058205       _encode                    00459205 f    CIL library: CIL module
 0001:00058236       _transform                 00459236 f    CIL library: CIL module
 0001:00058dd9       _ishex                     00459dd9 f    CIL library: CIL module
 0001:00058dfc       _fromhex                   00459dfc f    CIL library: CIL module
 0001:00059030       _findchanging              0045a030 f    CIL library: CIL module
 0001:00059030       _jbig2_find_changing_element 0045a030 f    CIL library: CIL module
 0001:00059089       _jbig2_find_changing_element_of_color 0045a089 f    CIL library: CIL module
 0001:00059089       _findchangingcolor         0045a089 f    CIL library: CIL module
 0001:000590c9       _setbits                   0045a0c9 f    CIL library: CIL module
 0001:00059343       _getcode                   0045a343 f    CIL library: CIL module
 0001:00059396       _dec1d                     0045a396 f    CIL library: CIL module
 0001:00059453       _dec2d                     0045a453 f    CIL library: CIL module
 0001:000599e7       _zmalloc                   0045a9e7 f    CIL library: CIL module
 0001:00059d39       _unstuff                   0045ad39 f    CIL library: CIL module
 0001:0005a3df       _getcomponent              0045b3df f    CIL library: CIL module
 0001:0005a46c       _putcomponent              0045b46c f    CIL library: CIL module
 0001:0005a4ee       _paeth                     0045b4ee f    CIL library: CIL module
 0001:0005a52b       _tiff                      0045b52b f    CIL library: CIL module
 0001:0005a5c9       _png                       0045b5c9 f    CIL library: CIL module
 0001:0005a8fb       _Horizontal_Sweep_Init     0045b8fb f    CIL library: CIL module
 0001:0005a8fb       _Horizontal_Sweep_Step     0045b8fb f    CIL library: CIL module
 0001:0005a8fb       _cid_driver_done           0045b8fb f    CIL library: CIL module
 0001:0005a8fb       _ft_black_set_mode         0045b8fb f    CIL library: CIL module
 0001:0005a8fb       _start_pass_dcolor         0045b8fb f    CIL library: CIL module
 0001:0005a8fb       _cff_driver_done           0045b8fb f    CIL library: CIL module
 0001:0005a8fb       _tt_face_free_hdmx_stub    0045b8fb f    CIL library: CIL module
 0001:0005a8fb       _tt_face_free_sbit_stub    0045b8fb f    CIL library: CIL module
 0001:0005a8fb       _T42_Driver_Done           0045b8fb f    CIL library: CIL module
 0001:0005a8fb       _gxv_just_classTable_entry_validate 0045b8fb f    CIL library: CIL module
 0001:0005a8fb       _mytermsource              0045b8fb f    CIL library: CIL module
 0001:0005a8fb       _myinitsource              0045b8fb f    CIL library: CIL module
 0001:0005a8fb       _T1_Driver_Done            0045b8fb f    CIL library: CIL module
 0001:0005a8fb       _finish_pass_1_quant       0045b8fb f    CIL library: CIL module
 0001:0005a8fb       _finish_pass2              0045b8fb f    CIL library: CIL module
 0001:0005a8fb       _ps_parser_done            0045b8fb f    CIL library: CIL module
 0001:0005a8fb       _fz_opj_info_callback      0045b8fb f    CIL library: CIL module
 0001:0005aaa1       _growarray                 0045baa1 f    CIL library: CIL module
 0001:0005aba7       _keystrcmp                 0045bba7 f    CIL library: CIL module
 0001:0005ac93       _growdict                  0045bc93 f    CIL library: CIL module
 0001:0005ada0       _dictfinds                 0045bda0 f    CIL library: CIL module
 0001:0005b0b8       _fromhex                   0045c0b8 f    CIL library: CIL module
 0001:0005b0ee       _parsename                 0045c0ee f    CIL library: CIL module
 0001:0005b168       _parsenumber               0045c168 f    CIL library: CIL module
 0001:0005b20d       _parsedict                 0045c20d f    CIL library: CIL module
 0001:0005b3f3       _parsearray                0045c3f3 f    CIL library: CIL module
 0001:0005b4f2       _parsestring               0045c4f2 f    CIL library: CIL module
 0001:0005b62e       _parsehexstring            0045c62e f    CIL library: CIL module
 0001:0005b714       _parseobj                  0045c714 f    CIL library: CIL module
 0001:0005c583       _fz_fillbuf                0045d583 f    CIL library: CIL module
 0001:0005c6a2       _newstm                    0045d6a2 f    CIL library: CIL module
 0001:0005ce23       _myerrexit                 0045de23 f    CIL library: CIL module
 0001:0005ce70       _myoutmess                 0045de70 f    CIL library: CIL module
 0001:0005ceb3       _myfillinput               0045deb3 f    CIL library: CIL module
 0001:0005ceb6       _myskipinput               0045deb6 f    CIL library: CIL module
 0001:0005d431       _fz_opj_error_callback     0045e431 f    CIL library: CIL module
 0001:0005d44c       _fz_opj_warning_callback   0045e44c f    CIL library: CIL module
 0001:0005d90d       _resolvedest               0045e90d f    CIL library: CIL module
 0001:0005de22       _pdf_newovernode           0045ee22 f    CIL library: CIL module
 0001:0005e291       _addcolorshape             0045f291 f    CIL library: CIL module
 0001:0005e330       _addinvisibleshape         0045f330 f    CIL library: CIL module
 0001:0005e3cf       _getmatrix                 0045f3cf f    CIL library: CIL module
 0001:0005e44d       _addpatternshape           0045f44d f    CIL library: CIL module
 0001:0005e810       _addshadeshape             0045f810 f    CIL library: CIL module
 0001:0005f167       _showglyph                 00460167 f    CIL library: CIL module
 0001:0005f4c6       _showspace                 004604c6 f    CIL library: CIL module
 0001:0005f7fc       _addtable                  004607fc f    CIL library: CIL module
 0001:0005f87a       _addrange                  0046087a f    CIL library: CIL module
 0001:0005fa69       _cmprange                  00460a69 f    CIL library: CIL module
 0001:0005fa69       _cmpv                      00460a69 f    CIL library: CIL module
 0001:0005fa69       _cmph                      00460a69 f    CIL library: CIL module
 0001:0005fde2       _initcs                    00460de2 f    CIL library: CIL module
 0001:0005fe20       _graytoxyz                 00460e20 f    CIL library: CIL module
 0001:0005fe62       _xyztogray                 00460e62 f    CIL library: CIL module
 0001:0005fedc       _rgbtoxyz                  00460edc f    CIL library: CIL module
 0001:0005ff6b       _xyztorgb                  00460f6b f    CIL library: CIL module
 0001:00060016       _devicecmyktoxyz           00461016 f    CIL library: CIL module
 0001:00060086       _xyztodevicecmyk           00461086 f    CIL library: CIL module
 0001:0006012b       _fung                      0046112b f    CIL library: CIL module
 0001:00060162       _invg                      00461162 f    CIL library: CIL module
 0001:0006019f       _labtoxyz                  0046119f f    CIL library: CIL module
 0001:000602cd       _xyztolab                  004612cd f    CIL library: CIL module
 0001:000603b5       _loadiccbased              004613b5 f    CIL library: CIL module
 0001:0006041c       _separationtoxyz           0046141c f    CIL library: CIL module
 0001:0006048e       _dropseparation            0046148e f    CIL library: CIL module
 0001:000604a8       _loadseparation            004614a8 f    CIL library: CIL module
 0001:0006060b       _dropindexed               0046160b f    CIL library: CIL module
 0001:0006062e       _loadindexed               0046162e f    CIL library: CIL module
 0001:00060f10       _fastrgbtogray             00461f10 f    CIL library: CIL module
 0001:00060f5b       _fastrgbtocmyk             00461f5b f    CIL library: CIL module
 0001:00060fee       _fastcmyktogray            00461fee f    CIL library: CIL module
 0001:0006106d       _fastcmyktorgb             0046206d f    CIL library: CIL module
 0001:000613f9       _voodoo50                  004623f9 f    CIL library: CIL module
 0001:0006143f       _voodoo19                  0046243f f    CIL library: CIL module
 0001:000614ba       _padpassword               004624ba f    CIL library: CIL module
 0001:000614ec       _pdf_parsecryptfilt        004624ec f    CIL library: CIL module
 0001:00061599       _pdf_parseencdict          00462599 f    CIL library: CIL module
 0001:0006182d       _algofromname              0046282d f    CIL library: CIL module
 0001:00061bc3       _createobjkey              00462bc3 f    CIL library: CIL module
 0001:00061c5b       _createkey                 00462c5b f    CIL library: CIL module
 0001:00061d4a       _createuser                00462d4a f    CIL library: CIL module
 0001:000622c1       _pdflog                    004632c1 f    CIL library: CIL module
 0001:000624da       _ftkind                    004634da f    CIL library: CIL module
 0001:000625d5       _ftcharindex               004635d5 f    CIL library: CIL module
 0001:000625fa       _ftcidtogid                004635fa f    CIL library: CIL module
 0001:00062626       _cleanfontname             00463626 f    CIL library: CIL module
 0001:00062796       _loadsimplefont            00463796 f    CIL library: CIL module
 0001:000631af       _loadcidfont               004641af f    CIL library: CIL module
 0001:00063cfa       _loadtype0                 00464cfa f    CIL library: CIL module
 0001:0006482c       _fz_readbyte               0046582c f    CIL library: CIL module
 0001:0006482c       _fz_readbyte               0046582c f    CIL library: CIL module
 0001:0006482c       _fz_readbyte               0046582c f    CIL library: CIL module
 0001:0006482c       _fz_readbyte               0046582c f    CIL library: CIL module
 0001:0006482c       _fz_readbyte               0046582c f    CIL library: CIL module
 0001:0006482c       _fz_readbyte               0046582c f    CIL library: CIL module
 0001:0006484c       _pspushbool                0046584c f    CIL library: CIL module
 0001:00064890       _pspushint                 00465890 f    CIL library: CIL module
 0001:000648d5       _pspushreal                004658d5 f    CIL library: CIL module
 0001:0006491c       _pspopbool                 0046591c f    CIL library: CIL module
 0001:00064970       _pspopint                  00465970 f    CIL library: CIL module
 0001:000649c4       _pspopnum                  004659c4 f    CIL library: CIL module
 0001:00064a39       _pstopisint                00465a39 f    CIL library: CIL module
 0001:00064a51       _pstoptwoareints           00465a51 f    CIL library: CIL module
 0001:00064a71       _pstoptwoarenums           00465a71 f    CIL library: CIL module
 0001:00064a9f       _pscopy                    00465a9f f    CIL library: CIL module
 0001:00064af7       _psroll                    00465af7 f    CIL library: CIL module
 0001:00064b78       _psindex                   00465b78 f    CIL library: CIL module
 0001:00064bc1       _resizecode                00465bc1 f    CIL library: CIL module
 0001:00064c12       _parsecode                 00465c12 f    CIL library: CIL module
 0001:0006517a       _loadpostscriptfunc        0046617a f    CIL library: CIL module
 0001:00065252       _evalpostscriptfunc        00466252 f    CIL library: CIL module
 0001:0006713a       _loadsamplefunc            0046813a f    CIL library: CIL module
 0001:0006760d       _evalsamplefunc            0046860d f    CIL library: CIL module
 0001:0006794a       _loadexponentialfunc       0046894a f    CIL library: CIL module
 0001:00067b32       _evalexponentialfunc       00468b32 f    CIL library: CIL module
 0001:00067c77       _loadstitchingfunc         00468c77 f    CIL library: CIL module
 0001:0006809b       _evalstitchingfunc         0046909b f    CIL library: CIL module
 0001:00068d54       _loadcolorkey              00469d54 f    CIL library: CIL module
 0001:000693db       _maskcolorkey              0046a3db f    CIL library: CIL module
 0001:00069450       _maskcolorkeyindexed       0046a450 f    CIL library: CIL module
 0001:00069865       _clearstack                0046a865 f    CIL library: CIL module
 0001:00069895       _pdf_keepmaterial          0046a895 f    CIL library: CIL module
 0001:000698c8       _pdf_dropmaterial          0046a8c8 f    CIL library: CIL module
 0001:000698ff       _gsave                     0046a8ff f    CIL library: CIL module
 0001:00069962       _grestore                  0046a962 f    CIL library: CIL module
 0001:00069a57       _runxobject                0046aa57 f    CIL library: CIL module
 0001:00069d7d       _runinlineimage            0046ad7d f    CIL library: CIL module
 0001:00069ec6       _runextgstate              0046aec6 f    CIL library: CIL module
 0001:0006a486       _runkeyword                0046b486 f    CIL library: CIL module
 0001:0006cee7       _fz_peekbyte               0046dee7 f    CIL library: CIL module
 0001:0006cee7       _fz_peekbyte               0046dee7 f    CIL library: CIL module
 0001:0006cee7       _fz_peekbyte               0046dee7 f    CIL library: CIL module
 0001:0006cf01       _isregular                 0046df01 f    CIL library: CIL module
 0001:0006cf01       _isregular                 0046df01 f    CIL library: CIL module
 0001:0006cf48       _isnumber                  0046df48 f    CIL library: CIL module
 0001:0006cf68       _fromhex                   0046df68 f    CIL library: CIL module
 0001:0006cf8f       _lexname                   0046df8f f    CIL library: CIL module
 0001:0006d00f       _lexstring                 0046e00f f    CIL library: CIL module
 0001:0006d13b       _lexhexstring              0046e13b f    CIL library: CIL module
 0001:0006d1bb       _pdf_tokenfromkeyword      0046e1bb f    CIL library: CIL module
 0001:0006d69d       _pdf_lookupdestimp         0046e69d f    CIL library: CIL module
 0001:0006d88c       _iswhite                   0046e88c f    CIL library: CIL module
 0001:0006d88c       _iswhite                   0046e88c f    CIL library: CIL module
 0001:0006d88c       _iswhite                   0046e88c f    CIL library: CIL module
 0001:0006d8b0       _loadversion               0046e8b0 f    CIL library: CIL module
 0001:0006d982       _readstartxref             0046e982 f    CIL library: CIL module
 0001:0006dacf       _readoldtrailer            0046eacf f    CIL library: CIL module
 0001:0006dd90       _readnewtrailer            0046ed90 f    CIL library: CIL module
 0001:0006dde1       _readtrailer               0046ede1 f    CIL library: CIL module
 0001:0006ded1       _readoldxref               0046eed1 f    CIL library: CIL module
 0001:0006e21f       _readnewxrefsection        0046f21f f    CIL library: CIL module
 0001:0006e3b4       _readnewxref               0046f3b4 f    CIL library: CIL module
 0001:0006e6c2       _readxref                  0046f6c2 f    CIL library: CIL module
 0001:0006e7d2       _readxrefsections          0046f7d2 f    CIL library: CIL module
 0001:0006ec11       _pdf_loadxref2             0046fc11 f    CIL library: CIL module
 0001:0006ee0b       _runone                    0046fe0b f    CIL library: CIL module
 0001:0006eeb0       _runmany                   0046feb0 f    CIL library: CIL module
 0001:0006f0a2       _loadpagecontents          004700a2 f    CIL library: CIL module
 0001:0006f56a       _getpagecount              0047056a f    CIL library: CIL module
 0001:0006f888       _getpageobject             00470888 f    CIL library: CIL module
 0001:00070e08       _parseobj                  00471e08 f    CIL library: CIL module
 0001:000711ff       _pdf_repairxref2           004721ff f    CIL library: CIL module
 0001:0007182c       _preloadcolorspace         0047282c f    CIL library: CIL module
 0001:000718db       _preloadpattern            004728db f    CIL library: CIL module
 0001:000719b3       _preloadxobject            004729b3 f    CIL library: CIL module
 0001:00071b16       _preloadfont               00472b16 f    CIL library: CIL module
 0001:00071b75       _preloadmask               00472b75 f    CIL library: CIL module
 0001:00071bd5       _scanfontsandmasks         00472bd5 f    CIL library: CIL module
 0001:00071d2e       _copyresolved              00472d2e f    CIL library: CIL module
 0001:0007215e       _pdf_loadcompositeshadefunc 0047315e f    CIL library: CIL module
 0001:0007221c       _pdf_loadcomponentshadefunc 0047321c f    CIL library: CIL module
 0001:0007250e       _loadshadedict             0047350e f    CIL library: CIL module
 0001:00073716       _buildannulusmesh          00474716 f    CIL library: CIL module
 0001:00073ca3       _growshademesh             00474ca3 f    CIL library: CIL module
 0001:0007424f       _getdata                   0047524f f    CIL library: CIL module
 0001:00074ac4       _midcolor                  00475ac4 f    CIL library: CIL module
 0001:00074ae2       _filltensorinterior        00475ae2 f    CIL library: CIL module
 0001:00074cbf       _split_curve_s             00475cbf f    CIL library: CIL module
 0001:00074df2       _split_patch               00475df2 f    CIL library: CIL module
 0001:00074eda       _split_stripe              00475eda f    CIL library: CIL module
 0001:00074fc8       _setvertex                 00475fc8 f    CIL library: CIL module
 0001:00074ff4       _triangulatepatch          00475ff4 f    CIL library: CIL module
 0001:000750d1       _drawstripe                004760d1 f    CIL library: CIL module
 0001:00075182       _drawpatch                 00476182 f    CIL library: CIL module
 0001:00075bee       _kindstr                   00476bee f    CIL library: CIL module
 0001:00075c52       _keepitem                  00476c52 f    CIL library: CIL module
 0001:00075c8e       _dropitem                  00476c8e f    CIL library: CIL module
 0001:0007607d       _buildonefilter            0047707d f    CIL library: CIL module
 0001:000766c0       _buildfilterchain          004776c0 f    CIL library: CIL module
 0001:0007679b       _buildrawfilter            0047779b f    CIL library: CIL module
 0001:00076928       _pdf_buildfilter           00477928 f    CIL library: CIL module
 0001:00076c31       _loadcharproc              00477c31 f    CIL library: CIL module
 0001:00077eb8       _streq                     00478eb8 f    CIL library: CIL module
 0001:00077ee5       _fontnamematches           00478ee5 f    CIL library: CIL module
 0001:00077f49       _lookupcompare             00478f49 f    CIL library: CIL module
 0001:00077f84       _sortcompare               00478f84 f    CIL library: CIL module
 0001:00077fa8       _localbsearch              00478fa8 f    CIL library: CIL module
 0001:0007803e       _removeredundancy          0047903e f    CIL library: CIL module
 0001:000780d9       _finddefaultsubstitutes    004790d9 f    CIL library: CIL module
 0001:00078136       _decodeunicodeBMP          00479136 f    CIL library: CIL module
 0001:00078222       _decodemacintoshplatform   00479222 f    CIL library: CIL module
 0001:00078280       _growfontlist              00479280 f    CIL library: CIL module
 0001:00078300       _insertmapping             00479300 f    CIL library: CIL module
 0001:000783ab       _parseTTF                  004793ab f    CIL library: CIL module
 0001:00078830       _parseTTFs                 00479830 f    CIL library: CIL module
 0001:00078874       _parseTTCs                 00479874 f    CIL library: CIL module
 0001:00078a69       _pdf_createfontlistMS      00479a69 f    CIL library: CIL module
 0001:00078d05       _lookupwindowsfont         00479d05 f    CIL library: CIL module
 0001:00078dfc       _lookupcidfont             00479dfc f    CIL library: CIL module
 0001:00078e49       _lookupsystemsubstitutefont 00479e49 f    CIL library: CIL module
 0001:00078f83       _loadbuiltinsubstitutefont 00479f83 f    CIL library: CIL module
 0001:000790e7       _loadsubstitutefont        0047a0e7 f    CIL library: CIL module
 0001:0007915d       _loadwindowsfont           0047a15d f    CIL library: CIL module
 0001:000796e9       _pdf_cmaptokenfromkeyword  0047a6e9 f    CIL library: CIL module
 0001:0007992a       _codefromstring            0047a92a f    CIL library: CIL module
 0001:00079947       _lexcmap                   0047a947 f    CIL library: CIL module
 0001:00079994       _parsecmapname             0047a994 f    CIL library: CIL module
 0001:00079a2f       _parsewmode                0047aa2f f    CIL library: CIL module
 0001:00079ac7       _parsecodespacerange       0047aac7 f    CIL library: CIL module
 0001:00079bd2       _parsecidrange             0047abd2 f    CIL library: CIL module
 0001:00079d78       _parsecidchar              0047ad78 f    CIL library: CIL module
 0001:00079e95       _parsebfrangearray         0047ae95 f    CIL library: CIL module
 0001:00079fbe       _parsebfrange              0047afbe f    CIL library: CIL module
 0001:0007a268       _parsebfchar               0047b268 f    CIL library: CIL module
 0001:0007a6ce       _bio_bytein                0047b6ce f    CIL library: CIL module
 0001:0007a87f       _dwt_decode_1_             0047b87f f    CIL library: CIL module
 0001:0007a9f8       _dwt_decode_max_resolution 0047b9f8 f    CIL library: CIL module
 0001:0007aa21       _dwt_decode_tile           0047ba21 f    CIL library: CIL module
 0001:0007ac6a       _v4dwt_interleave_h        0047bc6a f    CIL library: CIL module
 0001:0007ad43       _v4dwt_interleave_v        0047bd43 f    CIL library: CIL module
 0001:0007adba       _v4dwt_decode_step1        0047bdba f    CIL library: CIL module
 0001:0007adf0       _v4dwt_decode_step2        0047bdf0 f    CIL library: CIL module
 0001:0007aebf       _v4dwt_decode              0047bebf f    CIL library: CIL module
 0001:0007b345       _j2k_read_soc              0047c345 f    CIL library: CIL module
 0001:0007b37c       _j2k_read_siz              0047c37c f    CIL library: CIL module
 0001:0007b620       _j2k_read_com              0047c620 f    CIL library: CIL module
 0001:0007b638       _j2k_read_cox              0047c638 f    CIL library: CIL module
 0001:0007b7ca       _j2k_read_cod              0047c7ca f    CIL library: CIL module
 0001:0007b8d0       _j2k_read_coc              0047c8d0 f    CIL library: CIL module
 0001:0007b93b       _j2k_read_qcx              0047c93b f    CIL library: CIL module
 0001:0007ba19       _j2k_read_qcd              0047ca19 f    CIL library: CIL module
 0001:0007ba6e       _j2k_read_qcc              0047ca6e f    CIL library: CIL module
 0001:0007baad       _j2k_read_poc              0047caad f    CIL library: CIL module
 0001:0007bba6       _j2k_read_crg              0047cba6 f    CIL library: CIL module
 0001:0007bbd7       _j2k_read_tlm              0047cbd7 f    CIL library: CIL module
 0001:0007bc45       _j2k_read_plm              0047cc45 f    CIL library: CIL module
 0001:0007bc91       _j2k_read_plt              0047cc91 f    CIL library: CIL module
 0001:0007bcc1       _j2k_read_ppm              0047ccc1 f    CIL library: CIL module
 0001:0007bd8b       _j2k_read_ppt              0047cd8b f    CIL library: CIL module
 0001:0007be53       _j2k_read_sot              0047ce53 f    CIL library: CIL module
 0001:0007c08f       _j2k_read_sod              0047d08f f    CIL library: CIL module
 0001:0007c1a8       _j2k_read_rgn              0047d1a8 f    CIL library: CIL module
 0001:0007c214       _j2k_read_eoc              0047d214 f    CIL library: CIL module
 0001:0007c338       _j2k_read_unk              0047d338 f    CIL library: CIL module
 0001:0007c34f       _j2k_dec_mstab_lookup      0047d34f f    CIL library: CIL module
 0001:0007c793       _jp2_read_boxhdr           0047d793 f    CIL library: CIL module
 0001:0007c80e       _jp2_read_ihdr             0047d80e f    CIL library: CIL module
 0001:0007c8bd       _jp2_read_bpcc             0047d8bd f    CIL library: CIL module
 0001:0007c938       _jp2_read_colr             0047d938 f    CIL library: CIL module
 0001:0007caa3       _jp2_read_ftyp             0047daa3 f    CIL library: CIL module
 0001:0007cb48       _jp2_read_jp2c             0047db48 f    CIL library: CIL module
 0001:0007cb9b       _jp2_read_struct           0047db9b f    CIL library: CIL module
 0001:0007ce05       _mqc_bytein                0047de05 f    CIL library: CIL module
 0001:0007ce58       _mqc_renormd               0047de58 f    CIL library: CIL module
 0001:0007cf3c       _pi_next_lrcp              0047df3c f    CIL library: CIL module
 0001:0007d005       _pi_next_rlcp              0047e005 f    CIL library: CIL module
 0001:0007d0ce       _pi_next_rpcl              0047e0ce f    CIL library: CIL module
 0001:0007d45b       _pi_next_pcrl              0047e45b f    CIL library: CIL module
 0001:0007d800       _pi_next_cprl              0047e800 f    CIL library: CIL module
 0001:0007e0bc       _t1_updateflags            0047f0bc f    CIL library: CIL module
 0001:0007e112       _t1_dec_sigpass_step       0047f112 f    CIL library: CIL module
 0001:0007e1d9       _t1_dec_sigpass            0047f1d9 f    CIL library: CIL module
 0001:0007e291       _t1_dec_refpass_step       0047f291 f    CIL library: CIL module
 0001:0007e306       _t1_dec_refpass            0047f306 f    CIL library: CIL module
 0001:0007e3d1       _t1_dec_clnpass_step       0047f3d1 f    CIL library: CIL module
 0001:0007e473       _t1_dec_clnpass            0047f473 f    CIL library: CIL module
 0001:0007e689       _allocate_buffers          0047f689 f    CIL library: CIL module
 0001:0007e724       _t1_decode_cblk            0047f724 f    CIL library: CIL module
 0001:0007ec43       _t2_init_seg               0047fc43 f    CIL library: CIL module
 0001:0007ecaf       _t2_decode_packet          0047fcaf f    CIL library: CIL module
 0001:000810a0       _flsall                    004820a0 f   LIBCMT:fflush.obj
 0001:00082210       _swap                      00483210 f   LIBCMT:qsort.obj
 0001:00082240       _shortsort                 00483240 f   LIBCMT:qsort.obj
 0001:00082a48       __initterm                 00483a48 f   LIBCMT:crt0dat.obj
 0001:00082b85       _doexit                    00483b85 f   LIBCMT:crt0dat.obj
 0001:00082cf3       _vscan_fn                  00483cf3 f   LIBCMT:sscanf.obj
 0001:000836de       ?strtoxl@@YAKPAUlocaleinfo_struct@@PBDPAPBDHH@Z 004846de f   LIBCMT:strtol.obj
 0001:00083d21       _fast_error_exit           00484d21 f   LIBCMT:crt0.obj
 0001:00083d45       _check_managed_app         00484d45 f   LIBCMT:crt0.obj
 0001:00083d86       ___tmainCRTStartup         00484d86 f   LIBCMT:crt0.obj
 0001:000856a2       _write_char                004866a2 f   LIBCMT:output.obj
 0001:000856d5       _write_multi_char          004866d5 f   LIBCMT:output.obj
 0001:000856f9       _write_string              004866f9 f   LIBCMT:output.obj
 0001:0008626b       __use_encode_pointer       0048726b f   LIBCMT:tidtable.obj
 0001:000874c0       __unwind_handler4          004884c0 f   LIBCMT:exsup4.obj
 0001:00088603       _fastcopy_I                00489603 f   LIBCMT:p4_memcpy.obj
 0001:000887a4       __unwind_handler           004897a4 f   LIBCMT:exsup.obj
 0001:000889a5       __onexit_nolock            004899a5 f   LIBCMT:onexit.obj
 0001:00088e4d       _siglookup                 00489e4d f   LIBCMT:winsig.obj
 0001:0008905c       ___crtInitCritSecNoSpinCount@8 0048a05c f   LIBCMT:initcrit.obj
 0001:000891cb       ___check_float_string      0048a1cb f   LIBCMT:input.obj
 0001:0008921f       __inc                      0048a21f f   LIBCMT:input.obj
 0001:00089235       __whiteout                 0048a235 f   LIBCMT:input.obj
 0001:0008af38       ?CPtoLCID@@YAHH@Z          0048bf38 f   LIBCMT:mbctype.obj
 0001:0008af67       ?setSBCS@@YAXPAUthreadmbcinfostruct@@@Z 0048bf67 f   LIBCMT:mbctype.obj
 0001:0008afbc       ?setSBUpLow@@YAXPAUthreadmbcinfostruct@@@Z 0048bfbc f   LIBCMT:mbctype.obj
 0001:0008b1ea       ?getSystemCP@@YAHH@Z       0048c1ea f   LIBCMT:mbctype.obj
 0001:0008b847       __updatetlocinfoEx_nolock  0048c847 f   LIBCMT:setlocal.obj
 0001:0008c941       ?__crtLCMapStringA_stat@@YAHPAUlocaleinfo_struct@@KKPBDHPADHHH@Z 0048d941 f   LIBCMT:a_map.obj
 0001:0008ce90       _parse_cmdline             0048de90 f   LIBCMT:stdargv.obj
 0001:0008d9d1       __tsopen_nolock            0048e9d1 f   LIBCMT:open.obj
 0001:0008e677       _fastzero_I                0048f677 f   LIBCMT:p4_memset.obj
 0001:0008e75d       _has_osfxsr_set            0048f75d f   LIBCMT:cpu_disp.obj
 0001:0008ebdd       ?__crtCompareStringA_stat@@YAHPAUlocaleinfo_struct@@KKPBDH1HH@Z 0048fbdd f   LIBCMT:a_cmp.obj
 0001:0008f09e       _findenv                   0049009e f   LIBCMT:setenv.obj
 0001:0008f0eb       _copy_environ              004900eb f   LIBCMT:setenv.obj
 0001:0008f4f2       __shift                    004904f2 f   LIBCMT:cvt.obj
 0001:0008f52b       __cftoe2_l                 0049052b f   LIBCMT:cvt.obj
 0001:0008faf5       __cftof2_l                 00490af5 f   LIBCMT:cvt.obj
 0001:0008fee4       ?__crtGetStringTypeA_stat@@YAHPAUlocaleinfo_struct@@KPBDHPAGHHH@Z 00490ee4 f   LIBCMT:a_str.obj
 0001:000911fc       ?x_ismbbtype_l@@YAHPAUlocaleinfo_struct@@IHH@Z 004921fc f   LIBCMT:ismbbyte.obj
 0001:00092437       __hw_cw                    00493437 f   LIBCMT:ieee87.obj
 0001:000924c5       ___hw_cw_sse2              004934c5 f   LIBCMT:ieee87.obj
 0001:0009286e       __hypothlp                 0049386e f   LIBCMT:hypot.obj
